:100000000C94DB180D9414140D94E9130D94BE1385
:100010000D9493130D9468130D943D130D941213C6
:100020000D94E7120C940C190C940C190C940C19E7
:100030000C940C190C940C190C940C190D942A2B7B
:100040000C940C190C940C190C940C190C940C199C
:100050000C940C190C940C190C940C190D9452114D
:100060000C940C190D947A170D9450170C940C19CC
:100070000C940C190C940C190C940C190C940C196C
:100080000C940C190C940C190C940C190C940C195C
:100090000D94A6190D941C190D945E190D94CF2C76
:1000A0000C940C190C940C190C940C190C940C193C
:1000B0000C940C190C940C190C940C190C940C192C
:1000C0000C940C190C940C190C940C190D94261703
:1000D0000D94FC160C940C190D94D2160D94A816C0
:1000E0000C940C1907634236B79BD8A71A39685687
:1000F00018AEBAAB558C1D3CB7CC5763BD6DEDFD4A
:10010000753EF6177231BF000000803F0800000006
:10011000BE922449123EABAAAA2ABECDCCCC4C3EFC
:1001200000000080BEABAAAAAA3E00000000BF00EB
:100130000000803F0000000000084178D3BB4387E7
:10014000D1133D190E3CC3BD4282AD2B3E68EC82FB
:1001500076BED98FE1A93E4C80EFFFBE01C4FF7F80
:100160003F00000000000C94FB410C9496D90C94C5
:10017000EA7E0C94B8990C9455F00D94E5210C94FA
:10018000D2A50C94F6710C946D3F0D94240F0C9431
:10019000C4A50C94A5A50C943FE60C94B9E60C9468
:1001A000022A0C94FE7A0C94C9700C947FE60C948D
:1001B00096700C9401A10C946CE60C94F9D90C94F3
:1001C000CCDD0C94485A0C9465E90C94ACEF0C947B
:1001D000C1B90C941B720C94BBE60C94AE510C94F8
:1001E0001CF60C94A0A80C9466720C9471250C94C7
:1001F000E3670C943EBD0C9455A50C94FF990C94A8
:10020000E9E00C947EA50C94EC3A0C942D1F0C9410
:10021000181A0C944CE10C94AD410C9429320C94B6
:100220008ED90C941C430C941CAF0C9479C40C9480
:1002300056BE0C94E77E0D9434100C9463BD0C9460
:100240004FBD0C941C7B0C94B6430C94BF510D9481
:100250000B1F0C94BD7A0C94B97D0C9484650C949E
:1002600083E00C94FA720C9454230D941F0D0C949B
:10027000ED6C0C94343B0C941BF00C94F4A50C9492
:1002800044DD0C94C7810C9476E10C943B1C0D94D6
:10029000A01F0D94F30E0C94117B0C949BE20C9414
:1002A0005D9F0C9460E30C94D8A30C946AC40C94E6
:1002B00026F60C946B9F0C9470E10C94A6590C9448
:1002C0009A510C94641F0C9411DA0C943D1C0D94FB
:1002D000AD0F0C94ABBE0C9450800C94391C0C9454
:1002E000331C0C9467BD0C94151A0D94720E0C946B
:1002F00097BE0C946B7B0C94D6340D9410230C9405
:1003000047E00C94FBD90C94537F0C940CDE0C94B6
:1003100048800C94823A0C94FB510C9420820C94EB
:1003200064F50C9430E00D9415150C9408E00C94D1
:10033000D0A10D944E0F0C94FB240D946B0D0C94D6
:100340001F330C944BBD0C9407DD0D949C0E0C9444
:10035000D8DF0C9491590C9474A50C948DBE0C9418
:10036000B8340C9488F00D9451220C94DA190C9442
:1003700060BE0C94FED90D94B01E0C9484740C9441
:10038000EDA00C9429F50D94170E0C945AE60C94DC
:1003900077A10C94854A0C94F3B80C94817A0C9450
:1003A00025190C94F2A50C9451E60C943ADA0D94AC
:1003B000430E0C9469740C94AF350C94DEE50C94E8
:1003C000891F0C940DA40C94877B0D94260E0C941D
:1003D00092D90C9422660C94F5D90C94EAE60D940B
:1003E00069230C94EFDD0C949E1A0D941C310C942F
:1003F000581A0C94A2D90C94D0B80C94DA360D94F7
:1004000031310C94A2990D94380F0C9474BE0C9455
:100410009AD90C94F2DD0C9447BA0C94FBA40C947A
:1004200036BD0D94A60C0C94FFE10C9492210C9413
:10043000803A0C9470270C9494430C943F1C0C94B9
:10044000B3A50C9475DA0D94FF150C9448DA0C944E
:100450000A740C944FA10C94892F0C94451C0C9495
:10046000B0710D94E40E0C9425A00C943B510C94A7
:100470006BBD0C94833A0C9433AF0C9442800C9473
:10048000A5DD0C94F3A30C94E3DD0C94E0E10C9453
:10049000841A0C94AFE60C949E7A0C94C9B80D940F
:1004A00033230C943CBE0C94CD670C940F660C94D3
:1004B000A2E00C9465350C94B1350C9487360D94FC
:1004C000042A0C9422A10C94323B0C94471C0C94EB
:1004D00054DB0C94D7710C949FF40C942FA40C94BF
:1004E000927A0C9446BE0D94AE0E0C94F1190C94B5
:1004F000DBA40C9470340C9441680C947BEF0C9446
:10050000CCA40D9405100C94B9710D94640E0C9448
:10051000EE7A0C942DA50C9400DE0C9442BD0C9444
:1005200098A50C9473DA0D94E9210C9445BD0D94B3
:10053000AE0F0C9407660C94EDE60D94580F0D94D5
:100540005A0F0C945F720D942F0F0C940E2C0C9478
:10055000351C0C9408250C94B9E00C94BEF70C944F
:10056000E4660C94091B0C94D0710C944F3A0C94D3
:1005700092BA0C943ABD0C94E2D90C9438A00D9424
:100580009B230C94DEF40D94A70C0C94F2910C9424
:1005900021670C9492E60C9422410C94B8D90C94E7
:1005A000941F0C94AB350C949EF50C9440A50C94C0
:1005B0002D230C94E9410C941A740D94D80F0D94CA
:1005C000BE0F0C945A7F0D94D10F0C9448730C9469
:1005D0000C720C9489230C94C1DF0C94BDF50C941F
:1005E00051260C946BC40C94431C0C94AD240C94B5
:1005F0001B1A0D94782A0C944EBE0C94026C0C9429
:10060000B9DD0C94FD710C9429A60D94EE0C0D949B
:10061000B8100C94BF2A0D94A50C0C94C9650C94C9
:1006200049A60C94DCAE0D9443110C943F1A0C9423
:10063000A7B90C9432BE0C94C2700C949B350C94E8
:100640000B660C94D9A40D94811F0C94D7B80C940C
:1006500012F60D94C3260C9458470D940D0F0C946C
:10066000B91F0C9400230C94D8B90C9475BD0C944C
:10067000A1BE0D94370F0C94C2B80C942F190D9491
:10068000C81E0C944D5A0C94B3350C9486440C94AB
:100690009F360C94D7510C94A0740D942E0C0C948E
:1006A000D8D90C945DBD0C94BBA10C94D25C0C9475
:1006B000D5AE0C9403720C9485510C944B800D9420
:1006C00054100C9439710D94B50E0C945FE90C9490
:1006D000BFA50C94CC190D94110D0C943C710C9485
:1006E000EFF50C94F6210C9459BD0C94FDAE0C94CE
:1006F0001BBE0C9450720C947B430C9449E10C94F7
:100700006ABE0D94AF0F0C9453A20C940BA50C94DD
:100710004A240C94C8710C9423BE0C94C16D0C94A3
:10072000411C0C9470BD0C9407710C944D1A0C94E0
:1007300071BD0C94C0F70C94FDDD0C9425A40C94B1
:10074000C12B0C94E5B80C9419510C9460510C9485
:1007500054350C94B5BE0C94371C0D94A80C0C9415
:1007600056890D94B80D0C94B0A40C941E1A0C94D8
:10077000A5E60C9428190C9445720D94FD0C0C946C
:1007800056E90C9455BD0C9436730C94D59D0C947D
:1007900034670C943AF60D94DB220C949AA40C94D2
:1007A000B8B90C94E5A00C9459440C949D730C9426
:1007B000F4190C944FE10C94A6D90C94C4F70C9442
:1007C000BE200C94ACE10C94CD350C94D2650D9404
:1007D000DB1C0C94E4400C9428BE0C943BDA0C9483
:1007E00045800C94E0650D94CA1F0C9483BE0C9454
:1007F00091360C94813A0C94FB340C94A4240C9400
:1008000010A40C949ED90C943CDE0C94BD190D944C
:10081000090F0C94EEAE0C94595A0C94333B0D9482
:100820006C100C94D6F50C9493310D94C8290C944B
:10083000F07E0C94421A0D9450260C943A720C944B
:10084000ECB80D941D0F0C9490DF0C9430BD0C94FB
:100850001E730C9448E60C94B1500C942C440C94E8
:100860008B2C0D94C2220C94F2630C949B990C94E3
:10087000AC7A0C9459BA0C945EDF0C945CA10C9485
:1008800019350C9424DA0C9451410C9443980C942F
:100890007CC40C9445280C94A5560C9443620C948B
:1008A00034A10C94C31A4E414E494E495459494EF5
:1008B00046CDCCCC3D0AD7233C17B7D13877CC2BCB
:1008C000329595E6241FB14F0A000020410000C870
:1008D0004200401C4620BCBE4CCA1B0E5AAEC59DF1
:1008E000746364696E6F70737578585B00204F464F
:1008F0004600204F4E00204259504153530053614F
:1009000076656420746F20454550524F4D00536109
:1009100076696E6720636F6E66696720746F204525
:100920004550524F4D2E2E004343533831313A201B
:10093000416C726561647920696E697469616C6982
:100940007A6564004343533831313A20496E697403
:10095000206572726F7220004343533831313A2060
:10096000496E697400484443313038303A20416C54
:10097000726561647920696E697469616C697A6510
:1009800064004465766963652053657269616C2013
:100990004E756D6265723D00204465766963652021
:1009A00049443D3078004D616E75666163747572BF
:1009B00065722049443D3078004844433130383036
:1009C0003A20496E69742E2000432C2052483D0085
:1009D000484443313038303A205374617475733D64
:1009E00000484443313038303A204E6F7420696EED
:1009F000697469616C697A6564004D7367496E76E4
:100A0000616C69640052656164526567496E766124
:100A10006C6964004D6561734D6F6465496E766104
:100A20006C6964004D6178526573697374616E63BB
:100A300065004865617465724661756C740048654F
:100A400061746572537570706C790043435338312B
:100A5000313A204572726F7220004343533831316E
:100A60003A204661696C656420746F206765742064
:100A70004552524F525F49442072656769737465ED
:100A8000722E005D20626173656C696E655B005D4E
:100A90002074564F435B0020434F325B0063637307
:100AA0003831313A2064617461206E6F7420617650
:100AB00061696C61626C6500636373383131206E0B
:100AC0006F7420696E697469616C697A656400206D
:100AD0003C3C0041433A200041433A20536572694F
:100AE000616C2075736564206279204143202D205C
:100AF00064697361626C696E672073657269616CA9
:100B0000206C6F6767696E6720616E6420636D6437
:100B10000041433A204F7574206F66206D656D6FFC
:100B200072790041433A20496E69743A200041438A
:100B30003A2044652D496E69743A200045525200AE
:100B400041433A204F4B00203E3E200041433A2093
:100B50000041433A20506F6C6C696E670041433A24
:100B600020556E6D757465000000000000000000E7
:100B7000004F4E000000000000004F4646000000FD
:100B8000000000524553540000000000544F4747F6
:100B90004C4500000048414C540000000000584FF4
:100BA0004E000000000000584F46460000000000C4
:100BB000494E4352454153450044454352454153F4
:100BC0004500454E41424C450000004449534142D6
:100BD0004C450000554E465245455A450046524543
:100BE000455A450000004155544F000000000046A2
:100BF000414E5F4F4E4C59004849474800000000A5
:100C0000004D454449554D0000004C4F5700000031
:100C1000000000484541540000000000434F4F4C85
:100C2000000000000044525900000000000053542E
:100C30004F5000000000005247420000000000003A
:100C4000485356000000000000726177007175651E
:100C50006974007377696E67006C6F636B00556E23
:100C60006B6E6F776E207375666669782000556EBF
:100C70006B6E6F776E20636D642000436F756E74CA
:100C800065723A2000444D582D4F757420496E69A5
:100C9000743A2000444D582D4F75742073746F7052
:100CA0003A200041737369676E65643A00444D5899
:100CB000206374726C3A2000693136000169333266
:100CC000000275313600037533320004693868005C
:100CD0000569386C0006753868000775386C0008BF
:100CE0007831300009313030000A44656661756C36
:100CF000742073657269616C206D6F6465204E3875
:100D000031207573656400384531002600384E3156
:100D1000000600384532002E00384E32000E0038F2
:100D20004F31003600384F32003E00374531002445
:100D300000374532002C00374F31003400374F3236
:100D4000003C00374E31000400374E32000C004D9D
:100D50004255533A204D6F646275732074656D700F
:100D60006C617465206E6F7420666F756E643A20D6
:100D7000004D4255533A20496E76616C6964207487
:100D8000656D706C6174652E002C002C002C002C9D
:100D9000004D4255533A20636F6E66696720666165
:100DA000696C65643A004D4255533A20636F6E6634
:100DB0006967206572726F72004D4255533A206325
:100DC0006F6E666967206C6F6164656420004D42D8
:100DD00055533A204F7574206F66206D656D6F72A4
:100DE00079004D4255533A20506F6C6C696E672004
:100DF0006572726F7220004D4255533A204E6F74E7
:100E000020737570706F72746564207265672074EA
:100E10007970650A004D425553443A2049676E6F18
:100E2000726564202D20657175616C207769746826
:100E3000207365747465642076616C004D4255536F
:100E40003A204164642040533A20004D42555344B7
:100E50003A204D61707065643A004D425553443AF2
:100E6000204E65737465644D61707065643A004C22
:100E70006173744B6E6F776E2076616C75653A2086
:100E800000536561726368696E67207265673A2016
:100E900000206F7574206F662072616E6765206236
:100EA00075666665722C206665746368696E670096
:100EB000646566207265672320004D425553443AAD
:100EC00020536561726368696E67207265672300ED
:100ED0003A002066726F6D207479706520004D4273
:100EE0005553443A2020676F7420002076616C3A95
:100EF0000020004D425553207265733A2000207641
:100F0000616C206E6F74206368616E6765642E206B
:100F1000436F6E74696E7565004D4255533A003AE1
:100F200020657175616C20746172676572742E0042
:100F30003D004D4255533A002076616C2063686154
:100F40006E6765642E004D4255533A00204E6F7710
:100F50003A00204C6173743A0020230020707265BF
:100F600066657463682000205265672F636F696C43
:100F7000206D75737420626520696E740020696E3F
:100F80007465726E616C2073656E64206572726F39
:100F900072202D206E6F207265672F636F696C0061
:100FA00020696E7465726E616C2073656E64206575
:100FB00072726F72202D206E6F2074656D706C617F
:100FC00074650020696E7465726E616C2073656E65
:100FD00064206572726F72202D206E6F2073746FA3
:100FE0007265004D425553443A20656E64506F6CF3
:100FF0006C20004D425553443A20506F6C6C2000D9
:10100000206E6F7420666F756E64004D4255533AC2
:101010002020706172616D20002073656E64696EBE
:10102000672063616E63656C6C6564004D42555367
:101030003A2020706172616D20002073656E64201B
:101040006572726F722E20004D4255533A20200077
:101050004164642040563A20002056616C3A2000DA
:101060004D425553443A207375666669783A0020BC
:101070006F722073756666697820004D4255533A49
:10108000204E6F2074656D706C61746520666F72A0
:1010900020004D6F746F723A2074696D656F7574BE
:1010A00000556E6B6E6F776E20636D64004D6F74CC
:1010B0006F723A20466F7263656420657865637568
:1010C00074696F6E0056454E543A20636F6E6669C0
:1010D00067206661696C65640056454E543A206924
:1010E0006E69740056454E543A2044652D496E6928
:1010F0007400204F75743A00205265713A005645CD
:101100004E543A2000206D33002066726F6D20002F
:10111000204D6178207265713A002066616E253A33
:10112000002061637469766520563A0056454E5436
:101130003A20546F74616C20563A005049443A206A
:10114000616C726561647920696E697469616C694A
:101150007A6564005049443A20496E76616C69644E
:1011600020706172616D2061727261792E002C00B5
:101170002C002C002C005049443A20636F6E6669A5
:1011800067206661696C65643A005049443A20639F
:101190006F6E666967206572726F72005049443ADB
:1011A00020636F6E666967206C6F61646564200000
:1011B0005049443A204F7574206F66206D656D6FFD
:1011C0007279005049443A2044652D496E69742073
:1011D00000203C414C4D3E0020443A0020493A005A
:1011E00020503A0020696E3A00207365743A00502E
:1011F00049443A20005049443A20496E76616C696E
:101200006420706172616D2061727261792E005389
:101210006574206F757420746F200020504944203D
:10122000616C61726D2E20002050494420616C6118
:10123000726D3A20636C6F736564005049443A20C4
:10124000556E6B6E6F776E207375666669782000D9
:101250005049443A20556E6B6E6F776E20636D6413
:10126000200020536574706F696E743A00504944D1
:101270003A200020496E7075742076616C75653A6D
:10128000005049443A200020696E697400200050E3
:10129000574D2D4F75742023002073746F700020FC
:1012A0000050574D2D4F75742023003D0050696E3E
:1012B0003A0020696E69740052656C61792D4F7532
:1012C000742023002073746F700052656C61792D57
:1012D0004F75742023003D3E003A00707562206116
:1012E0006374696F6E200069646C65006F666600E8
:1012F00068656174696E670066616E006472796921
:101300006E6700636F6F6C696E6700206973200001
:101310004F75742000556E6B6E6F776E2073756617
:101320006669782000556E6B6E6F776E20636D6412
:101330002000616374696F6E0072656C617943743B
:10134000723A200053686F770020636D643D002D72
:10135000005B305D3A2000202D202D202D20EFBB9A
:10136000BF003E003E31202D200000000000006341
:101370006D640000736574000076616C0000646544
:101380006C00004853560000524742000066616EF0
:1013900000006D6F6465006374726C0068756500B1
:1013A00000736174000074656D70007261770000F5
:1013B00020002E00696E00735F6F7574006D796890
:1013C0006F6D65004354524C2F657865633A204F2A
:1013D00075744F664D656D6F72793A2000202D3E11
:1013E00020004D5154543A2000202D3E2000456DE0
:1013F00069743A203C00202D3E20004974656D43FD
:101400006D643A2000202D3E20004974656D3A201D
:10141000003157543A204275732072657365742009
:101420006572726F72003157543A204275732052C0
:101430006573657420646F6E65003157543A2044BB
:1014400053323438322070726573656E742C20729A
:1014500065736574004932432052657365740053A7
:1014600074617475732064656666657265640A00EC
:101470002D3E005075623A20002D3E005075623AB4
:1014800020002D3E005075623A2000000000000050
:10149000636D640000736574000076616C00006425
:1014A000656C0000485356000052474200006661D8
:1014B0006E00006D6F6465006374726C0068756522
:1014C0000000736174000074656D700072617700D4
:1014D000002D3E005075623A20002D3E005075628E
:1014E0003A200053454E445354415455533A2055E5
:1014F0006E6B6E6F776E20636D64200A00000000D3
:101500000000000000004F4E000000000000004FEF
:101510004646000000000000524553540000000001
:1015200000544F47474C4500000048414C540000D0
:10153000000000584F4E000000000000584F464683
:101540000000000000494E435245415345004445C8
:1015500043524541534500454E41424C4500000031
:1015600044495341424C450000554E465245455A68
:101570004500465245455A450000004155544F002C
:101580000000000046414E5F4F4E4C59004849470D
:101590004800000000004D454449554D0000004CF6
:1015A0004F57000000000000484541540000000073
:1015B00000434F4F4C00000000004452590000000F
:1015C00000000053544F50000000000052474200FA
:1015D0000000000000485356000000000000206694
:1015E00061696C65643A004D6F64627573206F7059
:1015F00020004D423A206F6B003D004D423A20568C
:1016000043230020636D643D003D004D423A205667
:10161000435F6865617423004D423A204E6F742029
:10162000737570706F727465642072656720747969
:1016300070650A002056616C3A30780020543A00F8
:10164000205265673A3078004D423A204164647216
:101650003A00444D58000000000000444D585247E5
:1016600042570000444D5852474200000050574D29
:101670000000000000004D42555344494D00005405
:101680004845524D4F00000052454C415900000062
:101690000047524F555000000000564354454D50EE
:1016A0000000004D4255535643000000414348415D
:1016B00049455200005350494C45440000004D4FED
:1016C000544F520000000050494400000000000048
:1016D0004D425553000000000055415254425244BF
:1016E000470052454C415950574D00444D585247C0
:1016F0004257570056454E545300000000454C4594
:101700005641544F5200434F554E544552000048E5
:10171000554D0000000000004D4552435552590000
:101720000020002D3E00436F6E76657274696E670F
:1017300020002D3E0057726F6E67204173736967FA
:101740006E6D656E742000524742783A2000207614
:101750004C6576656C3A0020436F6E76563A0020F1
:10176000436F6E76533A0020486F743A00436F6CB3
:10177000643A0020436F6E76657274656420563A51
:1017800000436F6E76657274656420533A002D3E97
:101790000057726F6E672041737369676E6D656E77
:1017A0007420002D3E0057726F6E6720417373697D
:1017B000676E6D656E742000000000000000000080
:1017C000004F4E000000000000004F4646000000A1
:1017D000000000524553540000000000544F47479A
:1017E0004C4500000048414C540000000000584F98
:1017F0004E000000000000584F4646000000000068
:10180000494E435245415345004445435245415397
:101810004500454E41424C45000000444953414279
:101820004C450000554E465245455A4500465245E6
:10183000455A450000004155544F00000000004645
:10184000414E5F4F4E4C5900484947480000000048
:10185000004D454449554D0000004C4F57000000D5
:10186000000000484541540000000000434F4F4C29
:1018700000000000004452590000000000005354D2
:101880004F500000000000524742000000000000DE
:1018900048535600000000000020537566663A0069
:1018A0002041543A00206973200044656C657469D6
:1018B0006E6720636F6E662E2052414D20776173F4
:1018C0003A0053746F70706564006E6F7468696E6F
:1018D0006720746F2073746F700053746F70706939
:1018E0006E67206368616E6E656C73202E2E2E000D
:1018F00043616E206E6F7420636C65616E202D20D5
:101900006C6F636B6564004D5154543A20436F6DA6
:10191000706C6574652E2052656D6F766520746FEE
:10192000706963200024636F6D6D616E64004D51BA
:1019300054543A20436C65616E5570207265746131
:10194000696E656420746F70696320002200220054
:101950004F75744F664D656D6F727921005D200083
:101960003A5B004D5154543A005D00456D707479F6
:101970003A205B000A003A004D41433A005544507A
:10198000205379736C6F6720696E697469616C6943
:101990007A65642E0A005379736C6F6720706172E8
:1019A000616D733A002E6C6F63616C0053657276E3
:1019B000696365207265636F72643A20006D444EFE
:1019C0005320726573706F6E6465722073746172F8
:1019D0007465642E004572726F7220736574746949
:1019E0006E67207570204D444E5320726573706F82
:1019F0006E6465722100476F7420495020616464F1
:101A0000726573733A00276970205B69705B2C64A0
:101A10006E735B2C67775B2C7375626E65745D5DAE
:101A20005D5D27202D207365742073746174696374
:101A30002049500A004661696C656420746F206318
:101A40006F6E6669677572652045746865726E654C
:101A500074207573696E6720444843502E20596F77
:101A6000752063616E20736574206970206D616EEE
:101A700075616C6C792100204D41534B3A00204731
:101A8000573A0020444E533A004C6F61646564201D
:101A900066726F6D20666C6173682049503A000A67
:101AA0007573657320444843500A0053746172741F
:101AB000696E67206C616E004D5154543A20747207
:101AC0007969796E67206E656E78742062726F6BCB
:101AD0006572004D5154543A20546F6F206D616E01
:101AE0007920636F6E6E656374696F6E20657272C4
:101AF0006F72732E2052657374617274204C414E64
:101B0000002074727920616761696E20696E2035EA
:101B1000207365636F6E6473004D5154543A2066B0
:101B200061696C65642C2072633D004D5154543AD8
:101B3000204177616974696E6720666F72207265F3
:101B40007461696E656420746F7069637300636F9C
:101B50006E6E65637465642061732000202E2E2EE6
:101B60000020757365723A003A000A4D5154543A98
:101B700020417474656D7074696E6720636F6E6E5A
:101B8000656374696F6E20746F2000646973636F9E
:101B90006E6E6563746564005573696E67204D51A0
:101BA00054542070617373776F72642066726F6D26
:101BB00020636F6E666967002E6C6F63616C006DE9
:101BC000444E53206E616D65207570646174656468
:101BD0003A2000446576696365204E616D653A0080
:101BE0004D5154543A204174206C656173742064E3
:101BF0006576696365206E616D6520616E64206243
:101C0000726F6B6572204950206D75737420626528
:101C100020636F6E6669677572656400246E6F6419
:101C20006573004F4E2C4F46462C48414C542C5265
:101C30004553542C584F4E2C584F46462C544F4722
:101C4000474C450024666F726D617400656E756D5A
:101C50000024646174617479706500687376006350
:101C60006F6C6F7200302D32353500696E746567A8
:101C7000657200666C6F617400332E302E31002463
:101C8000686F6D696500757074696D652C66726545
:101C9000656865617000666638393937665F32306D
:101CA00032342D30382D3233004C696768744875F2
:101CB000622000246E616D6500526562696E642069
:101CC000737563636573732E204950206164647279
:101CD0006573733A004572726F723A207265626979
:101CE0006E64206661696C0052656E65776564207C
:101CF000737563636573732E204950206164647249
:101D00006573733A004572726F723A2072656E6540
:101D1000776564206661696C000A4E6F206C696E9D
:101D20006B00436F6E74696E756520776974682007
:101D300070726576696F75736C79206C6F6164651C
:101D40006420636F6E6669670033307320454550C9
:101D5000524F4D206973206E6F742072656C6F61F5
:101D60006465642E205265626F6F74004D51545447
:101D70003A20416363657074696E6720636F6D6DAF
:101D8000616E64732E2E2E0A004E6F204D515454F6
:101D900020636F6E66696775726564004C6F61647D
:101DA000696E6720636F6E6669672066726F6D206B
:101DB000706F7274616C2064697361626C65642E0B
:101DC0002075736520676574204F4E20746F206501
:101DD0006E61626C6500436F6E666967206973208F
:101DE00076616C696400436F6E74696E7565207707
:101DF0006974682070726576696F75736C79206C90
:101E00006F6164656420636F6E6669670053657413
:101E10007570204F5441004D5154543A20736574ED
:101E20002066697273742062726F6B65720043750D
:101E30007272656E74204C414E20636F6E666967E6
:101E40002869702C646E732C67772C7375626E65CD
:101E500074293A000A5573652074686573652063B8
:101E60006F6D6D616E64733A202768656C70272012
:101E70002D207468697320746578740A276D616316
:101E80002064653A61643A62653A65663A66653A25
:101E90003030272073657420616E642073746F7214
:101EA00065204D41432D6164647265737320696ED2
:101EB00020454550524F4D0A276970205B69705B81
:101EC0002C646E735B2C67775B2C7375626E657424
:101ED0005D5D5D5D27202D207365742073746174D2
:101EE00069632049500A277361766527202D207386
:101EF0006176652063757272656E7420636F6E66BD
:101F0000696720696E204E5652414D3B204F4E7CF2
:101F10004F4646202D20656E61626C652F646973A3
:101F200061626C65206175746F736176650A2767FD
:101F3000657427205B636F6E6669672061646472F5
:101F40005D27202D2067657420636F6E66696720AA
:101F500066726F6D207072652D636F6E666967754E
:101F60007265642055524C20616E642073746F72E8
:101F70006520616464722C204F4E7C4F4646202DB4
:101F800020656E61626C652F64697361626C6520A7
:101F9000646F776E6C6F6164206F6E207374617212
:101FA0007475700A276C6F616427202D206C6F6137
:101FB0006420636F6E6669672066726F6D204E568F
:101FC00052414D0A2770776427202D206465666989
:101FD0006E6520616E642073746F7265204D51547C
:101FE000542070617373776F72640A276F74617025
:101FF000776427202D20646566696E6520616E64B4
:102000002073746F72652048545450204150492009
:1020100070617373776F72640A276C6F67205B73EC
:10202000657269616C5F6C6F676C6576656C5D206D
:102030005B7564705F6C6F676C6576656C5D27209F
:102040002D20646566696E65206C6F67206C65760F
:10205000656C2028302E2E37290A276B696C6C2777
:10206000202D2074657374207761746368646F67D2
:102070000A27636C65617227202D20636C6561728D
:1020800020454550524F4D0A27736561726368279A
:10209000202D2073656172636820312D7769726528
:1020A000206465760A277265626F6F7427202D2081
:1020B0007265626F6F7420636F6E74726F6C6C65A3
:1020C0007200536F6674207265626F6F74696E6719
:1020D0002E2E2E00206E6577002069732000315768
:1020E000543A003157543A20536561726368696EFF
:1020F00067206465760052414D3D000A5379736C48
:102100006F6720000A312D7769726520000A6D71B2
:10211000747420000A6D6F64627573207632000A51
:102120006D6F6462757320763120282B29000A694F
:102130006E7075747320000A6974656D7320000AEF
:10214000436F6E666967757265643A00496E6974BB
:1021500069616C697A696E6720496E707574730085
:102160003157543A207365747570207265736F6CC3
:102170007574696F6E20003157543A2044533234DD
:1021800038322D313030206E6F7420707265736577
:102190006E74003157543A204453323438322D3162
:1021A00030302049324320726573746F7265640069
:1021B0003157543A204275732072657365742065F7
:1021C00072726F72003157543A2042757320526513
:1021D00073657420646F6E65003157543A20445320
:1021E000323438322D3130302070726573656E7440
:1021F0002C207265736574004572726F7220312DE8
:102200007720696E6974003157543A204453323450
:1022100038325F3130305F4932435F544F5F31575E
:102220005F42524944474520696E697400444D58E5
:102230004F75742E20467265653A00444D58696E9C
:102240002042756666657220616C6C6F63206572F2
:102250007200496E697420696E2063683A003B0021
:102260003D0050696E3A003B003D4C4F57005468AA
:1022700065726D6F3A004F6E652077697265205206
:10228000656164790A00467265653A00444D5820DC
:102290006F757420737461727465642E2043686175
:1022A0006E6E656C733A2000444D5820696E207341
:1022B0007461727465642E204368616E6E656C7320
:1022C0003A0042726F6B65727320636F6E66696766
:1022D000757265643A004170706C79696E6720634D
:1022E0006F6E666967004C6F616465642045544198
:1022F000473A004E6F2073746F72656420636F6E8F
:10230000666967004C6F616465642066726F6D205A
:10231000454550524F4D006C6F6164206661696C99
:102320006564004A534F4E20646574656374656448
:10233000004C6F6164696E6720436F6E6669672049
:1023400066726F6D20454550524F4D00436F6E666B
:102350006967206175746F736176653A000A537915
:10236000736C6F67206465627567206C6576656C59
:102370003A0053657269616C206465627567206C10
:102380006576656C3A0053617665640A005365743E
:102390002064796E616D69632049500A004F544191
:1023A0002050617373776F72642075706461746517
:1023B000640A004E6F204950206164726573730097
:1023C000205361766564004C6F6164696E672048D4
:1023D00054545020636F6E666967206F6E2073746B
:1023E00061727475703A0000000000000000000087
:1023F0004F4E000000000000004F46460000000065
:102400000000524553540000000000544F47474C11
:102410004500000048414C540000000000584F4E59
:10242000000000000000584F464600000000004930
:102430004E4352454153450044454352454153455F
:1024400000454E41424C4500000044495341424C36
:10245000450000554E465245455A450046524545B1
:102460005A450000004155544F000000000046410D
:102470004E5F4F4E4C59004849474800000000004D
:102480004D454449554D0000004C4F570000000099
:102490000000484541540000000000434F4F4C00ED
:1024A0000000000044525900000000000053544F47
:1024B00050000000000052474200000000000048A9
:1024C0005356000000000000636F756C64206E6F4F
:1024D000742070617273653A200055706461746590
:1024E000640A00454550524F4D20636C656172652A
:1024F000640A004D5154542050617373776F7264B5
:1025000020757064617465640A002B002D004554C9
:1025100061673A200047657420455441473A2000DE
:10252000485454502F312E310025733A2025730D15
:102530000A0020485454502F312E310D0A486F7331
:10254000743A2025730D0A4163636570743A202A3A
:102550002F2A0D0A436F6E6E656374696F6E3A20A1
:10256000636C6F73650D0A0025730020000D0A006F
:10257000474554006661696C656420746F20636F21
:102580006E6E6563740A004552524F523A2053658D
:10259000727665722072657475726E656420004390
:1025A0006F6E666967206E6F74206368616E676521
:1025B000640A00446F6E652E0A00436F6E66696799
:1025C0002070617273696E67206661696C65640A68
:1025D000004765742061626F7274656400676F7490
:1025E00020436F6E6669670A0068747470207265B4
:1025F00074636F64652000667265652000436F6ECA
:10260000666967205552493A20687474703A2F2FD2
:10261000002044656661756C7420636F6E6669673F
:102620002073657276657220757365643A20006C5C
:10263000617A79686F6D652E7275000A282D2943BD
:10264000414E000A282D294D455243555259000A42
:10265000282B294D554C544956454E54000A282BD9
:102660002950574D5F52454C4159000A282B294D9E
:10267000444E53000A282D29554152544252494490
:102680004745000A282B295359534C4F47000A2825
:102690002B29504944000A282D294D43503233300C
:1026A0003137000A282D294152544E4554000A283A
:1026B0002D294F5441000A282B29535049204C45BD
:1026C00044000A282B294D4F544F522043545200A6
:1026D0000A282B294143204841494552206F6E204A
:1026E00053657269616C33000A282B2943435338C0
:1026F000313120262048444331303830000A282B1D
:1027000029524553544152545F4C414E5F4F4E5FE6
:102710004D5154545F4552524F5253000A282D29AF
:102720004841524452455345542C207573696E6795
:1027300020736F6674000A282B29434F554E544569
:1027400052000A282B29444854000A282B294453B4
:10275000323438322D313030000A282B294F574976
:102760005245000A282D2949504D4F4442555300E7
:102770000A282B294D4F44425553203078303620BB
:1027800061742053657269616C3220737065656491
:102790003A39363030000A282B29414441465255F7
:1027A0004954204C4544000A282B29444D58000A1E
:1027B000282B2957697A6E657435313030000A2824
:1027C0002B294672656552616D207072696E74695D
:1027D0006E67000A282B295741544348444F47004D
:1027E0006C617A79686F6D652E7275000A436F6E41
:1027F000666967207365727665723A0032303131EE
:1028000030334C0020432B2B2076657273696F6E3A
:102810003A00666638393937665F323032342D30E7
:10282000382D3233000A4C617A79686F6D652E72EB
:1028300075204C6967687448756220636F6E7472A6
:102840006F6C6C6572200000002200250028002BB0
:10285000002E003100340002010000050108010BC8
:102860000100000A0B02090C0D0E08070304010009
:102870000000000000000000000000000000000058
:102880000000000000000000000000000012111015
:102890000000000000000000000000000000000038
:1028A0000000000000000000002100240027002A92
:1028B000002D003000330001010000040107010A6F
:1028C0000101021020200808102040102040800242
:1028D0000102010804020101020408102040808066
:1028E00040201008040201800402018040201008EA
:1028F00004020108040201010204081020408001C2
:102900000204081020408005050505070508080891
:1029100008020202020A0A08080404040401010170
:102920000101010101030303030303030304070778
:10293000070C0C0C0C0C0C0C0C0202020206060616
:1029400006060606060B0B0B0B0B0B0B0B556E73DB
:102950007065636966696564206572726F722E00C6
:1029600047454E455249435F4552524F5200494EEA
:102970005445524E414C5F4552524F5200493243EA
:102980005F4552524F520049445F4552524F5200E8
:1029900053554343455353004343533831313A2051
:1029A0000057726F6E67207061796C6164004D51E1
:1029B00054543A204354524C2F7478743A204F7533
:1029C000744F664D656D6F72793A2000202D3E2060
:1029D00041543A004368616E20747970653A004E44
:1029E0006F2073746F7265642076616C75657320F7
:1029F0002D2064656661756C743A200053617665BC
:102A00006420455441473A0053657420455441477A
:102A10003A2000556E6B6E6F776E2073756666692F
:102A2000782000556E6B6E6F776E20636D642000AA
:102A3000636C724374723A2000454F46002F004980
:102A40006E3A20002500C2B04320483D0020444893
:102A500054323220747970652E20543D00494E3A2C
:102A600000204E6F20656D697420646174612100DF
:102A700020436F756E74657220747970652E2076B0
:102A8000616C3D00494E3A0020436F756E7465726B
:102A900020747970652E20494E434F52524543545D
:102AA00020496E74657272757074206E756D626502
:102AB00072212121004952513A002D3E002000236D
:102AC000002D3E00200050656E6465643A202300AE
:102AD0003D00494E3A003D004C454741435920498D
:102AE0004E3A0020666F7220286D73293A004354D5
:102AF000524C3A205363686564756C6520636D645D
:102B00002000206D73203A0041726D656420666F6D
:102B10007220002044697361726D656400207469DD
:102B20006D653A004354524C3A205265733A002086
:102B300054533A0020543A00544845524D3A004309
:102B40006C65616E696E6720616C61726D20003D1D
:102B50000050696E3A004354524C3A20436F6D6DF9
:102B6000616E6420626C6F636B65642062792064BF
:102B70007269766572206F72206368616E6E656C33
:102B80002066726F7A656E004354524C3A204F4E65
:102B90003A416C7265616479204163746976650AB3
:102BA000004354524C3A2048414C543A416C7265AF
:102BB00061647920496E6163746976650A004354E3
:102BC000524C3A20584F4E3A2044697361626C650A
:102BD000640A004354524C3A20584F4E3A416C72AA
:102BE00065616479204163746976650A00435452D3
:102BF0004C3A20584F464620736B69707065642EBE
:102C0000205072657620636D643A004354524C3A0A
:102C1000205475726E6564206F66662066726F6DF3
:102C20003A004354524C3A20526573746F72656493
:102C30002066726F6D3A004354524C3A2049676ED9
:102C40006F7265642C206368616E6E656C20636DC5
:102C5000643D0020457865633A004354524C3A2065
:102C60004163746976653A004354524C3A204841B6
:102C70004C543A416C726561647920496E616374A9
:102C80006976650A004354524C3A20584F4E3A2018
:102C900044697361626C65640A004354524C3A2083
:102CA000584F4E3A416C7265616479204163746992
:102CB00076650A004354524C3A20584F46462073DA
:102CC0006B69707065642E205072657620636D6448
:102CD0003A004354524C3A205475726E6564206F2A
:102CE00066662066726F6D3A004354524C3A205229
:102CF0006573746F7265642066726F6D3A00435439
:102D0000524C3A204E6F7420656E6F756768206D67
:102D1000656D6F727920666F722067726F757020B3
:102D20006F7065726174696F6E00496E76616C696F
:102D3000642061726700496E76616C69642061721B
:102D400067004354524C3A20556E6B6E6F776E207D
:102D500073756666697800536B6970706564206886
:102D60006F6D696520737475666600200020537569
:102D7000623D00204974656D3D004354524C3A2039
:102D800052414D3D004354524C3A204F75744F66AA
:102D90004D656D6F72793A2000282D292000282B6F
:102DA0002920002076616C756520697320002075EC
:102DB0006E6B6E6F776E0A005D3D005B0020696E82
:102DC00076616C69640020004143544956453A00DD
:102DD000206F6B003A00206661696C6564003A0000
:102DE0005265747279696E6720564354454D502080
:102DF000434D440A005265747279696E67205643E8
:102E000020434D440A005265747279696E67206DE3
:102E10006F6462757320434D440A00526574727981
:102E2000696E6720434D440A00206572726F723DDF
:102E3000004D423A20706F6C6C696E67200020561E
:102E4000616C3A20004D423A20004D423A204E6FCC
:102E50007420737570706F7274656420726567207A
:102E6000747970650A004D423A20706F6C6C696E1F
:102E7000672064696D6D657220004D423A20496C8F
:102E80006C6567616C20617267756D656E74730A3D
:102E900000206572726F723D004D423A20706F6C77
:102EA0006C696E6720504920002D004D423A205039
:102EB000492056616C203A004D423A20706F6C6C8C
:102EC000696E6720504920004D423A20706F6C6C4B
:102ED000696E6720464D206661756C742000206520
:102EE00072726F723D004D423A20706F6C6C696E69
:102EF0006720002D004D423A20464D2056616C203F
:102F00003A004D423A20706F6C6C696E6720464DF6
:102F100020004354524C2F706F6C6C3A204F7574E4
:102F20004F664D656D6F72793A200020736563209E
:102F300072656D61696E696E6700005EBCE2613F3B
:102F4000DD83C29C7E20A3FD1F419DC3217FFCA287
:102F5000401E5F01E3BD3E6082DC237D9FC1421CB9
:102F6000FEA0E1BF5D0380DE3C62BEE0025CDF816B
:102F7000633D7C22C09E1D43A1FF4618FAA4277919
:102F80009BC584DA3866E5BB5907DB856739BAE447
:102F900006581947A5FB7826C49A653BD987045A79
:102FA000B8E6A7F91B45C6987A24F8A6441A99C72B
:102FB000257B3A6486D85B05E7B98CD2306EEDB3D9
:102FC000510F4E10F2AC2F7193CD114FADF3702E07
:102FD000CC92D38D6F31B2EC0E50AFF1134DCE9039
:102FE000722C6D33D18F0C52B0EE326C8ED0530DEB
:102FF000EFB1F0AE4C1291CF2D73CA947628ABF599
:1030000017490856B4EA6937D58B5709EBB53668C6
:103010008AD495CB2977F4AA4816E9B7550B88D6F8
:10302000346A2B7597C94A14F6A8742AC896154BAA
:10303000A9F7B6E80A54D7896B35436F6E6E65639E
:103040007465642E00436F6E6E2E2061626F727421
:103050006564003E3E2000496E76616C69642063C1
:103060006F6D6D616E640000002000230026002952
:10307000002C002F003200000100000301060109AE
:10308000013E3E3E004E6F204D414320636F6E6611
:103090006967757265643A20736574206669726D3C
:1030A000776172652773204D41430A0045455052B0
:1030B0004F4D207369676E6174757265206F6B0088
:1030C000496E697469616C697A696E67204545501B
:1030D000524F4D2E002072656164206572726F72CE
:1030E00020666F7220003E2000203C003157543A89
:1030F000003157543A206E6F7420696E6974003144
:1031000057543A20425553592074696D656F757450
:10311000003157543A204453323438325F455252CA
:103120004F525F434F4E464947003157543A203182
:103130002D776972652073686F72746564007265BB
:103140006164790024737461746500757074696DCD
:1031500065006672656568656170002473746174EA
:10316000730020457870697265640A00202D7461CF
:1031700072676574207A6F6E652D0020416C6172F4
:103180006D20457870697265640A0020636D643A49
:1031900000204375723A00205365743A0020546948
:1031A0006D65723A00204C6F636B733A0052414D6B
:1031B0003D00FF01F50111241FBECFEFD1E2DEBFBC
:1031C000CDBF00E00CBF1AE0A0E0B2E0E6E8FDE908
:1031D00002E00BBF02C007900D92A235B107D9F7EC
:1031E00022E1A2E5BAE001C01D92AD35B207E1F7D8
:1031F00018E1CAEDD8E100E006C021970109802F4F
:10320000FE010F948746C93DD10780E00807A9F762
:103210000F9458350D94B14E0C94000090E0FC01D1
:10322000E95FF64DE491F0E0EE0FFF1FE95BF74D2B
:10323000A591B4912C918F53974DFC0184918223D9
:1032400091E009F490E0892F089590E080E00895DE
:10325000DC01ED91FC910284F385E02D1994DF925D
:10326000EF92FF920F931F93CF93DF93EC010C89A2
:103270001D890115110559F01D8A1C8AC801DF91AD
:10328000CF911F910F91FF90EF90DF900895EC8503
:10329000FD858E859F85DF01A80FB91F2C912432F3
:1032A00009F055C011962C912B3709F050C00296A9
:1032B000E80FF91FF12CE12CDF01D190DD2009F49A
:1032C00046C08DE7D816E9F08FEFE81AF80AF4CF78
:1032D000198A188A2C853D852115310579F08E854E
:1032E0009F85280F391FF9012081222321F00196A3
:1032F0009F878E873EC01D861C86C0CF0FEF1FEFB5
:10330000BDCFE114F10419F11C928E859F850296C0
:103310006C857D85680F791FE881F9810684F785C2
:10332000E02DCE011995998B888B1B8A1A8AEC8522
:10333000FD858E859F85E80FF91FEE0DFF1DD2825A
:103340008E859F850396E80EF91EFF86EE862889F6
:1033500039892115310509F4BDCF8A899B89280F48
:10336000391FF9012081222309F4B2CF01969B8BEA
:103370008A8B022F220F110B81CFDC011C96ED915D
:10338000FC911D971E968D919C91E80FF91F8081ED
:10339000082E000C990B0895DC0115968D919C91D7
:1033A000009739F0DC01ED91FC910680F781E02D6A
:1033B00019940895FC01838594859C0144E035951A
:1033C00027954A95E1F756E0959587955A95E1F747
:1033D0002817390719F081E090E0089582E090E025
:1033E000089583E090E00895DC011296ED91FC9140
:1033F00013973097B9F016968D919C918430910572
:1034000041F08530910541F0039749F482E090E066
:10341000089581E090E0089581E190E0089582852B
:1034200090E0089590E080E0089585E090E00895B0
:1034300090E080E008958EE090E00895DC0112961F
:10344000ED91FC9113973097B9F016968D919C9160
:103450008430910541F08530910541F0039749F49E
:1034600082E090E0089581E090E0089581E190E0AD
:103470000895828590E0089590E080E0089584E1C9
:1034800090E00895DC01ED91FC910484F585E02D38
:1034900060E0199581E090E00895DC011496ED91CB
:1034A000FC9180E0309711F085A1817090E0089543
:1034B000CF93DF93EC016AEC72E18CEB9FE00F9409
:1034C00057166C817D814AE050E08CEB9FE00F94B1
:1034D000F81564EC72E18CEB9FE00F9457168CEBBF
:1034E0009FE00F94EB1460E08C810E94A7BDE881FF
:1034F000F9810484F585E02D60E0CE01199581E025
:1035000090E0DF91CF910895CF93DF93EC0164EECB
:1035100070E18CEB9FE00F9457168CEB9FE00F94BB
:10352000EB14E881F9810484F585E02D60E0CE019B
:10353000199581E090E0DF91CF910895CF93DF93CB
:10354000EC0164E97CE08CEB9FE00F945716EA8174
:10355000FB810280F381E02D608171818CEB9FE023
:103560000F9441168CEB9FE00F94EB14E881F981E6
:103570000484F585E02D60E0CE01199581E090E0AE
:10358000DF91CF910895EF92FF920F931F93CF9306
:10359000DF93EC018B0180915C0A90915D0A0097AA
:1035A000A9F0FC0120852F70263081F40E94F6AD31
:1035B000FC0190859F70943049F481859285DF915C
:1035C000CF911F910F91FF90EF900895EE88FF88A3
:1035D000C70101970D97D0F46DEB75E0C8010F940A
:1035E000F44A892B99F48FE2888F85E08E9DB00193
:1035F0008F9D700D112466597C4E46E050E0CE013F
:1036000049960F94083FCE014896D9CF90E080E0CC
:10361000D6CF4F925F926F927F92BF92CF92DF92FE
:10362000EF92FF920F931F93CF93DF9300D000D0C0
:10363000CDB7DEB77C01B62E8091590A882309F4F4
:10364000BDC0D70114969C9180914402891708F45B
:10365000B5C08091BA0A9091BB0ABAE06B13EFC073
:103660008659954FFC011082D70118960D911C9137
:103670000115110509F49EC0F80161857285611577
:10368000710591F445805680678070848091FC0CB0
:103690009091FD0CA091FE0CB091FF0C48165906BC
:1036A0006A067B0609F486C0D8011B964D915C9191
:1036B0001C974115510509F47DC0F70124815396EB
:1036C0008C91539790E0322F377002C09595879573
:1036D0003A95E2F780FF6EC0C22ED12CC601887FDA
:1036E0009370892B39F451968D919C91887F9370BA
:1036F000C82AD92AD8018D919C91DC01ED91FC91C9
:103700006115710509F485C00688F789E02D1995C2
:10371000019709F04FC06CE3F801808191810F940B
:10372000A9154AE050E0B601D8018D919C910F9403
:103730000815F80122818081918164E673E12223DA
:1037400011F062E673E10F945716D8011D966D9142
:103750007C911E978D919C910F94411660E2F80127
:10376000808191810F94A915D8011F966D917C914C
:1037700050978D919C910F944116F8012281808180
:10378000918167E573E1222311F061E573E10F9404
:1037900057166AE67AE0D8018D919C910F944116F4
:1037A000F80180819181DC01ED91FC91008CF18D1B
:1037B000E02D19951092BB0A1092BA0AD7011596FE
:1037C0008D919C911697009771F014963C912091E1
:1037D0004502231740F0DC01ED91FC910190F0814E
:1037E000E02D6B2D199581E090E026960FB6F894A8
:1037F000DEBF0FBECDBFDF91CF911F910F91FF9024
:10380000EF90DF90CF90BF907F906F905F904F9040
:1038100008950488F589E02D23E635E03A8329836D
:10382000D80115964D905D906D907C9018974B82C5
:103830005C826D827E82BE016F5F7F4F68CF8F3466
:1038400091050CF0BBCFBDE06B1709F4B7CF9C011D
:103850002F5F3F4F3093BB0A2093BA0A8659954F8A
:10386000FC016083ABCF0D94343D0D94343D0D9439
:10387000343D0D94343D0D94343D0D94343D0D9400
:10388000343D0D94343D0D94343D0D94343D2F92D0
:103890003F924F925F926F927F928F929F92AF92E0
:1038A000BF92CF92DF92EF92FF920F931F93CF932D
:1038B000DF93CDB7DEB7AA970FB6F894DEBF0FBE81
:1038C000CDBF5C010E8F1F8F28A339A34AA35BA332
:1038D0006CA37DA31C8A1B8ADC0118968D919C9198
:1038E00001979E8B8D8BE114F104D1F0CE014596AA
:1038F0009F938F9302979F938F9381EC95E09F9373
:103900008F93FF92EF920F94A94B0FB6F894DEBFFE
:103910000FBECDBF019721F48B899C899E8B8D8B27
:103920006B897C894AE050E08CEB9FE00F94F8159E
:103930006FE473E18CEB9FE00F9457166D897E89DD
:103940004AE050E08CEB9FE00F94F81569E473E1D6
:103950008CEB9FE00F945716FE8DFAA74AE050E0DB
:103960006F2F8CEB9FE00F940E158CEB9FE00F9464
:10397000EB1419861A861B861C861D861E861F86DA
:10398000188A8A85807F84608A87D50118968D91F0
:103990009C912D893E89281739071CF001979E8B31
:1039A0008D8B8B899C8997FF02C01C8A1B8A8B8810
:1039B0009C885401312C212C8D899E898A159B0568
:1039C0000CF46AC1BAA5B13091F1B23009F453C117
:1039D000EE24EA94FE2C0E8D1F8D28A139A14AA158
:1039E0005BA16CA17DA1CE0109960E947FA32983D2
:1039F0003A834B835C836D837E838F83988780912A
:103A0000680A9091690AFC0122813381A216B306EB
:103A100008F088C06F852E8530E050E040E0542FDC
:103A2000432F322F2227462B6D85262B33C1E09062
:103A3000680AF090690AF70182819381A816B90695
:103A400008F070C096855385018512854084A92FA2
:103A5000B0E06484712C658570E09401220D331D03
:103A6000951372C0A901440F551F240F351F200F55
:103A7000311FA20FB31F9C91F301E20FF31F1081BE
:103A8000260F371FD9010C91442009F452C0512C44
:103A9000712C612C692F70E0762F6627072E000CA1
:103AA000880B990BA30192010F941046C901772747
:103AB00066276EA37FA388A799A7612F70E0762F52
:103AC0006627072E000C880B990BA30192010F9417
:103AD0001046542F432F322F22278EA19FA1A8A535
:103AE000B9A5822B932BA42BB52B8EA39FA3A8A79C
:103AF000B9A7602F70E0762F6627072E000C880B81
:103B0000990BA30192010F9410466EA17FA188A585
:103B100099A5262B372B482B592B232B242B252BD0
:103B200009F4A0C0FFEFAF1ABF0A2FEF221A320A22
:103B300043CF212F30E050E040E0542F432F322F6D
:103B40002227492B202BE9CFC901880F991F880F05
:103B5000991F800F911FA80FB91F3C91DC01A50F81
:103B6000B11D0C91F301E80FF91FD080860F971F4C
:103B7000DC011C91442009F463C0512C712C612C90
:103B8000632F70E0762F6627072E000C880B990BA9
:103B9000A30192010F941046922F8827772766275A
:103BA0006EA37FA388A799A7602F70E0762F662762
:103BB000072E000C880B990BA30192010F9410465D
:103BC000A901332722278EA19FA1A8A5B9A5822BE1
:103BD000932BA42BB52B8EA39FA3A8A7B9A7612FC6
:103BE00070E0762F6627072E000C880B990BA30137
:103BF00092010F9410466EA17FA188A599A5622B12
:103C0000732B842B952B6EA37FA388A799A76D2D6B
:103C100070E0762F6627072E000C880B990BA30106
:103C200092010F941046542F432F322F22278EA13A
:103C30009FA1A8A5B9A5282B392B4A2B5B2B6DCFAB
:103C4000802F90E0B0E0A0E0DC0199278827B32B1B
:103C5000AC01412B8A019D011D29012B022B032B55
:103C600009F060CF2FEF3FEF4FEF50E0B501C701F4
:103C70000F94061857CF8091680A9091690ADC0169
:103C800012962D913C91A216B30608F04BCF20E07E
:103C900030E0A901B501ECCFCC2009F488C0009137
:103CA000680A1091690AD80119968D919C91892B07
:103CB00009F473C00E94D7BEF801C784D088E18898
:103CC000F2886C157D058E059F0520F46787708B43
:103CD000818B928BF801C784D088E188F2886C19B7
:103CE0007D098E099F096C3271408105910510F3A1
:103CF000F894D80114968D919C9115979A8B898B85
:103D00001996ED91FC917F01BFEFEB1AFB0A8081C0
:103D10008D8FF80190810388F489E02DD8015596A4
:103D20008C91992309F45EC09081982B9C8F90818F
:103D3000809589238B8F8B8D888F88E08F8B5C8D0E
:103D40006B8D4D8D3F89288D89899A89D701508344
:103D500047FD252F3A952083262F39F0441F00C0B8
:103D600000006083000000C0F2CF38E04D91608316
:103D70000000019761F7D8015496FC93EE93539796
:103D80004D8F3F8B288F9A8B898B78940E94D7BE5A
:103D9000F8016787708B818B928B64E473E18CEB05
:103DA0009FE00F9457168CEB9FE00F94EB1481E08B
:103DB00090E0AA960FB6F894DEBF0FBECDBFDF919C
:103DC000CF911F910F91FF90EF90DF90CF90BF9018
:103DD000AF909F908F907F906F905F904F903F90AB
:103DE0002F9008959081982B9C8F908180958923A6
:103DF0008B8F8B8D8A8F88E0898F5C8D6B8D4D8D3D
:103E0000398D2A8D89899A89D701508347FD252FBD
:103E100000C000C0208300C000C000C000C000C0BF
:103E200060830000262F3A9541F0441F000000C037
:103E300000C000C000C000C0E8CF38E04D9100C015
:103E4000608300C0019709F7D8015496FC93EE9364
:103E500053974D8F398F2A8F96CF0F931F93CF9300
:103E6000DF938C0167EC75E08CEB9FE00F94EF140F
:103E7000C091680AD091690A4C815D8170E060E070
:103E800089859A850F942144209771F089859A85B8
:103E90000F94343D8E819F8197FD03C060E00E94A6
:103EA000A7BDCE010F94343DD801ED91FC9104845F
:103EB000F585E02D60E0C801199581E090E0DF9183
:103EC000CF911F910F910895CF93DF93EC0165E897
:103ED0007CE08CEB9FE00F945716EA81FB81028017
:103EE000F381E02D608171818CEB9FE00F9441168E
:103EF0008CEB9FE00F94EB14E881F9810484F58545
:103F0000E02D62E0CE01199581E090E0DF91CF9144
:103F10000895DC01ED91FC910484F585E02D62E0CB
:103F2000199581E090E00895CF93DF93EC0167ED60
:103F300075E08CEB9FE00F94EF1440E050E0BA0185
:103F40008A819B810E9407E4E881F9810484F585D8
:103F5000E02D60E0CE0119956D858C810E9479BDC0
:103F60006D858D810E9479BD81E090E0DF91CF91D8
:103F70000895FC01828193810E94DDE621E030E01A
:103F8000823011F430E020E0C90108950F931F93AF
:103F9000CF93DF938C01D0E0C0E001151105B1F0A3
:103FA000BE016854734FC8010F94D13E892B51F460
:103FB000FE01E454F34F849190E0DF91CF911F9183
:103FC0000F9108952596C233D10539F781E090E02D
:103FD000F4CFFF920F931F93CF93DF93CDB7DEB74C
:103FE00064970FB6F894DEBF0FBECDBF8C01F62EDE
:103FF0008FE290E09A838983FE01339688E0DF01A7
:104000001D928A95E9F7F8016681FF2011F081E0A1
:104010006827D80114968C910E9479BDF801878198
:104020009085A185B285883E9340A105B10508F42D
:1040300091C060E173E18CEB9FE00F945716D801BB
:1040400014966D917C914AE050E08CEB9FE00F94C8
:10405000F8156BE073E18CEB9FE00F9457166F2D12
:1040600070E04AE050E08CEB9FE00F94F8158CEB89
:104070009FE00F94EB1462E373E1CE0101960F947D
:10408000C63EF801828193810E94DDE6FF2009F49B
:104090006DC063E073E1843151F06CEF72E1853102
:1040A00031F060EF72E18F3011F468EF72E1CE0110
:1040B0000B960F94DA3E6BED72E18CEB9FE00F9460
:1040C0005716D8011296ED91FC9113970280F38157
:1040D000E02D60817181ED91FC910288F389E02DE2
:1040E0009E012F5F3F4FAE01455F5F4FC80119959D
:1040F0004AE050E0BC018CEB9FE00F94F81569EDAD
:1041000072E18CEB9FE00F945716D8011296ED9157
:10411000FC910280F381E02D608171818CEB9FE046
:104120000F944116BE016F5F7F4F8CEB9FE00F94A1
:10413000411666ED72E18CEB9FE00F945716BE01BD
:10414000655F7F4F8CEB9FE00F9441168CEB9FE0F7
:104150000F94EB1464960FB6F894DEBF0FBECDBF7C
:10416000DF91CF911F910F91FF9008956CEE72E156
:10417000823009F49CCF67EE72E199CFAF92BF9283
:10418000CF92DF92EF92FF920F931F93CF93DF9323
:10419000CDB7DEB768970FB6F894DEBF0FBECDBFC0
:1041A000FC01098B1A8B2B8B3C8B4D8B5E8B6F8BA1
:1041B000788F82819381009709F4A1C02481358191
:1041C000232B09F49CC0CC2009F499C06F0170E046
:1041D00060E00E94EBE4192FD601ED91FC91048C74
:1041E000F58DE02DC60119955C018230910509F429
:1041F0007AC0039709F445C095E0F1E0AF16B10429
:1042000009F091E019861A861B861C861D861E867B
:104210001F86188A8A85807F892B8A87EE24EA94F4
:10422000FE2C09891A892B893C894D895E896F8901
:10423000788DCE0109960E947FA3F1E0AF16B104FC
:1042400009F453C082E0A816B10409F049C06F8593
:1042500070E0D60114968C910E94E3BD61E070E09D
:10426000C6010F94BB0B6E8570E00E94E3BD62E057
:1042700070E0C6010F94BB0B6D8570E00E94E3BD3A
:104280002FC0612F661F6627661FCE0141960E94D0
:1042900076705C01BC01D60114968C910E94E3BD3E
:1042A0006DEA72E18CEB9FE00F945716F601648182
:1042B00075814AE050E08CEB9FE00F94F8156BEAB3
:1042C00072E18CEB9FE00F9457164AE050E0B50185
:1042D0008CEB9FE00F94F8158CEB9FE00F94EB14A0
:1042E00081E090E00EC094E08DCF63E070E0C60105
:1042F0000F94BB0B688970E00E94E3BDA8CF90E0EB
:1043000080E068960FB6F894DEBF0FBECDBFDF9198
:10431000CF911F910F91FF90EF90DF90CF90BF90C2
:10432000AF900895CF93DF93EC0161EA72E18CEBDB
:104330009FE00F9457166C817D814AE050E08CEB32
:104340009FE00F94F8156FE972E18CEB9FE00F94FA
:104350005716EA81FB810280F381E02D6081718133
:104360008CEB9FE00F94411669E972E18CEB9FE0C2
:104370000F9457168CEB9FE00F94EB14E881F981B2
:10438000048CF58DE02DCE0119958130910529F031
:10439000029759F060E08C811AC063E070E0CE01B2
:1043A0000F94BB0B60E00E94A7BD60E08C810E946F
:1043B000A7BD61E070E0CE010F94BB0B60E00E94EE
:1043C000A7BD62E070E0CE010F94BB0B60E00E94DD
:1043D000A7BDE881F9810484F585E02D60E0CE0178
:1043E000199581E090E0DF91CF910895CF93DF930D
:1043F000EC016FE872E18CEB9FE00F9457166C8133
:104400007D814AE050E08CEB9FE00F94F8156DE859
:1044100072E18CEB9FE00F945716EA81FB810280DA
:10442000F381E02D608171818CEB9FE00F94411648
:1044300067E872E18CEB9FE00F9457168CEB9FE0DE
:104440000F94EB148A819B81892B09F451C08C81D4
:104450009D81892B09F04CC0E881F981048CF58D90
:10446000E02DCE0119958130910529F0029759F080
:1044700061E08C811AC063E070E0CE010F94BB0B49
:1044800061E00E94A7BD61E08C810E94A7BD61E050
:1044900070E0CE010F94BB0B61E00E94A7BD62E00B
:1044A00070E0CE010F94BB0B61E00E94A7BD80912C
:1044B000A100887F8093A10080919100887F8093E4
:1044C00091008091A10082608093A1008091910071
:1044D000826080939100E881F9810484F585E02D64
:1044E00062E0CE01199581E090E0DF91CF910895CF
:1044F00090E080E0FACFCF92DF92EF92FF920F939D
:104500001F93CF93DC011296ED91FC9160E08481C2
:1045100095810E94A8AE8C01009729F0FC0180854E
:104520008F708530D1F065EF71E185E19FE00F94E8
:10453000571685E19FE00F94EB14C12CD12C90E825
:10454000E92E9FEBF92EC701B601CF911F910F9174
:10455000FF90EF90DF90CF900895C8010E9439AF8F
:10456000813040F18630A8F1893020F565E0C8013E
:104570000E94A8AEFC0190859F709330F9F4C1842D
:10458000D284E384F484C1E060E0C8010E94A8AE54
:10459000FC0190859F70933009F561857285838554
:1045A000948520E030E0A9010F94C64487FF1FC026
:1045B000C111C9CFC12CD12C7601C5CF923049F49D
:1045C00061857285838594850F94CD446B017C0150
:1045D000DACFC0E0C12CD12C7601D6CF923039F49D
:1045E00061857285838594850F94CD44DACFC1119E
:1045F000AACFC12CD12C8FE7E82E83E4F82EA3CFCD
:10460000CF93DF93EC0163EC71E18CEB9FE00F94AF
:104610005716EA81FB810280F381E02D6081718170
:104620008CEB9FE00F94EF14EC81FD81309721F02B
:10463000808191810F94343D8C819D810F94343D14
:1046400070E060E08A819B810E94B4E31D821C823D
:1046500081E090E0DF91CF910895CF93DF93EC015B
:1046600066EE75E08CEB9FE00F944116EA81FB81CA
:104670000280F381E02D608171818CEB9FE00F94CB
:10468000EF148C819D81009711F00F94343D70E000
:1046900060E08A819B810E94B4E31D821C8281E0DC
:1046A00090E0DF91CF910895CF93DF93FC012281B9
:1046B0003381232B59F1EC016EE27BE08CEB9FE020
:1046C0000F9457164AE050E06E818CEB9FE00F94F8
:1046D0000E158CEB9FE00F94EB148C819D810F9451
:1046E000343D70E060E08A819B810E94B4E31D82CA
:1046F0001C82E881F9810484F585E02D60E0CE011B
:10470000199581E090E0DF91CF91089590E080E0ED
:10471000FACF0F931F93CF93DF938C01DC01149694
:10472000ED91FC91309709F456C0C681D78120974E
:10473000C1F1E881F981309781F18081882369F1A5
:104740006FE776E0CE010E94F6AD892B41F42FEFA2
:104750003FEFA9016FE776E0CE010E9494B764E8CD
:1047600076E0CE010E94F6AD892B41F42FEF3FEFAA
:10477000A90164E876E0CE010E9494B765EF75E088
:10478000CE010E94F6AD892B41F42FEF3FEFA90136
:1047900065EF75E0CE010E9494B70A80DB81C02DE1
:1047A000C6CF69ED70E18CEB9FE00F9457168CEB50
:1047B0009FE00F94EB14D801ED91FC910484F585F2
:1047C000E02D62E0C801199581E090E0DF91CF9182
:1047D0001F910F91089565EC70E18CEB9FE00F94B1
:1047E00057168CEB9FE00F94EB1490E080E0EECF37
:1047F0008F929F92AF92BF92CF92DF92EF92FF92F1
:104800000F931F93CF93DF93CDB7DEB760970FB6AB
:10481000F894DEBF0FBECDBFE986FA860B871C87F2
:104820002D873E874F87588B6115710511F0011157
:1048300003C090E080E0CCC07B015C01DB018D9087
:104840009C9019821A821B821C821D821E821F82EA
:1048500018868A81807F8A8369EF75E0C7010E948C
:10486000F6AD6C016EEF75E0C7010E94F6AD7C01FC
:10487000C114D10451F1F60180858F70843029F57F
:10488000818592850E94C61F182F8930B1F134F4BA
:104890008130E4F4C12CD12C760168C08A30D1F784
:1048A000B701CE0109960E94097829833A834B8388
:1048B0005C836D837E838F8398873F7009F4B9CFC3
:1048C000CE0101960E941F7215C011E0B701CE0102
:1048D00009960E94097829833A834B835C836D8310
:1048E0007E838F8398873F7009F4A3CFCE01019612
:1048F0000E94DB716B017C0139C0B701CE010996C2
:104900000E94097829833A834B835C836D837E837D
:104910008F8398873F7009F48CCF31503B3008F07B
:10492000B9CFE32FF0E08827E756FB4D8F4F0D946A
:104930008746AD24AD244A24A424A4240825FB24BE
:10494000FB24FB24A424A4242D813E814F8158857F
:10495000AAE0B0E00F945146CDCFCD80FAE0CF9ED3
:10496000600111240D2C000CEE08FF088091450217
:10497000893020F4809144028930E8F060E670E1EB
:104980008CEB9FE00F945716B4018CEB9FE00F94D3
:10499000411669E570E18CEB9FE00F9457162AE011
:1049A00030E0B701A6018CEB9FE00F94B0158CEBC3
:1049B0009FE00F94EB14D5011296ED91FC9162E00B
:1049C000848195810E94A8AE009779F581E090E0FE
:1049D00060960FB6F894DEBF0FBECDBFDF91CF91CA
:1049E0001F910F91FF90EF90DF90CF90BF90AF900D
:1049F0009F908F90089520E030E040E251E46D8177
:104A00007E818F8198850F942C450F94984772CFA3
:104A10006D817E818F8198852AE030E040E050E012
:104A20000F94324669017A01A1CFFC0120852F70D5
:104A3000263061F6B4010E94F6AD5C01009731F2B8
:104A4000DC0118968C9118978F709BEF980F92301D
:104A500008F0BCCF4501853029F416968C90169746
:104A600017969C90F50180858068808762E076E0EB
:104A7000C4010E94F6ADFC01892B61F0C186D2868B
:104A8000E386F486812F8295807F10851F70182B16
:104A900010879CCF60E570E18CEB9FE00F94571678
:104AA000D5016D917C918CEB9FE00F9441168CEBBE
:104AB0009FE00F94EB14A701960162E076E0C40139
:104AC0000E9494B762E076E0C4010E94F6ADFC015A
:104AD000892B09F47BCF1295107F90859F70192B3D
:104AE000D7CF2F923F924F925F927F928F929F9259
:104AF000AF92BF92CF92DF92EF92FF920F931F93EC
:104B0000CF93DF9300D000D01F921F92CDB7DEB7B6
:104B100009831A832B833C834D835E836F8378875D
:104B2000DC011496ED91FC910FEF1FEF3097F9F037
:104B300057014C01C288D388E114F10489F1F701CF
:104B40008081882369F1C114D10489F1B701C601BC
:104B50000E94F6ADE980FA800B811C812D813E8197
:104B60004F815885BC01C4010E94F8238C01C80103
:104B700028960FB6F894DEBF0FBECDBFDF91CF9160
:104B80001F910F91FF90EF90DF90CF90BF90AF906B
:104B90009F908F907F905F904F903F902F900895BF
:104BA000C114D10421F0D6011696CD90DC907B8003
:104BB000F12C0FEF1FEF272C312C512C412CC1145D
:104BC000D10449F165E076E0C6010E94F6AD009798
:104BD000E9F0FC0120852F702230C1F48185928597
:104BE000A385B48582159305A405B50579F4E980FC
:104BF000FA800B811C812D813E814F815885B60141
:104C0000C4010E94F8238C01FF24F394D60112966C
:104C1000CD90DC90D4CFF110AACF6BE770E185E1A5
:104C20009FE00F945716B50185E19FE00F94411660
:104C30006FE670E185E19FE00F945716672D70E0F5
:104C40004AE050E085E19FE00F94F81585E19FE090
:104C50000F94EB148CCFCF93DF93EC01EC81FD81AB
:104C600040815181052E000C660B770B22818DE56A
:104C70009CE00F94A41770E060E08A819B810E9401
:104C8000EBE4EBE5FDE082838DE59CE0918380839E
:104C900010926B0E10926D0E10926C0EDF91CF91F0
:104CA00008954F925F926F927F928F929F92AF92F0
:104CB000BF92CF92DF92EF92FF920F931F93CF9309
:104CC000DF93CDB7DEB768970FB6F894DEBF0FBE9F
:104CD000CDBF098B1A8B2B8B3C8B4D8B5E8B6F8BD7
:104CE000788FDC0112962D913C911397232B09F4B8
:104CF000DEC0CC2009F4DBC06C01ED91FC91048C8A
:104D0000F58DE02D19955C016DEA7CE08CEB9FE060
:104D10000F945716CE0141960E94A974A114B104B4
:104D200071F460E0CE0141960E947670682FF60122
:104D3000848195810F94132C81E090E0BAC0CE015C
:104D400041960E946A724C0194E0F2E0AF16B10401
:104D500059F081E1A816B10409F445C091E0A1E041
:104D6000AA16B10409F495E019861A861B861C86DA
:104D70001D861E861F86188A8A85807F892B8A87D2
:104D8000EE24EA94FE2C09891A892B893C894D89E5
:104D90005E896F89788DCE0109960E947FA363EAB0
:104DA0007CE08CEB9FE00F945716CE0109960E9491
:104DB000A974B2E0AB16B10489F0E1E1AE16B1041A
:104DC000B1F0AA94AB2809F0B7CF188963E070E07E
:104DD000C6010F94BB0B612F0F94132C6F85F60146
:104DE0008481958151C0888D8170888FBCCF0FE7F9
:104DF00010E08FEF88169806A9F0092C000CAA087D
:104E0000BB08A50194012959310941095109AFEFA6
:104E1000B0E00F9451462BE531E040E050E00F94B4
:104E20003246890163E070E0C6010F94BB0B5C0160
:104E3000288930E0D8010F949E46412C512C320134
:104E40004A94A30192010F943246622FC5010F9438
:104E5000132C64E070E0C6010F94BB0B5C01AFEF54
:104E6000B0E0A01BB10B288930E00F949E46A3014F
:104E700092010F943246622FC5010F94132C6F8557
:104E8000D60114968D919C910F94132C1E8561E090
:104E900070E0C6010F94BB0B612F0F94132C1D857E
:104EA00062E070E0C6010F94BB0B612F43CF90E02E
:104EB00080E068960FB6F894DEBF0FBECDBFDF91DD
:104EC000CF911F910F91FF90EF90DF90CF90BF9007
:104ED000AF909F908F907F906F905F904F900895CC
:104EE0000F931F93CF93DF9300D000D01F92CDB7C5
:104EF000DEB78091630A882369F068E279E085E192
:104F00009FE00F94571685E19FE00F94EB1490E01B
:104F100080E0B0C068E579E08BE09FE00F947B16FD
:104F20000E948EB88091500290915102A09152023D
:104F3000B091530289839A83AB83BC838EE09DE05A
:104F400090931B0D80931A0D1E8280E197E22E81B3
:104F50002F5F2E830197D9F71D82BE016B5F7F4FB4
:104F600080E20E9404B88C01892BF1F48D8101E06C
:104F700010E08138C9F4BE016F5F7F4F8FEF0E9450
:104F800054B81F8280E89EE32F812F5F2F83019703
:104F9000D9F7BE016B5F7F4F80E00E9404B88D811E
:104FA00080FF0CC003E010E064E479E085E19FE05D
:104FB0000F945716C8010E94D1B7A9CFBE016B5FED
:104FC0007F4F80E00E9404B8892B61F78D8184FFB8
:104FD000E9CF80911C0D0E94FAB780911A0D909133
:104FE0001B0DDC01ED91FC910190F081E02D64EF4F
:104FF000199580911A0D90911B0D0F94F32D882314
:1050000019F002E010E0D0CFBE016B5F7F4F81E06E
:105010000E9404B88C01892B39F61D811F7810611C
:105020001D8380911C0D0E94FAB780911A0D9091FA
:105030001B0DDC01ED91FC910190F081E02D61E010
:10504000199580911A0D90911B0DDC01ED91FC9149
:105050000190F081E02D612F199580911A0D9091AA
:105060001B0D0F94F32D8111CCCF81E08093630A47
:1050700081E090E027960FB6F894DEBF0FBECDBF5B
:10508000DF91CF911F910F910895EF92FF920F93AF
:105090001F93CF93DF93CDB7DEB760970FB6F89429
:1050A000DEBF0FBECDBF80915E0A8823C9F065E6E2
:1050B00079E08CEB9FE00F9457168CEB9FE00F94F8
:1050C000EB1490E080E060960FB6F894DEBF0FBE60
:1050D000CDBFDF91CF911F910F91FF90EF90089579
:1050E00069EB79E08CEB9FE00F9457160E948EB825
:1050F00080E48093310D0E948EB810E01B7F809178
:10510000310D0E94FAB762E08EE09DE00F94051029
:10511000612F8EE09DE00F94051060E08EE09DE031
:105120000F9405108EE09DE00F94F32D6AE070E07F
:1051300080E090E00E94ECBF66EA79E08CEB9FE0B3
:105140000F9457168EEF0E941FC040E150E0BC0143
:105150008CEB9FE00F94081568E979E08CEB9FE0F9
:105160000F9457168FEF0E941FC040E150E0BC0122
:105170008CEB9FE00F9408158CEB9FE00F94EB14E1
:1051800062E879E08BE09FE00F9457168BEF0E9466
:105190001FC0182F092F8CEF0E941FC0F82EE92E78
:1051A0008DEF0E941FC09F938F93EF92FF920F93FA
:1051B0001F9388E096E09F938F938E010F5F1F4FA0
:1051C0001F930F930F94794BB8018BE09FE00F94DE
:1051D000EF1481E080935E0A0FB6F894DEBF0FBE35
:1051E000CDBF81E090E06FCF4F925F926F927F9240
:1051F000AF92BF92CF92DF92EF92FF920F931F93E5
:10520000CF93DF9300D01F92CDB7DEB72B013C01C7
:1052100029833A834B835C83A6019501C801B701BA
:10522000640D751D861D971D21153105410551051C
:1052300011F00F94104629813A814B815C816217ED
:10524000730784079507D0F42415350546055705DF
:1052500030F521E0822F0F900F900F900F90DF918B
:10526000CF911F910F91FF90EF90DF90CF90BF9063
:10527000AF907F906F905F904F90089546165706BD
:105280006806790650F421E089819A81AB81BC815E
:1052900084159505A605B705E8F220E0DBCF21E0EF
:1052A0004616570668067906A8F2F7CFCF93DF9324
:1052B000EA01282FDC01ED91F0E094E0F595E79507
:1052C0009A95E1F7E258FD4F80818883FD0131977F
:1052D000E081EF70F0E0E258FD4F808189832296F3
:1052E0008A2F821B861738F3615070E0660F771F94
:1052F000460F571FFA011282DF91CF9108950F9345
:105300001F93CF93DF9365E574E18CEB9FE00F94DF
:105310007B1681E00E94FCBE0F94562C61E085E173
:105320000E94A7BD60E084E10E94A7BDC4E1D0E077
:1053300010E001E0612F85E10E9479BD10276AE04D
:1053400070E080E090E00E94ECBF219799F764E163
:1053500070E080E090E00E94ECBF0E948EB88091E7
:10536000351190913611009749F10F94412C8EE040
:105370009DE00F94F32D811121C080913511909102
:1053800036110F94922F6AE374E18CEB9FE00F9437
:105390007B16E0913511F091361100838091351123
:1053A000909136110F94A02F66E274E1811102C032
:1053B00061E174E18CEB9FE00F947B1681E0DF915B
:1053C000CF911F910F9108950F931F93182F0E9453
:1053D000DEC104C096958795779567951A95D2F7A3
:1053E0008B019C0101501109210931090E3F1F4F0A
:1053F0002F4F3F4F20F061E070E080E090E01F9180
:105400000F910895AF92BF92CF92EF92FF920F93B8
:105410001F93CF93DF9300D000D01F921F92CDB780
:10542000DEB75C0109831A832B833C834D835E8343
:105430006F83788769E373E18CEB9FE00F945716D5
:10544000CE0101960E94A974E114F10439F062E3DF
:1054500073E1C7010F94D13E009729F1F501028154
:10546000138101151105E9F0898181115CC08B81DF
:10547000813009F460C048F1823029F1082F10E032
:1054800065E173E18CEB9FE00F9457164AE050E022
:10549000B8018CEB9FE00F94F8158CEB9FE00F9414
:1054A000EB1490E080E028960FB6F894DEBF0FBEB4
:1054B000CDBFDF91CF911F910F91FF90EF90CF90D3
:1054C000BF90AF900895CC20C1F060E0CE0101966E
:1054D0000E947670892B09F447C0C8010E9448E4F5
:1054E000672B682B692BE1F480E00E94E429AB0173
:1054F000BC01C8010E9407E413C0C8010E94DDE698
:105500008E3019F050F4813059F460E0CE010196EC
:105510000E947670892B21F0E0CF83518330A8F36D
:1055200081E090E0C0CF8031D0F48E30B0F6813091
:10553000A1F28230C9F065E273E18CEB9FE00F9439
:1055400057164AE050E069818CEB9FE00F940E15EE
:105550008CEB9FE00F94EB1401E010E091CF8351AE
:10556000833008F4BACFE7CF40E050E0BA01C80179
:105570000E9407E460E0C5010E94E91FD1CF2F928D
:105580003F924F925F926F927F928F929F92AF92D3
:10559000BF92CF92DF92EF92FF920F931F93CF9320
:1055A000DF93CDB7DEB760970FB6F894DEBF0FBEBE
:1055B000CDBF6130710509F495C0DC0112966D9183
:1055C0007C916115710509F48DC04C0119821A8214
:1055D0001B821C821D821E821F8218868A81807F08
:1055E0008A8340E052E0CE0101960E94B36F60E0F2
:1055F000CE0101960E9476701C01F4018281938194
:105600000E9448E42B013C01D40117962D913D9155
:105610004D915C911A97D1010F945C462FEF30E0C9
:1056200040E050E00F94104629873A874B875C870B
:105630000E94DEC19B01AC0189859A85AB85BC8542
:105640000097A105B10509F468C0A12CB12C650132
:105650007C018D01C301B2010E94F42889874114A5
:10566000510461047104F1F1D40117968D919D915B
:105670000D90BC91A02D8D879E87AF87B88B0E941F
:10568000DEC19B01AC018D859E85AF85B8890097F1
:10569000A105B10561F0A12CB12C65017C018D0142
:1056A000C301B2010E94F428882309F451C0D40137
:1056B00012966D907C9080E00E94E429AB01BC01C1
:1056C000C3010E9407E4232869F0F40184810E9449
:1056D0000E19D40116969C91891304C061E0C4018F
:1056E0000E94E91F90E080E060960FB6F894DEBF5C
:1056F0000FBECDBFDF91CF911F910F91FF90EF9023
:10570000DF90CF90BF90AF909F908F907F906F90E1
:105710005F904F903F902F90089591E099879FCF91
:10572000B985BB23F1F060E0C4010E94E91FF401D8
:10573000828193810E94C8E8892BA1F640E050E065
:10574000BA01D40112968D919C910E9407E4CACFB0
:10575000F40184810E940E19D40116969C9189133C
:10576000DFCF232809F4BECFF40184810E940E19F3
:10577000D40116969C918913B5CFB985B111B2CFDA
:10578000ADCFCF93DF93EC0168EB72E18CEB9FE040
:105790000F9457166C817D814AE050E08CEB9FE0BE
:1057A0000F94F81562EB72E18CEB9FE00F945716A3
:1057B0008CEB9FE00F94EB1461E08C810E94A7BDFD
:1057C0006E818C810E9479BD8A819B81009729F02E
:1057D00040E050E0BA010E9407E4E881F9810484C6
:1057E000F585E02D62E0CE0119958A819B810097B5
:1057F00081F00E94C8E8181619065CF40A80DB8163
:10580000C02D80E00E94E429AB01BC01CE010E94C2
:1058100007E481E090E0DF91CF910895CF92DF928D
:10582000FF920F931F93CF93DF9300D000D01F926E
:105830001F92CDB7DEB76C01F02E1A83022F10E055
:10584000FF2029F00115110511F401E010E040E0FE
:1058500050E460E070E0F601828193810E943FE5B0
:105860000130110591F10230110541F0012B99F53C
:105870006DEA70E18CEB9FE00F9457168A818F7070
:10588000A1F1F60102811381C8010E9448E4672B4F
:10589000682B692B89F401E010E0C80128960FB647
:1058A000F894DEBF0FBECDBFDF91CF911F910F9156
:1058B000FF90DF90CF90089580E00E94E429AB0133
:1058C000BC01C8010E9407E4E6CFF1E0FF1681F0B9
:1058D00082E0F81669F061EA70E18CEB9FE00F94CA
:1058E00057168CEB9FE00F94EB1410E000E0D5CF3F
:1058F000F601C280D380C6010E9448E4672B682B62
:10590000692B49F280E00E94E429AB01BC01C60189
:105910000E9407E4C2CF2F923F924F925F926F9204
:105920007F928F929F92AF92BF92CF92DF92EF922F
:10593000FF920F931F93CF93DF93CDB7DEB72E97D0
:105940000FB6F894DEBF0FBECDBF6130710509F40C
:1059500071C14C01DC011296ED90FC9040E050E4E6
:1059600060E070E0C7010E9468E5672B682B692B37
:1059700009F460C140E050E860E070E0C7010E94B7
:1059800068E5672B682B692B89F4809127028823AF
:1059900009F450C140E050E860E070E0C7010E94A7
:1059A0003FE580912702815080932702F401E28035
:1059B000F380C7010E9448E42B013C0119821A823E
:1059C0001B821C821D821E821F8218868A81807F14
:1059D0008A8340E052E0B701CE0101960E94B36F86
:1059E00060E0CE0101960E9476709E878D87D4017B
:1059F00012968D919C910E94DDE6823011F08530E7
:105A000011F41E861D86F40186819AEC980F903160
:105A100008F0C3C121853285A90170E060E04987A3
:105A20005A876B877C87C384D484F12CE12C0E9435
:105A3000BABE9C01990F440B550B2C193D094E0918
:105A40005F09AFEFB0E00F94514629853A854B8549
:105A50005C852C193D094E095F090F9432461901E6
:105A600037FDD3C15FEF2516310411F00CF0D0C122
:105A7000411451046104710409F097C1ED84FE845E
:105A8000E218F30896EFE9169FEFF9060CF001C152
:105A9000D4011D966C911D9715968C910E9479BD2D
:105AA000F401C280D380C6010E9448E4672B682BB2
:105AB000692B41F480E00E94E429AB01BC01C601DE
:105AC0000E9407E4D40114961C9114971D966C91C2
:105AD0008EEF810F8C3028F084ED810F833008F039
:105AE00074C0AA27BB27AE19BF09662309F460C09A
:105AF0009D01A1E0BFEF0F94964629E130E040E020
:105B000050E00F943246BA01A90141505F4F6F4FE8
:105B10007F4F942F852F692F782F6F3F710519F0D4
:105B200014F06FEF70E06634710514F466E470E011
:105B3000812F7EC062E970E18CEB9FE00F945716D5
:105B40008CEB9FE00F94EB1467E176E08CEB9FE029
:105B50000F94EF14F401658584810E9479BDD4010E
:105B60001D966C911D9715968C910E9479BD40E011
:105B700050E0BA01F401828193810E9407E440E081
:105B800050E460E070E0D40112968D919C910E94E7
:105B900016E540E050E860E070E0F4018281938116
:105BA0000E9416E5809127028F5F8093270242C0F2
:105BB0002FEF30E00F949E4629E130E040E050E0C6
:105BC0000F943246922F832FA6CFF401858191E066
:105BD00069279EEF980F9C3020F08C52833008F09C
:105BE000D8C0812F0E9479BDAA27BB27AE19BF0953
:105BF000F40185858823C9F12FEF30E00F949E468C
:105C000029E130E040E050E00F943246922F832F9C
:105C1000692F782F6F3F710519F014F06FEF70E066
:105C20006634710514F466E470E0D40115968C9125
:105C30000E94E3BD90E080E02E960FB6F894DEBFA0
:105C40000FBECDBFDF91CF911F910F91FF90EF90CD
:105C5000DF90CF90BF90AF909F908F907F906F908C
:105C60005F904F903F902F9008959D01A1E0BFEF6E
:105C70000F94964629E130E040E050E00F94324620
:105C8000BA01A90141505F4F6F4F7F4F942F852F6D
:105C9000BFCFBBE0EB16F1040CF456CFF4016585E1
:105CA00084810E9479BDD4011296CD90DC90C6010A
:105CB0000E9448E4672B682B692B41F480E00E9426
:105CC000E429AB01BC01C6010E9407E4F40115817F
:105CD00065858EEF810F8C3020F084ED810F83304D
:105CE000B0F4662351F09701A1E0BFEF0F94964600
:105CF00023E330E040E050E004CF2FEF30E0D70165
:105D00000F949E4623E330E040E050E059CF848179
:105D100091E069279EEF980F9C3018F08C528330E9
:105D2000C0F5812F0E9479BDF40185858823E9F0B3
:105D30002FEF30E0D7010F949E4629E130E040E09C
:105D400050E00F943246922F832F692F782F77FFE0
:105D500002C070E060E06F3F710519F014F06FEF62
:105D600070E0D40114968C9163CF9701A1E0BFEF4E
:105D70000F94964629E130E040E050E00F9432461F
:105D8000BA01A90141505F4F6F4F7F4F942F852F6C
:105D9000DCCF812F0E9479BD4DCF22242A94322C52
:105DA000411451046104710451F1D40117968D918D
:105DB0009C919C01990F440B550B29873A874B877F
:105DC0005C870E94DEC19B01AC0169857A858B8569
:105DD0009C85611571058105910509F4ABCEA12C57
:105DE000B12C65017B018C01C301B2010E94F42832
:105DF0008111A0CE7FEF2716370609F03FCEED8444
:105E0000FE848FE7E81AF1083DCE312C212C30CEEC
:105E100022242A94312C2CCE1F93CF93DF9300D0D1
:105E200000D0CDB7DEB76130710509F468C05CF40D
:105E3000672B09F45AC067EF7DE08CEB9FE00F946D
:105E4000571680E048C06230710571F0633071050B
:105E500091F79093600D80935F0D55275093620DDD
:105E60004093610D84E009C09093600D80935F0DB5
:105E70005093620D4093610D83E00E9404C3182F7C
:105E800080E00E94E4296093640A7093650A80931D
:105E9000660A9093670A1123D9F062EE7DE085E1EE
:105EA0009FE00F945716812F90E0B0E0A0E0898327
:105EB0009A83AB83BC8380E190E09E838D83BE0197
:105EC0006F5F7F4F85E19FE00E9450FE0F94EB14BF
:105ED00081E01111B6CF26960FB6F894DEBF0FBE43
:105EE000CDBFDF91CF911F9108959093600D809366
:105EF0005F0D5093620D4093610D81E0BECF909392
:105F0000600D80935F0D5093620D4093610D82E0B0
:105F1000B4CFAF92BF92CF92DF92EF92FF920F93E6
:105F20001F93CF93DF93EC018C819D81892B61F4CA
:105F30000A811B8184E190E00F94983CBC01C80168
:105F40000E94B4E39D838C830C811D810115110592
:105F500069F46EEC7DE085E19FE00F94571685E1D2
:105F60009FE00F94EB1490E080E0A0C180E00E94DD
:105F7000E429D80116966D937D938D939C93199780
:105F8000CC80DD80C114D104D9F0EA81FB81309747
:105F9000B9F0048115810115110591F0F801808592
:105FA0008F70853069F4C8010E9439AF823040F0AB
:105FB000E090550AF090560AE114F10409F086C009
:105FC00061E97DE085E19FE00F94571661E070E0A4
:105FD0008C819D81892B11F470E060E04AE050E0F3
:105FE00085E19FE00F94F8156FE87DE085E19FE083
:105FF0000F94571661E070E08A819B81892B11F420
:1060000070E060E04AE050E085E19FE00F94F81511
:106010006DE87DE085E19FE00F945716EA81FB81F2
:1060200061E070E084819581892B11F470E060E07B
:106030004AE050E085E19FE00F94F8156BE87DE0C1
:1060400085E19FE00F945716EA81FB810480F5817A
:10605000E02D80858F7061E070E0853011F470E094
:1060600060E04AE050E085E19FE00F94F81569E8B0
:106070007DE085E19FE00F945716EA81FB818481E2
:1060800095810E9439AF61E070E0823010F070E0DD
:1060900060E04AE050E085E19FE00F94F81585E16B
:1060A0009FE00F94EB1466EA7DE085E19FE00F949A
:1060B000571685E19FE00F94EB14E881F981048481
:1060C000F585E02D61E0CE0119954DCF61E0C80165
:1060D0000E94A8AE8C01DC0118968C9118978F70E5
:1060E000843031F419966D917C916115710539F404
:1060F00061E77DE085E19FE00F945716D0CFC7019F
:106100000E94F6AD7C01009771F46FE47DE085E1BB
:106110009FE00F945716F8016185728585E19FE035
:106120000F944116BCCF65E276E00E94F6AD009771
:1061300009F4DAC0DC0118962C9118972F702430DE
:1061400009F0D2C01996AD90BC9010E000E0A11407
:10615000B10409F4BCC0B801695F724FC5010F9466
:10616000D13E892B09F0ADC0F801E55FF24F2591D2
:106170003491922F832FF601928383836CE276E031
:10618000C7010E94F6ADEC81FD81009709F4B4C00F
:10619000DC0118962C9118972F70223009F0ACC0B2
:1061A00019964D915D916D917C911C97411551050A
:1061B0006105710509F4A0C051834083408151817C
:1061C000052E000C660B770B22818DE59CE00F9469
:1061D000A41761E376E0C7010E94F6AD6C010C8163
:1061E0001D81009709F495C0FC0180858F70863071
:1061F00009F08FC066E376E0C6010E94F6ADD801D3
:106200001B969C938E931A976BE376E0C6010E94CF
:10621000F6ADF801958784876FE376E0C6010E94AA
:10622000F6ADD8011F969C938E931E9765E476E099
:10623000C6010E94F6ADF801918B808B6AE476E08E
:10624000C6010E94F6AD009709F45BC0DC01199607
:106250008D919C91F8019583848360E576E0C70178
:106260000E94F6ADD80153969C938E93529769EB9A
:106270007DE08BE09FE00F945716EA81FB8102805E
:10628000F381E02D608171818BE09FE00F944116D6
:106290008BE09FE00F94EB14E881F9810484F5858D
:1062A000E02D62E0CE01199581E090E0DF91CF9181
:1062B0001F910F91FF90EF90DF90CF90BF90AF9024
:1062C00008950A5F1F4F0834110509F040CF6AEEA8
:1062D0007CE08CEB9FE00F9457168CEB9FE00F94C3
:1062E000EB1496E080E047CF86E090E0D60113966D
:1062F0009C938E93129742CF80E895E2918380839E
:106300005DCF88EE93E0D80115969C938E931497F9
:10631000A4CFF8011386128688EE93E095838483D8
:10632000158614869ACFCF92EF92FF920F931F9308
:10633000CF93DF9300D000D01F921F92CDB7DEB76E
:106340007C0109831A832B833C834D835E836F8397
:1063500078876BE77CE08CEB9FE00F945716CE01BB
:1063600001960E94A9748981811129C00B81013095
:1063700071F128F010E00230E9F5CC20E9F060E09E
:10638000CE0101960E947670F70102811381892B5C
:1063900069F0C8010E9448E4672B682B692B61F4FF
:1063A00080E00E94E429AB01BC0103C040E050E062
:1063B000BA01C8010E9407E481E090E02EC080315C
:1063C000D0F58E30D8F58130C9F18230D9F16EE642
:1063D0007CE08CEB9FE00F9457164AE050E0698117
:1063E0008CEB9FE00F940E158CEB9FE00F94EB1459
:1063F00001E010E06EE57CE08CEB9FE00F94571617
:106400004AE050E0B8018CEB9FE00F94F8158CEB5C
:106410009FE00F94EB1490E080E028960FB6F8947C
:10642000DEBF0FBECDBFDF91CF911F910F91FF90C7
:10643000EF90CF9008958351833048F6F7010281A1
:106440001381A7CF40E050E0BA01F7018281938128
:10645000B1CF4F925F926F927F928F929F92AF9245
:10646000BF92CF92DF92EF92FF920F931F93CF9341
:10647000DF93CDB7DEB72C970FB6F894DEBF0FBE13
:10648000CDBF6D7F6130710509F4C0C0DC0112968B
:10649000ED90FC90E114F10409F4B8C04C01C7017F
:1064A0000E9448E42B013C0161E070E0C7010E94BA
:1064B000A5E4411451046104710409F4A7C020E06B
:1064C00030E04AE754E40F942C450F949F476987C6
:1064D0007A878B879C87672B682B692B09F496C07A
:1064E0000E94DEC19B01AC01A12CB12C6501E984A5
:1064F000FA840B851C85C301B2010E94F42888230D
:1065000009F484C0F4016280738070E060E0C3012C
:106510000E94A5E420E030E048EC52E40F942C45C2
:106520000F949F476B017C0180E00E94E429AB013E
:10653000BC01C3010E9407E419821A821B821C82DB
:106540001D821E821F8218868A81807F8A83D401E1
:1065500012966D917C9140E053E0CE0101960E942D
:10656000B36FCE0101960E941F722B013C0164E5BE
:1065700076E08CEB9FE00F9441162AE030E0B30107
:10658000A2018CEB9FE00F94061563E676E08CEB9E
:106590009FE00F9441162AE030E0B701A6018CEB92
:1065A0009FE00F9406158CEB9FE00F94EB14C40C46
:1065B000D51CE61CF71C8A81807F86608A83CD8289
:1065C000DE82EF82F886F4016281738140E052E05E
:1065D000CE0101960E94726E67E676E08CEB9FE03A
:1065E0000F9441162AE030E0B701A6018CEB9FE042
:1065F0000F9406158CEB9FE00F94EB1460E072E0B3
:10660000D40112968D919C910E94648090E080E06C
:106610002C960FB6F894DEBF0FBECDBFDF91CF91A1
:106620001F910F91FF90EF90DF90CF90BF90AF90B0
:106630009F908F907F906F905F904F9008950F93F1
:106640001F93CF93DF93DC0112962D913C91232B66
:1066500081F1EC0163E27BE08CEB9FE00F94571635
:106660004AE050E06E818CEB9FE00F940E158CEBAE
:106670009FE00F94EB148C819D81892B61F40A813A
:106680001B818CE290E00F94983CBC01C8010E94F1
:10669000B4E39D838C83EC81FD81309769F461E1E3
:1066A0007BE085E19FE00F94571685E19FE00F9412
:1066B000EB1490E080E044C085E2DF011D928A95F2
:1066C000E9F7EC81FD8116A2EC81FD8115A2EC8138
:1066D000FD8117A20C811D8180E00E94E429F80150
:1066E00060A771A782A793A78E81811116C062E06F
:1066F0000E94A7BD68ED7AE08BE09FE00F945716EB
:106700008BE09FE00F94EB148FE19FE00F94B80DA6
:106710001092450281E08093211126E040E855E285
:1067200060E070E08F8198850F94A417E881F9816B
:106730000484F585E02D62E0CE01199581E090E0BA
:10674000DF91CF911F910F9108956F927F928F9259
:106750009F92AF92BF92CF92DF92EF92FF920F93F0
:106760001F93CF93DF93EC018C819D81892B09F4DA
:10677000A8C08A819B81892B09F4A3C03A014B01EF
:10678000E881F9810284F385E02DCE011995039704
:1067900001F5EC81FD8180A591A5A2A5B3A5892B6A
:1067A0008A2B8B2BB1F00E94DEC19B01AC01EC81E6
:1067B000FD8160A571A582A593A5A12CB12C6501D1
:1067C00016E9E12EF12C00E010E00E94F428882365
:1067D00001F38F81988521E0621A7108DC01ED9147
:1067E000FC910280F381E02DA301B40119958F8102
:1067F0009885DC01ED91FC910190F081E02DD401B0
:10680000129660E09D01281939092615370518F4FC
:106810002D91620FF7CF19950C811D8180E00E94A8
:10682000E429F80160A771A782A793A763ED7AE036
:106830008CEB9FE00F9457164AE050E06E818CEB92
:106840009FE00F940E156FEC7AE08CEB9FE00F94B5
:1068500057168401C8018819990986159705B8F457
:10686000D8016C9140E150E06A3050F46CE776E07A
:106870008CEB9FE00F94411640E150E0F8016081FD
:106880008CEB9FE00F940E150F5F1F4FE3CF8CEB47
:106890009FE00F94EB14E881F9810484F585E02DE5
:1068A00063E0CE01DF91CF911F910F91FF90EF90A8
:1068B000DF90CF90BF90AF909F908F907F906F9020
:1068C0001994DF91CF911F910F91FF90EF90DF907E
:1068D000CF90BF90AF909F908F907F906F900895D2
:1068E000CF92DF92EF92FF920F931F93CF93DF939C
:1068F000CDB7DEB762970FB6F894DEBF0FBECDBF3F
:106900006C010B871C872D873E874F87588B698BBF
:106910007A8B69E57CE0C7010F94D13EEEE0F0E0B0
:10692000892BF1F063E57CE0C7010F94D13EE0E1F3
:10693000F0E0892BA9F06DE47CE0C7010F94D13E13
:10694000EFE0F0E0892B61F01D8569E47CE0C70190
:106950000F94D13EE12FF0E0892B11F4EDE0F0E04F
:106960009B85992341F0309731F4EF2809F461C0F9
:106970008FEF9FEFD1C0E131F10508F03CC08827CF
:10698000EB53FB4C8F4F0D948746B8341935D634F2
:10699000FB34FB34FB34FB34CD358736FB34FB341E
:1069A000FB34FB34FB349136DA369F36CE010B963E
:1069B0000E94DB7120EF260F2931D0F6D601149604
:1069C000ED91FC91159723A39B01AC01332744273C
:1069D00055271296ED91FC9113970280F381E02DDB
:1069E00060817181ED91FC910684F785E02D0EE7C1
:1069F00016E0C6011995D6011496ED91FC911597F4
:106A0000118A1496ED91FC91159781E08187149677
:106A1000ED91FC9115978DE482871496ED91FC9190
:106A200015978FE5838714966D917C9145E250E030
:106A300048C0F6010481158180E00E94E429D80154
:106A400098966D937D938D939C939B97D601ED9132
:106A5000FC910484F585E02D64E0C6011995EB8571
:106A6000E150E53140F6F0E0D60114962D913C91CD
:106A700015978827E15CFA4C8F4F0D948746543563
:106A80006535FB34FB3465355435FB34FB34FB345E
:106A9000FB34FB34FB34FB349B35B335FB34FB3424
:106AA000FB34AF35AB35B135F90185A1858F14962F
:106AB000ED91FC91858D8160858F4DE050E06AE11C
:106AC00072E0C6010E94A53325C0F90185A1858F1A
:106AD0001496ED91FC91858D8E7F858F4DE050E071
:106AE0006DE072E0C6010E94A533D6011296ED91C9
:106AF000FC9113970280F381E02D60817181ED910B
:106B0000FC910288F389E02D23E836E04CEF56E053
:106B1000C601199581E090E062960FB6F894DEBF49
:106B20000FBECDBFDF91CF911F910F91FF90EF90DE
:106B3000DF90CF900895F901178AD6011496ED9150
:106B4000FC91159785A1858F1496ED91FC91858D0B
:106B50008160858F50CF81E0F901878BEECF82E095
:106B6000FBCF84E0F9CF83E0F901878B1496ED9198
:106B7000FC91159785A1858F1496ED91FC91159741
:106B8000858D8160858F1496ED91FC91818D833088
:106B900009F031CF82E0818F2ECF1982F601048176
:106BA00015819031F1F190F4923009F446C09E3095
:106BB000B9F0CE010B960E94DB716115710581055C
:106BC000910509F05BC0F80117A246C0913171F13F
:106BD000923179F782E0F801818F6AE07CE006C0AB
:106BE00083E0D80159968C9366EE7BE0CE01019646
:106BF0000F94DA3ED6011296ED91FC911397028024
:106C0000F381E02D60817181ED91FC910288F3891F
:106C1000E02D28E836E0AE014F5F5F4FC6011995C1
:106C2000EACEF801118E68EF7BE0E0CF81E0D80179
:106C300059968C9361E07CE0D9CFD80197961C924D
:106C40000481158180E00E94E429D80198966D9313
:106C50007D938D939C939B97D6011496ED91FC9117
:106C6000159785A1858F1496ED91FC91858D8E7F6A
:106C7000858F4DE050E06DE072E023CFD80197960C
:106C80001C926150710981099109660F771F881F55
:106C9000991F2EEF30E040E050E00F943246DA01C9
:106CA000C9010196A11DB11D813071F0A8F2823099
:106CB00029F1833009F09ECFD6011496ED91FC9115
:106CC000118E68EF7BE008C0D6011496ED91FC911F
:106CD00082E0818F6AE07CE0CE0101960F94DA3E7B
:106CE000D6011496ED91FC91159785A1858F149688
:106CF000ED91FC91858D8160858F7CCFD6011496B6
:106D0000ED91FC9181E0818F61E07CE0E5CFCE01E7
:106D10000B960E94DB71D6011496ED91FC91678B66
:106D20006ACED6011496ED91FC91913029F0923003
:106D300009F061CE148E5FCE80E5848F5CCEF601C3
:106D400004811581913049F09230F1F0CE010B961B
:106D50000E94DB71F801638F4ECE83E0D8015B9611
:106D60008C93D6010280F381E02D0280F381E02D27
:106D700060817181ED91FC910288F389E02D2DE80D
:106D800036E04BEE56E04ACFF801138ED60112964C
:106D9000ED91FC9113970280F381E02D6081718168
:106DA000ED91FC910288F389E02D2DE836E04CEF5F
:106DB00056E034CFD6011496ED91FC91913031F02C
:106DC000923009F018CE858D877FC3CE858D88607F
:106DD000C0CE8F929F92AF92BF92CF92DF92EF92EE
:106DE000FF920F931F93CF93DF937C014A015901C8
:106DF000C0915C0AD0915D0A062F660F110B209797
:106E000009F45CC088858F70863009F055C064E94C
:106E100076E0CE010E94F6AD6C0182E08816910406
:106E200049F065EF75E0E3E08E16910429F0D0E0BB
:106E3000C0E006C069E976E0CE010E94F6ADEC0143
:106E4000C114D104D9F1F60180858F708430B1F579
:106E500061857285A801C7010F94224BA80167E2E2
:106E600079E0C7010F94044B209779F188858F70E2
:106E7000843059F569857A85A801C7010F94044BC0
:106E8000A80167E279E0C7010F94044BA114B10493
:106E900029F0A801B501C7010F94044BC701DF9188
:106EA000CF911F910F91FF90EF90DF90CF90BF9007
:106EB000AF909F908F900895D0E0C0E0A8016DEB57
:106EC00073E1C7010F94083FC9CFF2E08F16910418
:106ED00081F083E08816910429F060915A0A70913C
:106EE0005B0ACACFA80167EB73E1C7010F94EA3EC2
:106EF000C7CFA80164EB73E1F8CFAF92BF92CF92F6
:106F0000DF92EF92FF921F93CF93DF9300D000D0D8
:106F1000CDB7DEB76C017C0110E08AE0A82EB12C61
:106F2000133061F1F701828190E0B0E0A0E0898345
:106F30009A83AB83BC83BE82AD82BE016F5F7F4FFD
:106F40008BE09FE00E9450FE62EB73E10F945716B6
:106F50001F5FFFEFEF1AFF0A143011F726960FB6E6
:106F6000F894DEBF0FBECDBFDF91CF911F91FF9090
:106F7000EF90DF90CF90BF90AF900895F60185819C
:106F800090E0B0E0A0E089839A83AB83BC83BE82AB
:106F9000AD82BE016F5F7F4F8BE09FE00E9450FE8D
:106FA00060EB73E1D3CFFC01DC018D918111FDCF4A
:106FB00030E020E050E040E08AE09191992301F137
:106FC000443051055CF59E3271F42F3F310509F0D4
:106FD0002CF5DB01A40FB51F12962C934F5F5F4F6A
:106FE00030E020E0EACF829FD001839FB00D1124D2
:106FF000292F990F330B205331092A0F3B1FDDCF67
:107000002F3F310509F054F4443051053CF4640F2E
:10701000751FFB01228381E090E0089590E080E0FD
:107020000895CF92DF92EF92FF920F931F93CF9329
:10703000DF93EC016A017B01CB01BA010F94984701
:107040008B011F936F938CE398E09F938F93DF9353
:10705000CF930F94794B0F900F900F900F900F904C
:107060000F9020E030E0A901C701B6010F94CE4790
:10707000181624F0F7FAF094F7F8F094099000202D
:10708000E9F721978EE28883B80117FF03C0719555
:1070900061957109072E000C880B990B0F94CD4454
:1070A0009B01AC01C701B6010F94B94620E030E066
:1070B00040E251E40F942C450F949847605D69833A
:1070C0001A82DF91CF911F910F91FF90EF90DF9087
:1070D000CF900895CF93DF931F921F92CDB7DEB765
:1070E0008091511290915212009711F48DE592E126
:1070F000BE016F5F7F4F681B790B072E000C880B5A
:10710000990B0F900F90DF91CF9108954F925F925E
:107110006F927F929F92AF92BF92CF92DF92EF9247
:10712000FF920F931F93CF93DF93CDB7DEB768978E
:107130000FB6F894DEBF0FBECDBFFC01198A1A8AC4
:107140001B8A1C8A1D8A1E8A1F8A188E9A89907F24
:1071500096609A8BA081B181109709F495C08C91AB
:10716000882309F491C000811181D8019C91992351
:1071700009F443C09D3209F4F3C090539A3028F0CB
:107180000F5F1F4F11830083EECFC801912CDC01EC
:107190006D01C81AD90A2D91022E000C330B205311
:1071A00031092A303105A0F37F016EE270E0C80199
:1071B0000F94E94AFC01009709F448C0DC015D0125
:1071C000AE1ABF0A11968C911197082E000C990BDC
:1071D000C09711960A9798F38181282F082E000CEA
:1071E000330B205331092A30310518F480330CF069
:1071F00072C020E030E0A90108C0912CD12CC12C34
:10720000D3CF29E030E040E050E0AAE0B0E00F94B6
:1072100051462B013C012281822F022E000C990B3A
:10722000C0978A30910570F420330CF45CC02A3387
:107230000CF05DC0092E000CAA0BBB0B480E591EAA
:107240006A1E7B1EA114B10409F056C0C8010F9438
:10725000833EAB01BC01CE0141960E948A6F298713
:107260003A874B875C876D877E878F87988B6CE228
:1072700070E0D7018D919C910F94E94A009709F035
:107280006AC0F7011182108288E0FE017196DE016A
:10729000119601900D928A95E1F729813A814B81EF
:1072A0005C816D817E818F81988568960FB6F89498
:1072B000DEBF0FBECDBFDF91CF911F910F91FF9029
:1072C000EF90DF90CF90BF90AF909F907F906F90A6
:1072D0005F904F9008958A330CF093CF032E000CEB
:1072E000440B550B92CF80E090E0DC01A7CF89E002
:1072F00090E0A0E0B0E0A2CFC801B3E0AB16B104CB
:10730000FCF4E8E0CE16D104DCF40F94833E9B013C
:10731000AC01A4E6B0E00F945146992041F070947E
:10732000609450944094411C511C611C711C460E89
:10733000571E681E791E4D8A5E8A6F8A788E97CF97
:107340000F94613E2A89207F27602A8B6D8B7E8B6C
:107350008F8B988F8CCF0196D7018D939C9394CF70
:10736000C80101969924939412CFCF92DF92EF92A5
:10737000FF920F931F93CF93DF93EC01A881B98104
:10738000109781F18C91882369F108811981F801A6
:107390009081992351F09D3241F090539A3028F01A
:1073A0000F5F1F4F19830883F0CFC8010F94833EEE
:1073B0006B017C016CE270E0C8010F94E94A009710
:1073C00069F419821882C701B601DF91CF911F912C
:1073D0000F91FF90EF90DF90CF90089501969983E1
:1073E0008883F1CFC12CD12C7601EDCF0097B1F17C
:1073F000FC01DB01AC01405F5F4F80E090812FE931
:10740000290F263098F497559295907F9C9321816F
:107410003FE9320F3630B0F42755922B9D933296C8
:10742000E417F50759F791E0892708952FEB290F05
:10743000263010F49753E8CF90539A3028F381E028
:1074400090E0E2CF3FEB320F363010F42753E5CF18
:1074500020532A3010F381E020E0DFCF80E0089550
:107460000097D1F0DC011696ED91FC913097A1F0D8
:1074700080858F70843021F481859285009771F426
:107480000680F781E02D309739F080858F70843049
:1074900019F481859285089590E080E0089508951B
:1074A0000F931F93CF93DF93EC010A811B8170E050
:1074B00060E0C8010E94EBE41816D4F48A8761E00A
:1074C00070E0C8010E94EBE4181619069CF4998735
:1074D000888762E070E0C8010E94EBE41816190684
:1074E00064F49C878B87DF91CF911F910F91089552
:1074F00083E0E4CF8BE290E0EACF88E590E0F1CF43
:1075000008950895089508950F931F93CF93DF93DF
:10751000EC011D860A811B8170E060E0C8010E94B9
:10752000EBE487FD44C08C838C818150853410F05E
:1075300080E28C8361E070E0C8010E94EBE487FD8B
:107540003BC08D838D818150853410F081E28D8325
:1075500062E070E0C8010E94EBE4863490F58E830F
:1075600063E070E0C8010E94EBE49C012150310906
:107570002115344040F59A87898764E070E0C8019E
:107580000E94EBE4813024E0920700F59C878B8712
:1075900065E070E0C8010E94EBE418161906CCF40F
:1075A00098878F83DF91CF911F910F9108958195D7
:1075B0008C8381E08D87B8CF81958D8381E08D8725
:1075C000C1CF1E82CDCF1A861986D7CF80E094E036
:1075D000DDCF80E197E2E4CFCF93DF93EC010E940F
:1075E000843A6EE976E08CEB9FE00F94EF1461E053
:1075F0008C810E94A7BD61E08D810E94A7BD6D8531
:107600008C810E9479BD6D858D810E9479BD60E07D
:107610008E810E94A7BD40E050E0BA018A819B8123
:107620000E9407E440E050E460E070E08A819B81C2
:107630000E9416E540E050E860E070E08A819B819E
:107640000E9416E5E881F9810484F585E02D62E069
:10765000CE01199582E08093270281E090E0DF91CE
:10766000CF910895089508950895CF93DF9300D0A2
:1076700000D01F921F92CDB7DEB7E5EFFEE0128A71
:10768000118A80E090E19587848784E890E0948B6C
:10769000838B81E0868787E7858B1C821B8288E548
:1076A00092E09A838983FE83ED838FEF9FEF988723
:1076B0008F836EE079E08BE09FE00F945716609126
:1076C000520A7091530ACE0101960E947FB985EF4C
:1076D0009EE00E9448DA6EEF78E08BE09FE00F9426
:1076E00057168BE09FE00F94EB140E949CCA2896DB
:1076F0000FB6F894DEBF0FBECDBFDF91CF910895D6
:10770000EF92FF921F93CF93DF93192F7B01C82F26
:10771000D92FD7FF03C0D195C195D10961E08C2F36
:107720000E94A7BD82E0E816F10499F460E08C2F76
:107730000E9479BD66EF78E08CEB9FE00F945716BE
:107740008CEB9FE0DF91CF911F91FF90EF900D9414
:10775000EB14612FEF2851F46095661F6627661FB2
:107760008C2F0E9479BD62EF78E0E6CF661F662716
:10777000661F8C2F0E9479BD6DEE78E0DDCF2F92D1
:107780003F924F925F926F927F928F929F92AF92B1
:10779000BF92CF92DF92EF92FF920F931F93CF93FE
:1077A000DF93CDB7DEB7CB57D1090FB6F894DEBF64
:1077B0000FBECDBF3C01362EE296EFAEE297E396C8
:1077C000FFAEE397E4960FAFE497E5961FAFE5971A
:1077D000E6962FAFE697E7963FAFE797E8964FAF6D
:1077E000E897E9965FAFE997EA96CFAEEA97EB960E
:1077F000DFAEEB97EC96AFAEEC972B2C2401009705
:1078000009F47CC1FC0180858F70843009F461C16A
:1078100028F4882309F466C180E02FC0853009F47C
:1078200046C08630C9F76AEA76E0C3010E94F6AD29
:107830002C01009709F476C0912C812CB12CA12C3D
:10784000D12CC12CE296EFACE297E396FFACE39724
:10785000E4960FADE497E5961FADE597E6962FAD5C
:10786000E697E7963FADE797E8964FADE897E9963C
:107870005FADE997632D0E94BF3BC558DF4F0FB640
:10788000F894DEBF0FBECDBFDF91CF911F910F9156
:10789000FF90EF90DF90CF90BF90AF909F908F9030
:1078A0007F906F905F904F903F902F9008958091C0
:1078B0003A118F5F80933A1166807780611471046A
:1078C00059F14201EC96AFACEC97B22CEA96CFACF2
:1078D000EA97EB96DFACEB97E296EFACE297E39694
:1078E000FFACE397E4960FADE497E5961FADE597FF
:1078F000E6962FADE697E7963FADE797E8964FAD52
:10790000E897E9965FADE997632DC3010E94BF3BFD
:10791000F30162807380D2CF80913A1181508093BD
:107920003A117ACF6EEA76E0C3010E94F6AD7C018F
:1079300063EB76E0C3010E94F6AD6C0168EB76E084
:10794000C3010E94F6AD332039F0F1E03F1609F48F
:10795000A1C010E000E00CC06CEB76E0C3010E9417
:10796000F6AD2C0161EC76E0C3010E94F6AD8C010E
:107970004114510409F423010115110509F483018F
:10798000E114F10431F4EA96EFACEA97EB96FFAC20
:10799000EB97C114D10421F4EC96CFACEC97D22C28
:1079A0004114510409F4A7C0F20180858F7084301E
:1079B00009F0A1C0618472840115110509F4AAC0FF
:1079C000F80180858F70843009F0A4C0418452840E
:1079D00010E000E0E114F10409F402C16114710443
:1079E00009F4BFC06AE074E18CEB9FE00F94571676
:1079F000F701618572858CEB9FE00F94411665E07D
:107A000074E18CEB9FE00F945716B3018CEB9FE071
:107A10000F9441168CEB9FE00F94EB14CE018F581E
:107A20009F4F0E94A974C114D10409F094C1F701B9
:107A300080858F70843009F08CC140914011509145
:107A4000411161857285CE0101960E942CE7CE011D
:107A500001960E94A7E38823C1F00E946A386B0157
:107A6000683C71050CF091C064EC73E185E19FE026
:107A70000F9457164AE050E0B60185E19FE00F945D
:107A8000F81585E19FE00F94EB14CE0101960E945A
:107A9000B6E75FC166EC76E0C3010E94F6AD2C014B
:107AA0006BEC76E0C3010E94F6AD8C0141145104E9
:107AB00009F056C16CEB76E0C3010E94F6AD2C01D3
:107AC0000115110509F44ECF892B09F059CF230177
:107AD00057CF10E000E0512C412CD12CC12CF12CBF
:107AE000E12C46CF10E000E0512C412CD12CC12CD0
:107AF000F12CE12C45CF712C612C5ECFEA96EFACD6
:107B0000EA97EB96FFACEB97EC96CFACEC97DB2CBF
:107B1000712C612C00E020E033E040E150E0BE0138
:107B20006F597F4FCE018F589F4F0E948B722C014F
:107B3000E4960FADE49710E00115110509F04ACF66
:107B4000E2968FADE297811109C0E3968FADE3977E
:107B50008F7009F43FCF02E010E03CCF01E010E06D
:107B600039CF6BEF73E18CEB9FE00F945716F70161
:107B7000618572858CEB9FE00F94411666EF73E18F
:107B80008CEB9FE00F94571649CF6114710431F0CC
:107B9000B301CE0101960E94AAB477CFA12CCC24C8
:107BA000C394F12CE12CE2960FADE297E3961FAD62
:107BB000E397E4962FADE497E5963FADE597E6961B
:107BC0004FADE697E7965FADE797E8966FADE8971C
:107BD000E9967FADE997CE0101960E94D4E955CF91
:107BE000C114D10409F4B5C04114510409F4B1C061
:107BF000F60180858F70843009F0A7C08185928559
:107C000025961FAE1EAE259748EE53E060E070E06B
:107C100029964CAF5DAF6EAF7FAF29972EE632E06D
:107C200023963FAF2EAF23972F969FAF8EAF2F9700
:107C300061961FAE1EAE619763961FAE1EAE639730
:107C400065961FAE1EAE659767961FAE1EAE679710
:107C500069961FAF0EAF69976A961FAE6A9740E4A8
:107C600050E0BE016F5F7F4FCE018F5B9F4F0E9440
:107C70009EAF21E030E02C0F3D1F820F931FFC01CF
:107C800010826EEE73E18CEB9FE00F945716F601B5
:107C9000618572858CEB9FE00F94411660ED76E074
:107CA0008CEB9FE00F944116BE016F5F7F4F8CEB12
:107CB0009FE00F94411669EE73E18CEB9FE00F9407
:107CC0005716B2018CEB9FE00F9441168CEB9FE0AE
:107CD0000F94EB140E9414AE8823B9F180913911EE
:107CE000811133C06FE270E0CE0101960F94E94A32
:107CF000892B51F4F6012185328543E050E060E4A0
:107D0000CE0101960E94E93662EE73E18CEB9FE0B2
:107D10000F945716BE016F5F7F4F8CEB9FE00F945F
:107D200041166DED73E18CEB9FE00F945716B20195
:107D30008CEB9FE00F9441168CEB9FE00F94EB14BB
:107D4000B201CE0101960E947BC2E114F10409F058
:107D50006ECE81E092CD4114510409F049CF67CE37
:107D6000892B09F00DCEFECD8F929F92AF92BF92DC
:107D7000CF92DF92EF92FF920F931F93CF93DF93F7
:107D800000D000D01F921F92CDB7DEB7DC01129653
:107D9000ED91FC91309709F468C024813581232B43
:107DA00009F463C08C01662309F472C00E947B222F
:107DB000E62EB72E6C01D8011296ED91FC9102804F
:107DC000F381E02D6081718185E19FE00F94411680
:107DD0006BE172E185E19FE00F94571685E19FE02A
:107DE0000F94EB1420E030E0A9016E2D7B2DC6012D
:107DF0000F94CE4787FD39C06FE072E185E19FE0C7
:107E00000F9457164E2D5B2DB60185E19FE00E9421
:107E10001FB385E19FE00F94EB14D8011296ED910A
:107E2000FC9161E0848195810E94A8AE19821A823A
:107E30001B821C822A81207F2760F22E2E2D4E2D40
:107E40005B2DB6014D835E836F837887912C812CE7
:107E5000B12CA12CD12CC12CE9800B811C813E813D
:107E60004F8158856FEF0E94BF3B28960FB6F8945C
:107E7000DEBF0FBECDBFDF91CF911F910F91FF905D
:107E8000EF90DF90CF90BF90AF909F908F9008952C
:107E90000280F381E02D608171818BE09FE00F947F
:107EA000411668E272E18BE09FE00F9457168BE079
:107EB0009FE028960FB6F894DEBF0FBECDBFDF91CE
:107EC000CF911F910F91FF90EF90DF90CF90BF90D7
:107ED000AF909F908F900D94EB144F925F926F92A2
:107EE0007F928F929F92AF92BF92CF92DF92EF924A
:107EF000FF920F931F93CF93DF93CDB7DEB7E89731
:107F00000FB6F894DEBF0FBECDBF09AB1AAB2BABDB
:107F10003CAB4DAB5EAB6FAB78AFDC011496ED9133
:107F2000FC91309719F490E080E0CAC02081318143
:107F3000232BC9F33C01DC01ED91FC910284F38514
:107F4000E02D1995029779F78BA9E82EF12C19A944
:107F5000112321F0E114F10409F432C1823009F453
:107F6000D8C0B8F4882309F4D4C08130B9F06BE3E9
:107F700072E18CEB9FE00F9457164AE050E0B70196
:107F80008CEB9FE00F94F8158CEB9FE00F94EB14B3
:107F9000CACF833009F446C0893049F7D30112961D
:107FA000ED91FC9161E0848195810E94A8AE2C0145
:107FB00019A61AA61BA61CA61DA61EA61FA618AAB1
:107FC0008AA5807F8AA719A761E0CE0189960E94C1
:107FD0001D6F29A33AA34BA35CA36DA37EA38FA31C
:107FE00098A71150153108F0F4C1E12FF0E088276F
:107FF000E350F04C8F4F0D9487462241E440E94115
:10800000E941E941E941E941E941E9415141AD41F4
:10801000E941E94122412241E941E941E941224165
:10802000224122418AA98F7009F47DCFCE01C196E9
:108030000E949571D3011496ED91FC91668377832C
:108040008087918761E872E18CEB9FE00F9457166F
:10805000D3011296ED91FC910280F381E02D6081B5
:1080600071818CEB9FE00F94411663E772E18CEB1A
:108070009FE00F945716D3011496ED91FC91468121
:108080005781608571858CEB9FE00E941FB38CEB5C
:108090009FE00F94EB14F301E480F5800E94DEC1B1
:1080A000D70152966D937D938D939C935597D301F1
:1080B0001496ED91FC918689811119C081E090E0C0
:1080C000E8960FB6F894DEBF0FBECDBFDF91CF911B
:1080D0001F910F91FF90EF90DF90CF90BF90AF90E6
:1080E0009F908F907F906F905F904F900895168A29
:1080F00060E0C3010E94B43ED3011496ED91FC915F
:1081000080E090E0A0E0B0EC86879787A08BB18BF1
:10811000D5CF8AA98F7009F406CFCE01C1960E94EF
:108120009571D3011496ED91FC91628773878487D2
:1081300095876DE672E18CEB9FE00F945716D301A3
:108140001296ED91FC910280F381E02D60817181A6
:108150008CEB9FE00F94411662E672E18CEB9FE09E
:108160000F945716D3011496ED91FC9142855385D7
:10817000648575858CEB9FE00E941FB38CEB9FE0BC
:108180000F94EB14D3011296ED91FC9162E084817F
:1081900095810E94A8AE009709F490CF912C812C74
:1081A000B12CA12CD12CC12CE9A8FAA80BA91CA98F
:1081B0002DA93EA94FA958AD6FEF0E94BF3B7ECFBE
:1081C000EE24E394F12CEACE80913E1190913F1180
:1081D0000597F1F019821A821B821C821D821E8271
:1081E0001F8218868A81807F8A836BE0CE01019688
:1081F0000E943F6F912C812CB12CA12CD12CC12C31
:1082000079018A019B01AC016FEFC2010E94BF3B63
:10821000912C812CB12CA12CD12CC12CE9A4FAA435
:108220000BA51CA52DA53EA54FA558A96FEFC20112
:108230000E94BF3B60E074E0F301828193810E9461
:1082400064803CCF19821A821B821C821D821E828E
:108250001F8218868A81807F8A8340E050E061E037
:1082600070E0D30112968D919C910E9468E5672B76
:10827000682B692BA1F06BE0CE0101960E943F6F45
:10828000912C812CB12CA12CD12CC12C79018A01EB
:108290009B01AC016FEFC2010E94BF3BBFCF6AE000
:1082A000EBCF80913E1190913F11059771F061E005
:1082B000D30112968D919C910E94BEE660E071E020
:1082C000F301828193810E94648040E050E460E089
:1082D00070E0D30112968D919C910E943FE5912C04
:1082E000812CB12CA12CD12CC12CE9A4FAA40BA572
:1082F0001CA52DA53EA54FA558A96FEFC2010E9450
:10830000BF3BD301ED91FC910688F789E02DC301B5
:108310001995892B09F4F0CE19821A821B821C82CE
:108320001D821E821F8218868A81807F8A8361E077
:10833000CE0101960E943F6F29873A874B875C8761
:108340006D877E878F87988B79018A019B01AC01AD
:108350006FEFC2010E94BF3BCFCE912C812CB12C7C
:10836000A12CD12CC12CE9A4FAA40BA51CA52DA5E8
:108370003EA54FA558A96FEFC2010E94BF3BD30194
:10838000ED91FC910688F789E02DC3011995892BA1
:1083900009F094CE19861A861B861C861D861E86B9
:1083A0001F86188A8A85807F8A8762E0CE010996B7
:1083B0000E943F6F29833A834B835C836D837E8366
:1083C0008F83988779018A019B01AC016FEFC2010D
:1083D000F4CE60E572E18CEB9FE00F9457164AE013
:1083E00050E069A98CEB9FE00F940E158CEB9FE099
:1083F0000F94EB14BCCD2F923F924F925F926F92ED
:108400007F928F929F92AF92BF92CF92DF92EF9224
:10841000FF920F931F93CF93DF93CDB7DEB765978E
:108420000FB6F894DEBF0FBECDBF1C01DC01149661
:108430008D919C911597892B99F41296ED91FC9151
:10844000FA83E98389E190E00F94983CBC0189812B
:108450009A810E94B4E3D10115969C938E93149750
:10846000F101048115810115110569F460EB71E1D9
:1084700085E19FE00F94571685E19FE00F94EB1480
:1084800090E080E0FCC4D8011D921C920280F38130
:10849000E02DFD8BEC8B309791F0848195819A8350
:1084A0008983009761F0DC0118968C9118978F7082
:1084B000853029F4CD010E9439AF811190C066E763
:1084C00071E185E19FE00F94571661E070E0F101E2
:1084D00084819581892B11F470E060E04AE050E0DE
:1084E00085E19FE00F94F81564E771E185E19FE075
:1084F0000F94571661E070E0D10112968D919C9116
:10850000892B11F470E060E04AE050E085E19FE0E3
:108510000F94F81562E771E185E19FE00F9457161B
:10852000D1011296ED91FC9161E070E0848195811A
:10853000892B11F470E060E04AE050E085E19FE0B3
:108540000F94F81560E771E185E19FE00F945716ED
:10855000D1011296ED91FC910480F581E02D80858A
:108560008F7061E070E0853011F470E060E04AE007
:1085700050E085E19FE00F94F8156EE671E185E12A
:108580009FE00F945716D1011296ED91FC918481D2
:1085900095810E9439AF61E070E0823010F070E0A8
:1085A00060E04AE050E085E19FE00F94F81585E136
:1085B0009FE00F94EB146AE871E185E19FE00F946E
:1085C000571685E19FE00F94EB14D101ED91FC91DA
:1085D0000484F585E02D61E0C101199551CF60E07B
:1085E00089819A810E94A8AE9B8B8A8B009729F083
:1085F000FC0180858F70853039F064E571E185E19B
:108600009FE00F945716D3CF8A899B890E9439AF78
:108610008150883008F0AEC1E82FF0E08827EC5E8A
:10862000FC4B8F4F0D948746864459442C44B643E7
:10863000944394437B431C4367E08A899B890E944F
:10864000A8AEFC0190859F70933009F045C08185EC
:108650009285A385B48589839A83AB83BC8391E09B
:108660009D8366E08A899B890E94A8AEFC01908563
:108670009F70933009F049C081859285A385B485A8
:108680008E839F83A887B98791E09D8364E08A8960
:108690009B890E94A8AEFC0180858F70833009F011
:1086A00056C061857285838594850F949F474B01E1
:1086B00063E08A899B890E94A8AEFC0180858F7047
:1086C000833009F068C081859285A385B4858E8743
:1086D0009F87A88BB98B6CC0923069F461857285D5
:1086E000838594850F94CD4469837A838B839C839F
:1086F000A1E0AD83B6CF80E090E0AFE7B3E489833B
:108700009A83AB83BC831D82ACCF9230D9F4618550
:108710007285838594850F94CD446E837F8388878B
:108720009987A1E0AD83B2CF80E090E0AFE7B3E4FA
:1087300089839A83AB83BC831E821F821886198625
:108740001D82A4CF1E821F82188619869FCF40ECFF
:10875000842E47E2942E49E0A42EB12C823009F0F9
:10876000A7CF81849284A384B484A2CF50EC852EB9
:1087700057E2952E59E0A52EB12C80E090E0AFE7AE
:10878000B3E489839A83AB83BC831E821F821886DD
:1087900019861D828DCF823009F07BC0618572857C
:1087A000838594850F94CD446E877F87888B998BC2
:1087B00062E08A899B890E94A8AEFC0180858F7047
:1087C000833009F06BC0418452846384748461E017
:1087D0008A899B890E94A8AEFC0180858F708330B6
:1087E00009F087C081859285A385B4858A879B8798
:1087F000AC87BD8760E08A899B890E94A8AEFC0196
:1088000090859F70933009F0AAC0C184D284E3841C
:10881000F48420E030E0A901C701B6010F94C644FA
:1088200087FFD6C0F7FAF094F7F8F094A1E0B0E033
:10883000BB8BAA8BAC89BD891696ED91FC91808586
:108840008F70823009F4C7C0833009F40AC280E017
:1088500090E0A0EAB1E409C230EC832E37E2932E17
:1088600039E0A32EB12C80E090E0A0EAB0E48E873E
:108870009F87A88BB98B80E090E0AFE7B3E4898352
:108880009A83AB83BC831E821F82188619861D8241
:108890008FCF80E090E0A0EAB0E419CF823029F5D4
:1088A00061857285838594850F94CD442B013C01AD
:1088B0008ECF20EC822E27E2922E29E0A22EB12C20
:1088C00080E090E0A0EAB0E48E879F87A88BB98B08
:1088D00080E090E0AFE7B3E489839A83AB83BC8305
:1088E0001E821F82188619861D82412C512C32014E
:1088F0006ECF823079F561857285838594850F947A
:10890000CD446A877B878C879D8774CF90EC892EB6
:1089100097E2992E99E0A92EB12C80E090E0A0EA90
:10892000B0E48E879F87A88BB98B80E090E0AFE79B
:10893000B3E489839A83AB83BC831E821F8218862B
:1089400019861D82412C512C32014A865B866C8629
:108950007D8650CF1A861B861C861D864BCF923093
:1089600089F561857285838594850F94CD446B016B
:108970007C014FCF80EC882E87E2982E89E0A82ECC
:10898000B12C80E090E0A0EAB0E48E879F87A88BAE
:10899000B98B80E090E0AFE7B3E489839A83AB833F
:1089A000BC831E821F82188619861D821B8A1A8A22
:1089B000412C512C32014A865B866C867D86730180
:1089C000620138CF1B8A1A8AC12CD12C760132CF92
:1089D0001B8A1A8A2FCF61857285838594850F94AF
:1089E000CD44F8016287738784879587D8011696EE
:1089F0001D921D921D921C921997F80112821382EA
:108A0000148215820E94DEC1D80152966D937D9327
:108A10008D939C935597D1011496ED91FC91B1E003
:108A2000B68B908E878A61E0C1010E94B43EF1014D
:108A300004811581D8018D919C916BE371E1892BA3
:108A400009F0DDCD8CE390E00F94983C9D8B8C8BEE
:108A5000C8010296EC89FD89978F868F0496958FC1
:108A6000848F065F1F4F11A300A312AE12AA13AA90
:108A700014AA15AA80E090E0AFE7B3E486AB97AB09
:108A8000A0AFB1AF84E690E0A0E0B0E086A797A7E2
:108A9000A0ABB1AB8A899B89918F808F20E030E0B9
:108AA000A901C701B6010F94C64487FD8AC020E022
:108AB00030E0A9016A857B858C859D850F94C6442D
:108AC00087FD7FC020E030E0A901C301B2010F940F
:108AD000C64487FD76C081E090E0AC89BD895B9695
:108AE0009C938E935A97E1E0DB96EC93DB97CD92C3
:108AF000DD92ED92FC9213978A859B85AC85BD85AE
:108B0000EC89FD8984839583A683B783408651864B
:108B100062867386C486D586E686F7862DEC3CECA5
:108B20004CEC5DE36A857B858C859D850F942C4597
:108B30004B015C01AC89BD8950968D929D92AD929E
:108B4000BC9253972DEC3CEC4CEC5DE3C301B201BD
:108B50000F9426472B013C01EC89FD89448A558AF4
:108B6000668A778A8A899B89019759F5A7019601B8
:108B700060E070E0CB010F94B946AC89BD891C96CA
:108B80006D937D938D939C931F97A501940160E055
:108B900070E0CB010F94B946EC89FD89608B718B35
:108BA000828B938BA301920160E070E0CB010F9464
:108BB000B946AC89BD8954966D937D938D939C93F2
:108BC00057970E94DEC1EC89FD8986A497A4A0A8CE
:108BD000B1A8681979098A099B0962A373A384A3C0
:108BE00095A3D1011496ED91FC918C899D89918377
:108BF0008083009709F4DFCCDC01DA968C91DA9758
:108C0000811147C05E96ED91FC915F97C080D18045
:108C1000E280F380FD01C6A2D7A2E0A6F1A65C9691
:108C2000ED91FC9180819181A281B381EC89FD89D4
:108C300082A793A7A4A7B5A746A857A860AC71AC14
:108C4000A3019201C701B6010F94CE4718169CF4F8
:108C5000AC89BD8996964D925D926D927C92999762
:108C600018C081859285A385B485F8018287938792
:108C7000A487B587BBCEEC89FD8942A853A864A818
:108C800075A8A3019201C701B6010F94C64487FDE0
:108C9000DFCF81E0EC89FD8982AFFD81FF2309F4FC
:108CA00074C029813A814B815C816E817F81888586
:108CB00099850F94CE4787FF68C08E819F81A885D4
:108CC000B985EC89FD8982AB93ABA4ABB5AB898147
:108CD0009A81AB81BC8186AB97ABA0AFB1AF068D5B
:108CE000178DD801CD90DD90ED90FC90A7019601F5
:108CF00069817A818B819C810F94C64487FF26C04D
:108D000089819A81AB81BC81F80180839183A283A0
:108D1000B383AC89BD8996964D905D906D907C90A3
:108D20009997D696CD90DD90ED90FC90D997A701BC
:108D30009601C301B2010F94CE471816B4F4EC8922
:108D4000FD89C6A2D7A2E0A6F1A61FC0A701960181
:108D50006E817F81888599850F94CE471816CCF651
:108D60008E819F81A885B985CFCFAC89BD89D296E8
:108D7000CD90DD90ED90FC90D597A7019601C301B1
:108D8000B2010F94C64487FDDACF20E030E04AE715
:108D900054E46E857F85888999890F942C450F94BA
:108DA000984716161706ECF56B01770FEE08FF08CB
:108DB000C701B6010F94CD442B013C01C501B4019C
:108DC0000F94CB449B01AC01C301B2010F94264721
:108DD0004B015C01AC019B01AC89BD8950966D9142
:108DE0007D918D919C9153970F942C45EC89FD8931
:108DF000608B718B828B938BA5019401648975893B
:108E0000868997890F942647AC89BD8954966D93BE
:108E10007D938D939C935797FD01C6A6D7A6E0AA94
:108E2000F1AA6CE971E18BE09FE00F945716D10134
:108E30001296ED91FC910280F381E02D60817181A9
:108E40008BE09FE00F9441168BE09FE00F94EB14B2
:108E5000D1011496ED91FC9180E090E0A0E0B0EC9F
:108E600086879787A08BB18BD101ED91FC9104840B
:108E7000F585E02D62E0C101199581E090E06596ED
:108E80000FB6F894DEBF0FBECDBFDF91CF911F911B
:108E90000F91FF90EF90DF90CF90BF90AF909F9099
:108EA0008F907F906F905F904F903F902F9008959C
:108EB0002F923F924F925F926F927F928F929F92EA
:108EC000AF92BF92CF92DF92EF92FF920F931F93D8
:108ED000CF93DF93CDB7DEB7A9970FB6F894DEBF77
:108EE0000FBECDBF6130710509F40CC3DC011496CF
:108EF000ED91FC913097D9F481E090E0A9960FB6FE
:108F0000F894DEBF0FBECDBFDF91CF911F910F91BF
:108F1000FF90EF90DF90CF90BF90AF909F908F9099
:108F20007F906F905F904F903F902F900895208199
:108F30003181232B09F31C01DC01ED91FC910284AA
:108F4000F385E02D19950297B9F6F101028113819D
:108F50000115110589F2C8010E94DDE6823061F237
:108F600040E050E061E070E0C8010E9468E5672BD6
:108F7000682B692B09F6D1011496ED91FC910081C3
:108F80001181F80182AD882309F468C20E94DEC114
:108F900069A37AA38BA39CA3F80182A193A1A4A1A6
:108FA000B5A149A15AA16BA17CA1481B590B6A0B21
:108FB0007B0B86A597A5A0A9B1A9481759076A07F1
:108FC0007B0708F44BC2048CF58DE02D80819181E4
:108FD000A281B3818D8F9E8FAF8FB8A3D801909659
:108FE000ED91FC912D8D3E8D4F8D58A16081718149
:108FF000828193810F94B9464B015C01F80122A54F
:1090000033A544A555A56D8D7E8D8F8D98A10F94A8
:10901000B9466B017C01D80150962D913D914D913F
:109020005C915397C501B4010F942C45F80126A11A
:1090300037A140A551A50F94BA462B013C01D80198
:1090400096964D925D926D927C929997DB96BC912B
:10905000BDA3B11116C0F801248535854685578515
:10906000C701B6010F942C459B01AC01C301B201AD
:109070000F94B946D80196966D937D938D939C93EA
:109080009997F80146A057A060A471A4F6A9F98F9A
:10909000D801D796BC91BA8FF801F0ADFB8FD801FB
:1090A000D996BC91BC8F298D3A8D4F2F5B2FC30170
:1090B000B2010F94CE4718160CF008C2898D9A8D14
:1090C000AB8DBC8DF80186A397A3A0A7B1A7FDA186
:1090D000FF2309F413C2D8011C962D913D914D91A7
:1090E0005C911F97C501B4010F942C454B015C01A5
:1090F000F8012489358946895789C701B6010F943B
:109100002C459B01AC01D80196966D917D918D9176
:109110009C9199970F94B946A50194010F94BA4672
:109120006B017C019B01AC01698D7A8D8B8D9C8DCF
:109130000F94C64487FD1CC0F801F2A9F98FD8012D
:10914000D396BC91BA8FF801F4A9FB8FD801D596BC
:10915000BC91BC8F298D3A8D4F2F5B2FB601C70173
:109160000F94C64487FD04C0C98EDA8EEB8EFC8E48
:10917000D8015E96ED91FC91898D9A8DAB8DBC8D59
:1091800080839183A283B3838D8D9E8DAF8DB8A193
:10919000F80182A793A7A4A7B5A789A19AA1ABA11B
:1091A000BCA182A393A3A4A3B5A3D1011496ED916E
:1091B000FC9186898823A1F0C1010E947B226B016A
:1091C0007C0120E030E0A9010F94CE4787FD08C064
:1091D000D1011496ED91FC91C282D382E482F58292
:1091E0006FEE71E18CEB9FE00F945716D101129650
:1091F000ED91FC910280F381E02D608171818CEB17
:109200009FE00F94411669EE71E18CEB9FE00F94A3
:109210005716D1011496ED91FC91428553856485D2
:1092200075858CEB9FE00E941FB364EE71E18CEBBF
:109230009FE00F945716D1011496ED91FC91468151
:109240005781608571858CEB9FE00E941FB363EDB1
:1092500076E08CEB9FE00F944116D1011496ED91CE
:10926000FC9142815381648175818CEB9FE00E9467
:109270001FB360EE71E18CEB9FE00F945716D101A4
:109280001496ED91FC910190F081E02D4081518187
:10929000628173818CEB9FE00E941FB36CED71E1E2
:1092A0008CEB9FE00F945716D1011496ED91FC9131
:1092B0000190F081E02D44815581668177818CEBAE
:1092C0009FE00E941FB368ED71E18CEB9FE00F946B
:1092D0005716D1011496ED91FC910190F081E02D8B
:1092E00040855185628573858CEB9FE00E941FB39A
:1092F000D1011496ED91FC918689882331F061EDBE
:1093000071E18CEB9FE00F9457168CEB9FE00F946C
:10931000EB14F10104811581D80156968C918111CD
:10932000EBCDE280F38061E0F701848195810E94BA
:10933000A8AE3C0120E030E0A901D8011E966D9155
:109340007D918D919C9151970F94C64481110CC0D1
:1093500020E030E0A901F801628173818481958168
:109360000F94CE4718165CF040E050E460E070E0E7
:10937000C7010E9468E5672B682B692B31F11982C0
:109380001A821B821C821D821E821F8218868A817D
:10939000807F8A8361E0CE0101960E943F6F29871A
:1093A0003A874B875C876D877E878F87988B912C58
:1093B000812CB12CA12CD12CC12C79018A019B01CB
:1093C000AC016FEFC3010E94BF3B40E050E460E09E
:1093D00070E0D10112968D919C910E9416E5D10109
:1093E0001496ED91FC914281538164817581198AB3
:1093F0001A8A1B8A1C8A8A89807F87608A8B4D8B98
:109400005E8B6F8B788F62E0CE0141960E941D6F5C
:1094100029833A834B835C836D837E838F83988714
:10942000912C812CB12CA12CD12CC12CE988FA884B
:109430000B891C892D893E894F89588D6FEFC30197
:109440000E94BF3BD1011496ED91FC9182819381E2
:10945000A481B58186879787A08BB18BD1011496A3
:10946000ED91FC918689811147CD8789908D009778
:1094700009F442CD28EE33E0829F7001839FF00C07
:10948000929FF00C11240E94DEC19B01AC01F101FE
:1094900084809580E114F10489F010E000E0D401AB
:1094A00052966D917D918D919C915597A12CB12CE7
:1094B00065010E94F428882309F41ECD81E0F4019F
:1094C000868B61E0C1010E94B43E16CDD801D296D0
:1094D0008D919D910D90BC91A02D8EA39FA3A8A7C7
:1094E000B9A79C01AD01C301B2010F94C64487FF27
:1094F000EECD8EA19FA1A8A5B9A5E4CD812C912C7C
:109500005401F6CD90E080E0F9CC2F923F924F923B
:109510005F926F927F928F929F92AF92BF92CF9203
:10952000DF92EF92FF920F931F93CF93DF93CDB70C
:10953000DEB7C257D1090FB6F894DEBF0FBECDBF5C
:10954000FC0162960FAF629763961FAF63976496B4
:109550002FAF649765963FAF659766964FAF669756
:1095600067965FAF679768966FAF689769967FAFAA
:10957000699786EF800F823008F414C5E396FFAE3A
:10958000EEAEE397A396FFAFEEAFA39730E0A196C0
:109590003FAF2EAFA1970023A1F12115310509F4AA
:1095A000E2C1273071F5013109F4A9C1023109F492
:1095B000CCC1003109F0DEC16FEF70E0CE018F5AEF
:1095C0009F4F0E9442702A962FAF2A972B963FAF4B
:1095D0002B972C964FAF2C972D965FAF2D972E96ED
:1095E0006FAF2E972F967FAF2F9760968FAF6097B4
:1095F00061969FAF619747E050E0A1965FAF4EAF95
:10960000A197A396AEADBFADA3971496ED91FC9133
:10961000309709F4ABC266807780AF961FAE1EAE5E
:10962000AF97A9961FAE1EAEA997A5961FAE1EAE08
:10963000A597512C412C312C212C6114710409F473
:10964000A1C26FE776E0C3010E94F6AD6B969FAFB3
:109650008EAF6B9764E876E0C3010E94F6AD6D961D
:109660009FAF8EAF6D9769ED76E0C3010E94F6ADB6
:10967000E1969FAF8EAFE1976B96EEADFFAD6B9726
:10968000309709F437C16D962EAD3FAD6D9721151A
:10969000310509F42FC180858F70823009F02AC10D
:1096A000D90118968C918F70823009F023C163E044
:1096B00076E0C3010E94F6ADDC0119962D913D9133
:1096C0004D915C911C97AD962CAF3DAF4EAF5FAF07
:1096D000AD97E396EEADFFADE397309709F4C0C0C8
:1096E000D301CD90DC90BF01C6010F94F44A892BC1
:1096F00009F0B6C062968FAD6297811142C1639640
:109700008FAD63978F70A196EEADFFADA1973797A0
:1097100009F0D3C1882309F47BC0CE018F5A9F4F33
:109720000E94DB716D96EEADFFAD6D9701851285E0
:1097300023853485672B682B692B09F4DEC1023041
:1097400011052105310529F00F3F1F4F2F4F3F4FC6
:1097500031F56DED76E08CEB9FE00F9441168CEBCC
:109760009FE00F94EB1421E030E040E050E06D9674
:10977000AEADBFAD6D9719962D933D934D935C9310
:109780001C9761E0CE018F5A9F4F0E943F6F29A323
:109790003AA34BA35CA36DA37EA38FA398A7CE018E
:1097A0008F5A9F4F0E94DB716B96EEADFFAD6B97AA
:1097B000618772878387948780913E1190913F11D2
:1097C000059731F1D301CD90DC90E12C23E0F22E0E
:1097D00062960FAD629763961FAD639764962FAD47
:1097E000649765963FAD659766964FAD66976796A9
:1097F0005FAD679768966FAD689769967FAD69971B
:10980000A396EEADFFADA397828193810E94427D26
:10981000E196EEADFFADE197309711F1912C812CDF
:10982000B12CA12CD12CC12C6296EFAC629763961F
:10983000FFAC639764960FAD649765961FAD65970F
:1098400066962FAD669767963FAD679768964FAD62
:10985000689769965FAD69976FEFCF010E94BF3B34
:109860006D96EEADFFAD6D9781859285A385B4852C
:1098700082309105A105B105B9F18F3F9F4FAF4FE0
:10988000BF4F91F16B96EEADFFAD6B9781859285E1
:10989000A385B485AB964EAD5FADAB97849F900129
:1098A000859F300D949F300D1124220E331EAF96EC
:1098B000EEADFFADAF97AF01FF0F660B770B48170B
:1098C00059076A077B0784F4AF969FAF8EAFAF97B7
:1098D000A9963FAF2EAFA997AB962EAD3FADAB97F4
:1098E000A5963FAF2EAFA597AB964EAD5FADAB97AC
:1098F000440E551ED30112966D907C909ECE60E86A
:1099000070E0CE018F5A9F4F0E94427022962FAF77
:10991000229723963FAF239724964FAF24972596FF
:109920005FAF259726966FAF269727967FAF27972D
:1099300028968FAF289729969FAF299787E090E0C8
:10994000A1969FAF8EAFA1975CCE6AE070E0CE018A
:109950008F5A9F4F0E944271A7E0B0E0A196BFAF1F
:10996000AEAFA1974ECEE1E0F0E0A196FFAFEEAF33
:10997000A19747CE27E030E0A1963FAF2EAFA19749
:1099800040CE482F50E070E060E06D96AEADBFADC8
:109990006D9719964D935D936D937C931C978130D1
:1099A00009F465C0823009F478C080913E1190912D
:1099B0003F11059779F16D96EEADFFAD6D978185FD
:1099C0009285A385B4850197A105B10519F56B961C
:1099D000EEADFFAD6B9781859285A385B4854497E5
:1099E000A105B105BCF42EE130E040E050E0218754
:1099F0003287438754876EE170E0CE018F5A9F4FC4
:109A00000E94427029A73AA74BA75CA76DA77EA723
:109A10008FA798AB80913E1190913F11059709F463
:109A2000F7CEF301C080D180E12C33E0F32E6296B3
:109A30000FAD629763961FAD639764962FAD6497E1
:109A400065963FAD659766964FAD669767965FAD35
:109A5000679768966FAD689769967FAD6997A3968B
:109A6000AEADBFADA39712968D919C91CFCE6B9664
:109A7000EEADFFAD6B9761857285CE018F5A9F4F1A
:109A80000E94427029AF3AAF4BAF5CAF6DAF7EAF73
:109A90008FAF21969FAF219788CF70E060E0CE0115
:109AA0008F5A9F4F0E94427029AB3AAB4BAB5CABD5
:109AB0006DAB7EAB8FAB98AF78CF882309F4A8CE7F
:109AC00060E0CE018F5A9F4F0E947670092E000CE5
:109AD000AA0BBB0B6B96EEADFFAD6B9781879287A0
:109AE000A387B48780913E1190913F11059709F4A7
:109AF0008FCEE12C92E0F92E9ACF0230110521058C
:109B0000310559F10F3F1F4F2F4F3F4F31F16EEE8F
:109B100076E08CEB9FE00F9441168CEB9FE00F9466
:109B2000EB1422E030E040E050E06D96AEADBFAD0A
:109B30006D9719962D933D934D935C931C9762E01E
:109B4000CE018F5A9F4F0E943F6F298F3A8F4B8FC4
:109B50005C8F6D8F7E8F8F8F98A36B96EEADFFAD70
:109B60006B97118612861386148626CEA9961FAE91
:109B70001EAEA997A5961FAE1EAEA597512C412CDF
:109B8000312C212C4114510409F40CC2C101B20141
:109B90000F9473468B016CE271E18CEB9FE00F94A4
:109BA00057164AE050E0B2018CEB9FE00F94F81595
:109BB00061E271E18CEB9FE00F945716EE24EA947A
:109BC000F12CC101B7010F9473464AE050E08CEBD1
:109BD0009FE00F94F8156AE171E18CEB9FE00F9420
:109BE00057164AE050E0B8018CEB9FE00F94F8154F
:109BF00060E171E18CEB9FE00F945716A9968EAD52
:109C00009FADA997B7010F9473464AE050E08CEBE3
:109C10009FE00F94F81569E071E18CEB9FE00F94E1
:109C200057164AE050E0A5966EAD7FADA5978CEB38
:109C30009FE00F94F81565E071E18CEB9FE00F94C5
:109C400057168CEB9FE00F94EB1419821A821B823B
:109C50001C821D821E821F8218868A81807F8A83D1
:109C60000115110509F459C0B801CE0101960E94F1
:109C7000427029873A874B875C876D877E878F87FD
:109C8000988B61E0CE0109960E943F6F79018A01AD
:109C90002B013C01298BFA8A4B8B1C8B6D8B5E8AC6
:109CA0008F8B788E61E07AE0A396EEADFFADA3973F
:109CB000848195810E94F6AD912C812CB12CA12C30
:109CC000D12CC12C9201A3016FEF0E94BF3BA39640
:109CD000AEADBFADA3971496ED91FC91309709F00E
:109CE00044C081E090E0CE58DF4F0FB6F894DEBF5D
:109CF0000FBECDBFDF91CF911F910F91FF90EF90DD
:109D0000DF90CF90BF90AF909F908F907F906F909B
:109D10005F904F903F902F90089570E060E0CE01EB
:109D200001960E94427079018A012B013C0129872A
:109D3000FA864B871C876D875E868F87788A61E0FD
:109D40007AE0A396EEADFFADA397848195810E9442
:109D5000F6AD912C812CB12CA12CD12CC12C9201CF
:109D6000A3016FEF0E94BF3BBCCF66807780A596B2
:109D70002EAD3FADA597032E000C440B550BA796B7
:109D80002CAF3DAF4EAF5FAFA797A9968EAD9FADFD
:109D9000A997092E000CAA0BBB0B6F968CAF9DAF39
:109DA000AEAFBFAF6F976114710409F49ACF63E04F
:109DB00076E0C3010E94F6AD7C0165EF75E0C3015A
:109DC0000E94F6AD6B969FAF8EAF6B976FE776E014
:109DD000C3010E94F6AD8C0164E876E0C3010E94E5
:109DE000F6AD6B96AEADBFAD6B97109709F4D2C0D0
:109DF0000115110509F4CEC0009709F4CBC01896DF
:109E00002C912F70223009F0C5C0F80120852F70E9
:109E1000223009F0BFC0DC0118962C9118972F70E2
:109E2000223009F0B7C0F701C184D284E384F484FE
:109E3000C114D10409F4AEC019968D919D910D9075
:109E4000BC91A02D82309105A105B10509F4A6C0F1
:109E50008F3F9F4FAF4FBF4F09F4A0C0A9962EADC3
:109E60003FADA997232B09F499C0D80119968D917C
:109E70009C918C9D80018D9D100D9C9D100D112439
:109E80002FEF30E0D8010F949E469601DD0C440B75
:109E9000550B0F943246A7966CAD7DAD8EAD9FAD40
:109EA000A7970F9400466F962CAD3DAD4EAD5FADBC
:109EB0006F970F94324619012A016EEF70E18CEB17
:109EC0009FE00F945716F301608171818CEB9FE046
:109ED0000F94411668EF70E18CEB9FE00F945716DA
:109EE000C8016FEF70E00F9473464AE050E08CEBCE
:109EF0009FE00F94F81562EF70E18CEB9FE00F94F8
:109F000057162AE030E0B201A1018CEB9FE00F94DC
:109F1000B0158CEB9FE00F94EB146B96EEADFFAD9C
:109F20006B9781859285A385B48582159305A405D9
:109F3000B50581F119861A861B861C861D861E862C
:109F40001F86188A8A85807F8A87B101CE0109968B
:109F50000E94427029833A834B835C836D837E83A6
:109F60008F839887912C812CB12CA12CD12CC12CC2
:109F700079018A019B01AC016FEFC3010E94BF3BD5
:109F80006B96AEADBFAD6B9719962D923D924D92EB
:109F90005C921C97F3016280738005CF212C312CD9
:109FA0002101BBCF90E080E09ECE2F923F924F9256
:109FB0005F926F927F928F929F92AF92BF92CF9259
:109FC000DF92EF92FF920F931F93CF93DF93CDB762
:109FD000DEB7CE56D1090FB6F894DEBF0FBECDBFA7
:109FE000A5969FAF8EAFA5971A01A8962FAFA897F9
:109FF000AD961FAF0EAFAD97AF96FFAEEEAEAF977B
:10A00000A996CFAEA997A796BFAEAEAEA797DC0133
:10A010001496ED91FC910288F389E02D868097805B
:10A02000AB2839F4FE01EE59FF4FA796FFAFEEAF14
:10A03000A79781E0A796AEADBFADA7978C936B01B4
:10A04000F12CE12C8114910409F472C5A896BFADDE
:10A05000A897B13009F482C008F479C0B23041F059
:10A06000B33009F471C0D40112968D909C90EACF60
:10A0700060E077E0C4010E94F6AD11E0009799F32B
:10A08000FC0181859285A385B4858C159D05AE055F
:10A09000BF0549F765E076E0C4010E94F6ADAB96D6
:10A0A0009FAF8EAFAB97A596AEADBFADA5971296FD
:10A0B000ED91FC9162E0848195810E94A8AE3C0103
:10A0C000822D0E9402BB7C01A2961FAEA297198A24
:10A0D0001A8A1B8A1C8A1D8A1E8A1F8A188E8A89E0
:10A0E000807F8A8B69EF75E0C4010E94F6AD6C0138
:10A0F0006EEF75E0C4010E94F6AD5C01C114D1049D
:10A1000051F0F60180858F70843029F48185928525
:10A110000E94C61F182FEFEFE10FEB3008F06BC164
:10A120000E2E000CFF0B8827E756FF4A8F4F0D9429
:10A130008746B1503B5119516051FB51FB519A5127
:10A140008551AE51BF51D75164E077E093CF67E0BE
:10A1500077E0C4010E94F6AD1BE090CF6CE077E0A1
:10A16000F8CF1701512C412CA701FF0C660B770B80
:10A17000CE0141960E948A6F6A962FAF6A976B96BE
:10A180003FAF6B976C964FAF6C976D965FAF6D97C7
:10A190006E966FAF6E976F967FAF6F97A0968FAFEB
:10A1A000A097A1969FAFA19780914502893020F496
:10A1B000809144028930B8F16EED7EE08CEB9FE037
:10A1C0000F94571600E020E033E040E150E0BE017C
:10A1D0006F5F7F4FCE0141960E948B72BC018CEB6A
:10A1E0009FE00F94411662ED7EE08CEB9FE00F94B0
:10A1F0005716612F110F770B4AE050E08CEB9FE070
:10A200000F94F81560ED7EE08CEB9FE00F945716ED
:10A21000D4016D917C918CEB9FE00F9441168CEBF7
:10A220009FE00F94EB14A114B10409F0E8C0D12C05
:10A230009AC21701512C412CB201A701CE014196BF
:10A240000E94616F62962FAF629763963FAF6397EC
:10A2500064964FAF649765965FAF659766966FAFEC
:10A26000669767967FAF679768968FAF689769968E
:10A270009FAF699799CFFE24EF24FE241701512C3C
:10A28000412CB201A101CE0141960E948A6F2A960B
:10A290002FAF2A972B963FAF2B972C964FAF2C972B
:10A2A0002D965FAF2D972E966FAF2E972F967FAF7F
:10A2B0002F9760968FAF609761969FAF619774CF2D
:10A2C000FE24EF24FE241701512C412CB201A101E0
:10A2D000CE0141960E94616F22962FAF229723965E
:10A2E0003FAF239724964FAF249725965FAF2597CE
:10A2F00026966FAF269727967FAF279728968FAF22
:10A30000289729969FAF29974FCFFF241701512CEB
:10A31000412CB201A701CE0141960E94616F29AF85
:10A320003AAF4BAF5CAF6DAF7EAF8FAF21969FAFB3
:10A3300021973ACFEF2CFF241701512C412CB20169
:10A34000A701CE0141960E94616F29AB3AAB4BAB9E
:10A350005CAB6DAB7EAB8FAB98AF26CF1701512CAA
:10A36000412C8A89807F86608A8B2AE030E0D70181
:10A370000F949E466D8B7E8B8F8B988F15CF170118
:10A38000512C412C8A89807F87608A8BB701FF0C12
:10A39000880B990B0F94CD4420E030E048EC52E458
:10A3A0000F9426476D8B7E8B8F8B988FFDCEC101CE
:10A3B00024E0969587952A95E1F70E9402BBFFE07D
:10A3C0002F22332402C0969587952A94E2F7817054
:10A3D00099271C01512C412CB201AC01CE014196B0
:10A3E0000E94616F29A73AA74BA75CA76DA77EA71C
:10A3F0008FA798ABD9CE212C312C2101D5CEF501D8
:10A4000080858F708550823008F011CFB501CE0164
:10A4100041960E94C675298B3A8B4B8B5C8B6D8B5A
:10A420007E8B8F8B988F211102C03F7009F1809134
:10A430004502893008F430C26BE47EE08CEB9FE08B
:10A440000F94571600E020E033E040E150E0BE01F9
:10A450006F5F7F4FCE0141960E948B72BC018CEBE7
:10A460009FE00F9441168CEB9FE00F94EB14DFCE2E
:10A4700060E177E0C5010E94F6AD7C01009709F428
:10A48000D6CEDC0118968C918F70823009F4F3C01F
:10A49000843009F0CCCE80914502893020F480913F
:10A4A0004402893090F061E87EE08CEB9FE00F94ED
:10A4B0005716D70119966D917C918CEB9FE00F9404
:10A4C00041168CEB9FE00F94EB146114710409F4B6
:10A4D00040C3F30180858F70863009F038C3D701FF
:10A4E00019966D917C91C3010E94F6AD009709F415
:10A4F0002EC366E377E00E94F6AD6C01009709F485
:10A5000026C3FC0180858F70823009F020C38091C2
:10A510004502893020F4809144028930B8F06FE61A
:10A520007EE08CEB9FE00F945716D60119964D9163
:10A530005D916D917C911C972AE030E08CEB9FE05F
:10A540000F94B0158CEB9FE00F94EB14F70161852D
:10A550007285A596AEADBFADA5971496ED91FC9111
:10A56000828993890E94F6AD7C01009709F4EFC2BD
:10A5700069EF75E00E94F6AD009749F0FC01208577
:10A580002F70243021F4818592850E94C61FD60148
:10A5900019964D915D916D917C911C97CE014196DC
:10A5A0000E948A6F29A33AA34BA35CA36DA37EA349
:10A5B0008FA398A76EEF75E0C7010E94F6ADBC01AE
:10A5C000009791F0FC0190859F709550923060F457
:10A5D000CE0141960E94C675298B3A8B4B8B5C8BC2
:10A5E0006D8B7E8B8F8B988F80914502893020F404
:10A5F000809144028930D8F06AE57EE08CEB9FE0E0
:10A600000F94571600E020E033E040E150E0BE0137
:10A610006F5F7F4FCE0141960E948B72BC018CEB25
:10A620009FE00F9441168CEB9FE00F94EB14D60142
:10A6300018968C911897982F92959F7090FD87C2CD
:10A6400021E0A2962FAFA29791609295907F8F7094
:10A65000892B18968C93DD24D394A996BFADA99726
:10A66000BB2309F490C0AB964EAD5FADAB97452BC5
:10A6700009F489C07CC280914502893020F4809120
:10A6800044028930A8F06AEB7EE08CEB9FE00F94E7
:10A690005716F70141855285638574852AE030E0BD
:10A6A0008CEB9FE00F94B0158CEB9FE00F94EB14B4
:10A6B000D70119966D917D918D919C911C97AD96C6
:10A6C000EEADFFADAD978F0130E020E06017710770
:10A6D000820793070CF485C0AF964EAD5FADAF9780
:10A6E0008A0130E020E006171707280739070CF425
:10A6F00078C0AB014E1B5F0BDE01AF59BF4F5D0150
:10A70000C12CAF96EEACFFACAF978F01A8962FADE2
:10A71000A897A5968EAD9FADA5970E94D54F298B82
:10A720003A8B4B8B5C8B6D8B7E8B8F8B988F64E120
:10A7300077E08CEB9FE00F94411661E377E08CEBC0
:10A740009FE00F944116A2966FADA29770E04AE089
:10A7500050E08CEB9FE00F94F8158CEB9FE00F948A
:10A76000EB14DD24D394A996BFADA997BB2339F090
:10A77000AB96EEADFFADAB97EF2B09F0F8C16114CE
:10A78000710409F4CDC0F30180858F70863009F023
:10A79000C7C0D4016D917C91C3010E94F6AD3C010C
:10A7A000892B09F4BDC0A996BFADA99781E0BB2351
:10A7B00009F485C0D3011696ED91FC9180E03097A5
:10A7C00009F47DC081117BC0A081B181109729F06F
:10A7D0009C919F7B81E009F480E00280F381E02D71
:10A7E000EECF60EB7EE08CEB9FE00F945716F70105
:10A7F00041855285638574852AE030E08CEB9FE0CB
:10A800000F94B01561E97EE08CEB9FE00F94571632
:10A810008CEB9FE00F94EB1481E080935E0DCE01F2
:10A8200049969093E40D8093E30DA896FFADA89709
:10A830006F2F70E041E050E0D70119968D919C9107
:10A840000E940C2FD82E8823E9F0F70161857285CC
:10A850009E012F593F4F5901C12C7B018B01A896B6
:10A860002FADA89750E040E0A5968EAD9FADA5977F
:10A870000E94D54F298B3A8B4B8B5C8B6D8B7E8BDB
:10A880008F8B988F80E480935E0D83E69DE090939C
:10A89000E40D8093E30D67CF80914402893008F482
:10A8A000C6CCCACDA596EEADFFADA59762817381EA
:10A8B00040E051E0CE0141960E94726E60CFF301FC
:10A8C00090859F70953009F056C00681178166E328
:10A8D00077E0C8010E94F6AD7C01009709F4C6C07C
:10A8E000DC0118968C9118978F70823009F046C061
:10A8F00019968D919D910D90BC91A02D8215930577
:10A90000A405B50509F07CC0A796EEADFFADA797ED
:10A910001082DD2029F0A996FFADA997F111BFC0E3
:10A9200088E0FE017196DE01599601900D928A959C
:10A93000E1F7298D3A8D4B8D5C8D6D8D7E8D8F8DE0
:10A9400098A1C259DF4F0FB6F894DEBF0FBECDBF3E
:10A95000DF91CF911F910F91FF90EF90DF90CF90FB
:10A96000BF90AF909F908F907F906F905F904F902F
:10A970003F902F90089583018111A9CFD110CBCFA3
:10A98000A796AEADBFADA7978C91882349F2A99643
:10A99000BFADA997BB2321F262E076E0C8010E9417
:10A9A000F6ADA5969FAF8EAFA597009709F49DC011
:10A9B000FC0180858F70823009F097C08185928577
:10A9C000A385B48582159305A405B50509F08DC04E
:10A9D00080914502893020F480914402893050F002
:10A9E00065E17EE08CEB9FE00F9457168CEB9FE0C7
:10A9F0000F94EB14A796AEADBFADA7971C9290CF66
:10AA0000D70119962D923D924D925C921C978091A0
:10AA10004502893020F4809144028930F8F069E3DE
:10AA200077E08CEB9FE00F9441162AE030E0B20112
:10AA3000A1018CEB9FE00F94061567E477E08CEBA7
:10AA40009FE00F944116F401608171818CEB9FE0CF
:10AA50000F9441168CEB9FE00F94EB14D7011896DE
:10AA60008C9118978F7E18968C9388CF6CE37EE03C
:10AA70008CEB9FE00F945716F401608171818CEB91
:10AA80009FE00F9441168CEB9FE00F94EB14A20112
:10AA9000910166E377E0C8010E9494B76FCFA29658
:10AAA0008FADA297811108C0A796AEADBFADA79795
:10AAB0008C91882309F434CF912C812CB12CA12CBA
:10AAC000D12CC12CE988FA880B891C892D893E89F3
:10AAD0004F89588D6FEFC3010E94BF3B81E0A7965D
:10AAE000EEADFFADA79780831BCF912C812CB12CAD
:10AAF000A12CD12CC12CE988FA880B891C892D89BD
:10AB00003E894F89588D6FEFC3010E94BF3BA596C8
:10AB1000EEADFFADA597309709F402CFD30118969B
:10AB20008C9187FDFDCE2186328643865486F8CEF1
:10AB300019821A821B821C828A81807F8A831D82ED
:10AB40001E821F82188688E0FE013196ECCED12C41
:10AB500084CDA996EFADA997EE2309F4E1CEAB968B
:10AB60002EAD3FADAB97D12C232B09F4D9CEAB96AC
:10AB7000AEADBFADAB9718968C9118978F708230A1
:10AB800009F0FDCD19968D919D910D90BC91A02D50
:10AB900081309105A105B10509F484CE0297A10584
:10ABA000B10509F0ECCDA596AEADBFADA597129657
:10ABB0006D917C9140E052E07DCE2F923F924F927A
:10ABC0005F926F927F928F929F92AF92BF92CF923D
:10ABD000DF92EF92FF920F931F93CF93DF93CDB746
:10ABE000DEB768970FB6F894DEBF0FBECDBF611514
:10ABF000710509F491C05E8B498B9D8B8C8BFB0199
:10AC0000868097808114910409F486C0F4018085C0
:10AC10008F70823031F0853031F1F4018280938081
:10AC2000F1CF6184728441E050E069897E89C3017B
:10AC30000E940C2F882389F3B12CA12CCC24C3941F
:10AC400073018301298950E040E0B3018C899D891B
:10AC50000E94D54F29873A874B875C876D877E870F
:10AC60008F87988BDACFC4010E9439AF8230A9F662
:10AC700060E0C4010E94A8AEFC01C184D284E384D8
:10AC8000F48461E0C4010E94A8AEFC0121843284F6
:10AC900043845484388E2F8ADB8ACA8AA1014C19D6
:10ACA0005D094F5F5F4F69897E89C6010E940C2F45
:10ACB000882309F4B2CF80914502893020F4809135
:10ACC0004402893020F08CEB9FE00F94EB14712C40
:10ACD000612C6A897B89660D771D8F89988D86170F
:10ACE00097070CF49ACFB12CA12CCC24C3947101FA
:10ACF0000A891B892989A3018C899D890E94D54FC6
:10AD000029833A834B835C836D837E838F8398870B
:10AD10009FEF691A790ADDCF68960FB6F894DEBF07
:10AD20000FBECDBFDF91CF911F910F91FF90EF909C
:10AD3000DF90CF90BF90AF909F908F907F906F905B
:10AD40005F904F903F902F9008952F923F924F9297
:10AD50005F926F927F928F929F92AF92BF92CF92AB
:10AD6000DF92EF92FF920F931F93CF93DF93CDB7B4
:10AD7000DEB72D970FB6F894DEBF0FBECDBF6130A2
:10AD80007105D9F490E080E02D960FB6F894DEBFFF
:10AD90000FBECDBFDF91CF911F910F91FF90EF902C
:10ADA000DF90CF90BF90AF909F908F907F906F90EB
:10ADB0005F904F903F902F9008952091570A3091C7
:10ADC000580A232BF9F64C01DC01ED91FC91028429
:10ADD000F385E02D19950297A9F68091640A909168
:10ADE000650AA091660AB091670A892B8A2B8B2B82
:10ADF00079F4D4011296ED91FC9162E08481958101
:10AE00000E94A8AE9C838B83892BD9F4712CC5C377
:10AE10000E94DEC19B01AC016091640A7091650AD9
:10AE20008091660A9091670AA12CB12C650118ECFB
:10AE3000E12EF12C00E010E00E94F4288111D9CF1E
:10AE4000A1CFEB81FC8180858F708630F9F626805A
:10AE500037801D82712C2114310409F49AC3D10169
:10AE600018968C91982F9F702BEF290F223008F0A5
:10AE700090C3BD81B1118DC3282F22952F7087FFFC
:10AE800028C522FD26C5953009F09DC0F1018681B7
:10AE9000978162E076E00E94F6AD2C01892B09F4DF
:10AEA00018C521E030E03093580A2093570A7110FA
:10AEB00003C0C4010E942B26D2011996ED90FC908C
:10AEC00062E577E08CEB9FE00F944116D401129677
:10AED000ED91FC910280F381E02D608171818CEB1A
:10AEE0009FE00F94411665E676E08CEB9FE00F94AF
:10AEF0004116F101A080B180D4011496ED91FC912E
:10AF000063EC7FE0309759F0B501828993890E9404
:10AF1000F6AD8C01009709F058C060EA7FE085E14A
:10AF20009FE00F94571685E19FE00F94EB14662481
:10AF30006A94762C9701FF0C440B550B2E833F83AC
:10AF400048875987D20119968D919D910D90BC919A
:10AF5000A02D8A879B87AC87BD872E813F8148853E
:10AF600059858A859B85AC85BD85281739074A0791
:10AF70005B0709F473C48091640A9091650AA091FB
:10AF8000660AB091670A892B8A2B8B2B09F494CF20
:10AF90000E94DEC19B01AC016091640A7091650A58
:10AFA0008091660A9091670AA12CB12C650118EC7A
:10AFB000E12EF12C00E010E00E94F42881117CCFFA
:10AFC0000E9453A2CACFC10164CF60E077E00E9423
:10AFD000F6AD6C01892B79F467E077E0C8010E9437
:10AFE000F6AD6C016DE77FE0892B69F0F201808599
:10AFF0008F70806B8087D60118968C918F7082300D
:10B0000079F067E67FE085E19FE00F94571685E1D0
:10B010009FE00F94EB149EEF692E77247A948ACFE9
:10B020006EE577E0C8010E94F6AD3C01009709F497
:10B0300051C1FC0180858F70813009F06FC181851D
:10B04000882309F46BC1D20118968C91807F10E09F
:10B0500000E0803B11F002E010E06CE57FE08CEB5B
:10B060009FE00F945716B5018CEB9FE00F944116AB
:10B0700069E57FE08CEB9FE00F945716F601418560
:10B080005285638574852AE030E08CEB9FE00F9455
:10B09000B01567E677E08CEB9FE00F9441164AE02D
:10B0A00050E0B8018CEB9FE00F94F81565E676E070
:10B0B0008CEB9FE00F944116F1E0F0935E0D21E0E0
:10B0C00030E02C0F3D1F3093E40D2093E30D41E061
:10B0D00050E0B801D60119968D919C910E940C2FD9
:10B0E000182F80E00E94E4296093640A7093650A37
:10B0F0008093660A9093670A112309F40CC1D40166
:10B100001296ED91FC9162E0848195810E94A8AE37
:10B110003C01009709F4D5C0FC0180858F70863012
:10B1200009F0F9C0B501C3010E94F6AD3C010097DA
:10B1300009F4C7C0DC0118968C9118978F70853080
:10B1400019F416966D907C9066E377E0C3010E9437
:10B15000F6AD3C01009709F4B4C0FC0180858F7006
:10B16000823009F0AEC080914502893020F4809190
:10B170004402893028F162E57FE08CEB9FE00F9478
:10B180005716D30119964D915D916D917C911C9745
:10B190002AE030E08CEB9FE00F94B0156CE47FE088
:10B1A0008CEB9FE00F94571669817A814AE050E05A
:10B1B0008CEB9FE00F9408158CEB9FE00F94EB1441
:10B1C000F301418552856385748589819A81B0E058
:10B1D000A0E0481759076A077B0719F166E47FE08A
:10B1E0008CEB9FE00F945716B5018CEB9FE00F940A
:10B1F000411668E37FE08CEB9FE00F9457168CEBD1
:10B200009FE00F94EB14F0E4F0935E0D23E63DE035
:10B210003093E40D2093E30D8DEF682E77247A941C
:10B2200089CEF20181859285A385B4854817590797
:10B230006A077B0789F562E37FE08CEB9FE00F9460
:10B240005716B5018CEB9FE00F94411660E37FE049
:10B250008CEB9FE00F94571669817A814AE050E0A9
:10B260008CEB9FE00F9408156FE17FE08CEB9FE083
:10B270000F9457168CEB9FE00F94EB14F0E4F093CF
:10B280005E0D23E63DE03093E40D2093E30D0CEFDB
:10B29000602E77247A944ECE69E17FE08CEB9FE0BC
:10B2A0000F945716B5018CEB9FE00F9441166EEF8B
:10B2B0007EE08CEB9FE00F9457168CEB9FE00F9491
:10B2C000EB1430E430935E0D43E65DE05093E40D03
:10B2D0004093E30DD2011896EC91E295EF70E150A6
:10B2E0000FEF1FEFEB3008F066C0F0E0D6011996C3
:10B2F0002D913C918827E058F64A8F4F0D94874650
:10B300009159A6599159A6594D5A485A4D5A485AD9
:10B3100091599159595A712C612CD3CF712C612CB0
:10B32000D9CFF201818592853093E60D2093E50D0A
:10B330001092E80D1092E70D9093EA0D8093E90DBD
:10B3400086E00E9404C3082F10E035C0D201199690
:10B350008D919C919827892798273093E60D20930B
:10B36000E50D1092E80D1092E70D9093EA0D809391
:10B37000E90D86E00E9404C3082F10E0F2018185E8
:10B380009285A385B4853A2F2B2FD60119968D91DE
:10B390009C9101969093E60D8093E50D1092E80D37
:10B3A0001092E70D3093EA0D2093E90D86E00E949C
:10B3B00004C3080F111D80E00E94E4296093640A11
:10B3C0007093650A8093660A9093670A63EF7EE044
:10B3D0008CEB9FE00F9457164AE050E0B8018CEBDD
:10B3E0009FE00F94F81561EF7EE08CEB9FE00F94E7
:10B3F0005716B5018CEB9FE00F9441166EE677E08F
:10B400008CEB9FE00F944116F601418552856385D0
:10B4100074852AE030E08CEB9FE00F94B0156BEE62
:10B420007EE08CEB9FE00F945716D20119964D9158
:10B430005D916D917C911C972AE030E08CEB9FE050
:10B440000F94B0158CEB9FE00F94EB1401151105D0
:10B45000B9F4F20180858F70823091F46114710427
:10B4600079F0D30118968C918F70823049F48185E0
:10B470009285A385B485F30181879287A387B487DA
:10B4800091E080E0012B09F090E0692E782E52CDFA
:10B49000F20181859285992747CFF20181859285B6
:10B4A000A385B485892F9A2FAB2FBB27A7FDBA950B
:10B4B000F2CFD20119968C913093E60D2093E50DD1
:10B4C000882341F080E09FEF9093E80D8093E70D93
:10B4D00085E037CF90E080E0F7CFF1018085806490
:10B4E000808768E470E185E19FE00F945716D101F1
:10B4F0006D917C9185E19FE00F9441166AE370E1C4
:10B5000085E19FE00F945716F1018085982F929561
:10B510009F70292F2370233031F09F5F9295907F89
:10B520008F70892B808764E777E085E19FE00F9437
:10B530004116D10118966C916295637070E04AE0F3
:10B5400050E085E19FE00F94F81585E19FE00F94AE
:10B55000EB14BDC16CE270E185E19FE00F945716DA
:10B56000F1016081718185E19FE00F94411669E1ED
:10B5700070E185E19FE00F94571685E19FE00F94FD
:10B58000EB14D10118968C9118978F7018968C93A4
:10B590009EC11092580A1092570AD4011496ED9148
:10B5A000FC9124803580512C412C0E94DEC19B01EE
:10B5B000AC01211431044104510491F0D4011496DA
:10B5C000ED91FC916681778180859185A12CB12CCC
:10B5D0006501820171010E94F428882309F4CDC01D
:10B5E0008091640A9091650AA091660AB091670AF9
:10B5F000892B8A2B8B2B09F0A8C0EB81FC81EF2BC8
:10B6000009F0C2C0D4011496ED91FC918285938516
:10B61000892B69F484859585892B49F486859785DE
:10B62000892B29F480899189892B09F409C180919A
:10B630004502893020F4809144028930B8F063EFEC
:10B640007FE08CEB9FE00F945716D4011296ED919A
:10B65000FC910280F381E02D608171818CEB9FE091
:10B660000F9441168CEB9FE00F94EB1481E090E077
:10B670009093580A8093570A711003C0C4010E9426
:10B680002B26D4011496ED91FC916285738542E0DE
:10B6900050E0C4010E94DD55D4011496ED91FC9157
:10B6A0006485758543E050E0C4010E94DD55D401F6
:10B6B0001496ED91FC916685778550E040E0C401D9
:10B6C0000E94DD55D4011496ED91FC916089718939
:10B6D00041E050E0C4010E94DD558091450289306F
:10B6E00020F4809144028930B8F063EE7FE08CEB67
:10B6F0009FE00F945716D4011296ED91FC910280B1
:10B70000F381E02D608171818CEB9FE00F944116F5
:10B710008CEB9FE00F94EB140E94DEC12B013C01E7
:10B720000E94DEC19B01AC01A12CB12C650112E38A
:10B73000E12EF12C00E010E0C301B2010E94F428D8
:10B7400081117AC00E9453A2EBCF0E94DEC19B01FF
:10B75000AC016091640A7091650A8091660A9091CB
:10B76000670AA12CB12C650118ECE12EF12C00E048
:10B7700010E00E94F428811140CFD4011496ED917D
:10B78000FC918481958100CBAB81BC8118968C9112
:10B7900018978F70863009F035CF16960D911C9151
:10B7A0000115110509F42ECFF8018085982F9F709F
:10B7B0002BEF290F223008F025CF82958F7082FF62
:10B7C00005C08B708295807F892B8087D801189661
:10B7D0008C9182958370833059F56EE777E085E12F
:10B7E0009FE00F944116D4011296ED91FC910280D6
:10B7F000F381E02D6081718185E19FE00F94411616
:10B8000067E279E085E19FE00F944116F8016081DD
:10B81000718185E19FE00F94411685E19FE00F94CF
:10B82000EB14D80118968C9118978F7018968C93FA
:10B83000F80102811381B4CF1092580A1092570A6E
:10B84000F4010481158180E00E94E429D801169654
:10B850006D937D938D939C9319978FCFBDEF6B164E
:10B86000BFEF7B0609F476CE14F5FCEF6F16FFEF01
:10B870007F0621F16BE070E185E19FE00F945716A0
:10B88000F1016081718185E19FE00F94411660E0D4
:10B8900070E185E19FE00F94571685E19FE00F94DA
:10B8A000EB14D10118968C9118978F776FCE611495
:10B8B000710409F412CE6A946728E1F6D101189652
:10B8C0008C9118978F7018968C93B1E0BD83772474
:10B8D0007394F10122803380BECA8F929F92AF92FF
:10B8E000BF92CF92DF92EF92FF920F931F93CF936D
:10B8F000DF9300D000D01F921F92CDB7DEB7E98250
:10B90000FA820B831C832D833E834F835887DC018F
:10B910001296ED91FC91309791F1048115810115FA
:10B92000110569F1F80180858F70853041F57B0143
:10B93000C8010E9439AF823010F161E0C8010E9455
:10B94000A8AE0097E1F0DC0118962C912F702630FC
:10B95000B1F4B7010E94F6AD009789F0912C812CCB
:10B96000B12CA12CD12CC12CE980FA800B811C8137
:10B970002D813E814F8158856FEF0E94BF3B2896F5
:10B980000FB6F894DEBF0FBECDBFDF91CF911F91F0
:10B990000F91FF90EF90DF90CF90BF90AF909F906E
:10B9A0008F9008954F925F926F927F928F929F92A5
:10B9B000AF92BF92CF92DF92EF92FF920F931F93BD
:10B9C000CF93DF93CDB7DEB7C258D1090FB6F89445
:10B9D000DEBF0FBECDBFDC0114962D913C911597B3
:10B9E000232B09F44DC53B014C01ED91FC910284E0
:10B9F000F385E02D19958230910509F40EC1C4F547
:10BA000097FF3EC5F40187819085DC01ED91FC91A3
:10BA10000084F185E02D199585970CF4EAC0F401B6
:10BA20006481758145E250E0878190850F946D14A3
:10BA3000D40117968D919C91DC01ED91FC910084CD
:10BA4000F185E02D19957C01892B09F432C162E062
:10BA500070E080E090E00E94ECBFF4018781908567
:10BA6000DC01ED91FC910284F385E02D1995E0CF86
:10BA70008430910509F467C04CF1059719F66A9472
:10BA8000672809F0FCC061E57BE08CEB9FE00F9438
:10BA90007B164DE050E060E072E0C4010E94A533E7
:10BAA000D4011496ED90FC9080E00E94E429F70107
:10BAB00060A771A782A793A7D401ED91FC9104849C
:10BAC000F585E02D62E0C40119959CCFD401149650
:10BAD000ED91FC9180A591A5A2A5B3A5892B8A2BF8
:10BAE0008B2B09F48FCF0E94DEC19B01AC01D401E6
:10BAF0001496ED91FC9160A571A582A593A5A12C4A
:10BB0000B12C650116E9E12EF12C00E010E00E9455
:10BB1000F428882309F476CFD401ED91FC910484B4
:10BB2000F585E02D62E0C4011995F401E480F5800B
:10BB300080E00E94E429D70198966D937D938D93C0
:10BB40009C939B975FCFD4011496ED91FC9180A5B7
:10BB500091A5A2A5B3A5892B8A2B8B2BF1F10E946D
:10BB6000DEC19B01AC01D4011496ED91FC9160A55E
:10BB700071A582A593A5A12CB12C650118E8E12E31
:10BB800013E1F12E00E010E00E94F428882329F14F
:10BB9000D401ED91FC910484F585E02D65E0C401AC
:10BBA0001995F401E480F58080E00E94E429D70132
:10BBB00098966D937D938D939C939B97D401149647
:10BBC000ED91FC9117A26DE57BE08CEB9FE00F946B
:10BBD00057168CEB9FE00F94EB14F401878190854E
:10BBE000DC01ED91FC910084F185E02D1995892B04
:10BBF00019F481E090E045C062E070E080E090E000
:10BC00000E94ECBFF40187819085DC01ED91FC91ED
:10BC10000284F385E02D1995E0CFD4011496ED91BF
:10BC2000FC9180A591A5A2A5B3A5892B8A2B8B2B6E
:10BC300011F10E94DEC19B01AC01D4011496ED917B
:10BC4000FC9160A571A582A593A5A12CB12C6501DD
:10BC500018E8E12E13E1F12E00E010E00E94F42834
:10BC6000882349F0D401ED91FC910484F585E02D01
:10BC700065E0C40119956A94672809F4C3CE90E081
:10BC800080E0CE57DF4F0FB6F894DEBF0FBECDBFBA
:10BC9000DF91CF911F910F91FF90EF90DF90CF90A8
:10BCA000BF90AF909F908F907F906F905F904F90DC
:10BCB00008956CE47BE08CEB9FE00F9457164AE00C
:10BCC00050E0F40166818CEB9FE00F940E1567E461
:10BCD0007BE08CEB9FE00F945716D4011496ED9106
:10BCE000FC91EE0DFF1D608140E150E06A3078F478
:10BCF0006CE776E08CEB9FE00F944116D40114962C
:10BD0000ED91FC91EE0DFF1D40E150E060818CEB68
:10BD10009FE00F940E15BFEFEB1AFB0AE4E2EE165C
:10BD2000F104D9F6D4011496ED91FC91159784A1F4
:10BD300097A1891709F4BCC287A31496ED91FC91D1
:10BD4000EF961CAE1DAE1EAE1FAEEF97C158DF4F73
:10BD5000188219821A821B82CF57D040ED968FAD80
:10BD6000ED97807FED968FAFED9783A190E06C010A
:10BD7000B0E1CB0ED11C499708F094C2B5848789F5
:10BD800086A3118D738CD40114962D913C91858DD1
:10BD9000D90195968C93E48CF12C878DF401208148
:10BDA0003181A281B38112960D90BC91A02D6D912D
:10BDB0007C91D9015296ED91FC9121E937E04BEE4F
:10BDC00056E080FD02C04CEF56E0C4011995B0E882
:10BDD000EB16F10409F09EC0D4011296ED91FC918E
:10BDE00013970280F381E02D60817181ED91FC91C8
:10BDF0000288F389E02D28E937E04BEE56E0C401D4
:10BE000019956EE977E08CEB9FE00F944116D40111
:10BE10001496ED91FC914AE050E065A18CEB9FE017
:10BE20000F940E158CEB9FE00F94EB14D401149635
:10BE3000ED91FC91159785A12D913C91119712964A
:10BE40000D90BC91A02D12960D90BC91A02D6D91DE
:10BE50007C91D9015296ED91FC9129EA37E04BEEA5
:10BE600056E083FD02C04CEF56E0C4011995D401A1
:10BE7000ED91FC9111970288F389E02D12968D9136
:10BE80009C91DC0112968D919C91DC016D917C91CD
:10BE9000D40114968D919C91DC0195968C9120EBA8
:10BEA00037E04BEE56E081FD02C04CEF56E0C40196
:10BEB00019951982113009F400C208F442C01230F9
:10BEC00009F420C2133009F442C26CE37BE0CE01D6
:10BED00001960F94DA3E60E0CE0185589F4F0E9494
:10BEE0003F6F64962FAF649765963FAF65976696F0
:10BEF0004FAF669767965FAF679768966FAF689723
:10BF000069967FAF69976A968FAF6A976B969FAF76
:10BF10006B973BC0EF2809F074CFD4011296ED91D6
:10BF2000FC9113970280F381E02D60817181ED9186
:10BF3000FC910288F389E02D28E937E04CEF56E0C8
:10BF40005ECF68EF7BE0CE0101960F94DA3E60E1B0
:10BF5000CE0185589F4F0E943F6FE4962FAFE49724
:10BF6000E5963FAFE597E6964FAFE697E7965FAF6A
:10BF7000E797E8966FAFE897E9967FAFE997EA967B
:10BF80008FAFEA97EB969FAFEB97D4011296ED91A6
:10BF9000FC9113970280F381E02D60817181ED9116
:10BFA000FC910288F389E02D28E836E0AE014F5F6E
:10BFB0005F4FC4011995EC96EFACEC97ED96FFAC92
:10BFC000ED97EE960FADEE97EF961FADEF97C15838
:10BFD000DF4F2881CF57D040C058DF4F3881C0583D
:10BFE000D040CF57DF4F4881C158D040CE57DF4FA8
:10BFF0005881C258D04069E876E0C4010E946D5C67
:10C00000F40180819181A281B38112960D90BC913F
:10C01000A02D6D917C91DC015296ED91FC912DE863
:10C0200036E04CEF56E0772011F04BEE56E0C401BD
:10C0300019950D2C000CEE08FF08D4011296ED9115
:10C04000FC9113970280F381E02D60817181ED9165
:10C05000FC910684F785E02D0EE716E0A701960116
:10C06000C40119954B2C512C712C612CBFEFBB16C0
:10C07000A9F0D4011296ED91FC9113970280F381FF
:10C08000E02D60817181ED91FC910684F785E02DB2
:10C090000CEB17E0A3019201C40119951B861C86C5
:10C0A0001D861E861F86188A198A1A8A8C85807FAB
:10C0B0008C87B701A601CE010B960E948A6F2C9641
:10C0C0002FAF2C972D963FAF2D972E964FAF2E97D3
:10C0D0002F965FAF2F9760966FAF609761967FAF97
:10C0E000619762968FAF629763969FAF639779016E
:10C0F0008A019B01AC016FE776E0C4010E946D5C90
:10C100001B861C861D861E861F86188A198A1A8A17
:10C110008C85807F8C87B301A201CE010B960E9493
:10C120008A6F2B8B3C8B4D8B5E8B6F8B788F898FBF
:10C130009A8F63E0CE0143960E941D6F24962FAF25
:10C14000249725963FAF259726964FAF269727969B
:10C150005FAF279728966FAF289729967FAF2997CB
:10C160002A968FAF2A972B969FAF2B9779018A013A
:10C170009B01AC016DEB77E0C4010E946D5C1982FC
:10C18000D4011496ED91FC9186A1811105C166EE52
:10C190007BE0CE0101960F94DA3E6EE0CE01855829
:10C1A0009F4F0E943F6F2BAF3CAF4DAF5EAF6FAF65
:10C1B00021967FAF219722968FAF229723969FAF2C
:10C1C0002397D4011496ED91FC91159726A130E0A8
:10C1D00050E040E01296ED91FC9113970280F381BC
:10C1E000E02D60817181ED91FC910684F785E02D51
:10C1F00002EC17E0C4011995D4011496ED91FC915D
:10C2000085A180FD14C06AE77BE0CE0101960F9402
:10C21000DA3E62E0CE0185589F4F0E943F6F2B8728
:10C220003C874D875E876F87788B898B9A8BD4018B
:10C230001296ED91FC9113970280F381E02D6081BD
:10C240007181ED91FC910288F389E02D23E836E0BD
:10C25000AE014F5F5F4FC4011995EC96EFACEC97C0
:10C26000ED96FFACED97EE960FADEE97EF961FAD06
:10C27000EF97C158DF4F2881CF57D040C058DF4FCC
:10C280003881C058D040CF57DF4F4881C158D04087
:10C29000CE57DF4F5881C258D04064E876E0C401E1
:10C2A0000E946D5C60E47BE08CEB9FE00F9457167E
:10C2B0008CEB9FE00F94EB149CCC61E07CE0CE0112
:10C2C00001960F94DA3E61E1CE0185589F4F0E949E
:10C2D0003F6FAC962FAFAC97AD963FAFAD97AE9694
:10C2E0004FAFAE97AF965FAFAF97E0966FAFE09767
:10C2F000E1967FAFE197E2968FAFE297E3969FAF2B
:10C30000E39743CE6AE07CE0CE0101960F94DA3EDB
:10C3100062E1CE0185589F4F0E943F6FA4962FAFD8
:10C32000A497A5963FAFA597A6964FAFA697A796B9
:10C330005FAFA797A8966FAFA897A9967FAFA99769
:10C34000AA968FAFAA97AB969FAFAB971ECE66EE1D
:10C350007BE0CE0101960F94DA3E6EE0CE01855867
:10C360009F4F0E943F6F6C962FAF6C976D963FAFBB
:10C370006D976E964FAF6E976F965FAF6F97A09663
:10C380006FAFA097A1967FAFA197A2968FAFA2970C
:10C39000A3969FAFA397F9CD8130A9F46CE17CE01F
:10C3A000CE0101960F94DA3E64E1CE0185589F4F8D
:10C3B0000E943F6F2BAB3CAB4DAB5EAB6FAB78AF2E
:10C3C00089AF9AAFFECE8230A9F463E17CE0CE0162
:10C3D00001960F94DA3E63E1CE0185589F4F0E948B
:10C3E0003F6F2BA73CA74DA75EA76FA778AB89AB84
:10C3F0009AABE7CE8330A9F46FEE7BE0CE010196D5
:10C400000F94DA3E6FE0CE0185589F4F0E943F6F38
:10C410002BA33CA34DA35EA36FA378A789A79AA7DC
:10C42000D0CE8430A9F465E27CE0CE0101960F9471
:10C43000DA3E65E1CE0185589F4F0E943F6F2B8FFA
:10C440003C8F4D8F5E8F6F8F78A389A39AA3B9CE4F
:10C450008D3609F0B6CE6CE37BE0CE0101960F94E9
:10C46000DA3E60E0CE0185589F4F0E943F6F2B8BD4
:10C470003C8B4D8B5E8B6F8B788F898F9A8FA1CE83
:10C480008FEF9FEFFECB2F923F924F925F926F9272
:10C490007F928F929F92AF92BF92CF92DF92EF9254
:10C4A000FF920F931F93CF93DF93CDB7DEB76897BB
:10C4B0000FB6F894DEBF0FBECDBF3C018091630A7A
:10C4C00068EB7AE0882309F46AC161E070E080E0FB
:10C4D00090E00E94ECBFBE016F5F7F4F80E00E9442
:10C4E00004B8892B09F059C1898183FF56C144E002
:10C4F000BE016F5F7F4F82E00E94FEB8009791F40B
:10C5000029813A813227232732273093280D20931F
:10C51000270D2B813C813227232732273093260D8C
:10C520002093250D0E94D1B767E97AE08CEB9FE05C
:10C530000F9457166091270D7091280D90E080E0C0
:10C540000F94CB44562E798B8A8B492E462F572F2A
:10C55000682F792F8CEB9FE00E941FB36FE87AE081
:10C560008CEB9FE00F9457166091250D7091260D6E
:10C5700090E080E00F94CB446B8B7C8B8D8B9E8BFB
:10C58000AB01BC018CEB9FE00E941FB363E87AE033
:10C590008CEB9FE00F94571642E0BE016F5F7F4F18
:10C5A00081E10E94FEB849815A81542745275427CA
:10C5B000892B11F050E040E070E060E040935F0AAA
:10C5C0005093600A6093610A7093620A2AE030E037
:10C5D0008CEB9FE00F94B01520E030E44CE156E482
:10C5E000652D79898A89942D0F94C64487FF7AC076
:10C5F000D3011296ED91FC912080318068EC77E0B8
:10C60000C1010E94F6AD988F8F8B6CEC77E0C10171
:10C610000E94F6AD1C0119821A821B821C828A813B
:10C62000807F8760F82E8A83252D852D9989AA8998
:10C63000B42D8D839E83AF83B887912C812CB12C30
:10C64000A12CD12CC12CE9800B811C813E814F8112
:10C6500058856FEF8F89988D0E94BF3B19821A828F
:10C660001B821C828A81807F8760F82E8A832B89B7
:10C67000822F9C89AD89BE898D839E83AF83B887C5
:10C68000E9800B811C813E814F8158856FEFC1018C
:10C690000E94BF3B21ED37E0452D59896A89742DF1
:10C6A000C3010F94060C26ED37E04B895C896D8938
:10C6B0007E89C3010F94060C60915F0A7091600A35
:10C6C0008091610A9091620A2AE0AE014F5F5F4F4C
:10C6D0000F94753F4CED57E0BE016F5F7F4FC30174
:10C6E0000F94D00B62EE77E08CEB9FE00F94EF1489
:10C6F000BE016F5F7F4F80EE0E9404B8892B19F452
:10C7000019811F3F49F46AE57AE085E19FE00F94C3
:10C710007B1681E090E04DC0112331F06BE47AE0AC
:10C7200085E19FE00F94571615FF06C06EE37AE08F
:10C7300085E19FE00F94571614FF06C062E37AE08C
:10C7400085E19FE00F94571613FF06C064E27AE07C
:10C7500085E19FE00F94571612FF06C064E17AE06E
:10C7600085E19FE00F94571611FF06C065E07AE05F
:10C7700085E19FE00F94571610FF0BC06AEF79E038
:10C7800085E19FE00F94571685E19FE00F94EB142D
:10C79000C0CF112309F4BDCFF7CF6DE97AE08CEB60
:10C7A0009FE00F9457168CEB9FE00F94EB1490E0F2
:10C7B00080E068960FB6F894DEBF0FBECDBFDF9164
:10C7C000CF911F910F91FF90EF90DF90CF90BF908E
:10C7D000AF909F908F907F906F905F904F903F9021
:10C7E0002F9008952F923F924F925F926F927F9277
:10C7F0008F929F92AF92BF92CF92DF92EF92FF9271
:10C800000F931F93CF93DF93CDB7DEB760970FB62B
:10C81000F894DEBF0FBECDBF6130710579F42C01F5
:10C8200080915E0A811125C061EE79E085E19FE08B
:10C830000F94571685E19FE00F94EB1490E080E091
:10C8400060960FB6F894DEBF0FBECDBFDF91CF91DB
:10C850001F910F91FF90EF90DF90CF90BF90AF901E
:10C860009F908F907F906F905F904F903F902F9010
:10C87000089560ED79E08CEB9FE00F94571682E00D
:10C880000E941FC0692E712C40E150E0B3018CEB77
:10C890009FE00F94F8158FEF6816710409F42DC10D
:10C8A00064EE77E08CEB9FE00F94411680E00E94ED
:10C8B0001FC0BC0190E080E00F94CB4420E030E04A
:10C8C00040E857E30F942C4520E030E045E253E484
:10C8D0000F942C4520E030E040E252E40F94B9463A
:10C8E000762E272E382E692E462F572F682F792F18
:10C8F0008CEB9FE00E941FB369EC79E08CEB9FE02A
:10C900000F94571681E00E941FC0BC0190E080E0A8
:10C910000F94CB4420E030E040E857E30F942C45DF
:10C9200020E030E048EC52E40F942C4569877A8788
:10C930008B879C87AB01BC018CEB9FE00E941FB3EF
:10C9400068EE77E08CEB9FE00F94EF14D201129623
:10C95000ED91FC91E080F1806DEB77E0C7010E94E2
:10C96000F6AD9E878D876AEE77E0C7010E94F6AD2F
:10C97000988B8F87272D322D432D562D672D722DA5
:10C98000832D962D0F942E48811140C019821A8252
:10C990001B821C828A81807F8760F82E8A83272DE4
:10C9A000872D922DA32DB62D8D839E83AF83B887BF
:10C9B000912C812CB12CA12CD12CC12CE9800B8184
:10C9C0001C813E814F8158856FEF8D859E850E9429
:10C9D000BF3B19821A821B821C828A81807F8760FA
:10C9E000F82E8A832985822F9A85AB85BC858D8315
:10C9F0009E83AF83B887E9800B811C813E814F8184
:10CA000058856FEF8F8598890E94BF3B2EEE37E0E7
:10CA1000472D522D632D762DC2010F94060C21EF68
:10CA200037E049855A856B857C85C2010F94060CD9
:10CA30008091630A882309F45DC020E030E048EC6F
:10CA400051EC672D722D832D962D0F94C64487FDD2
:10CA500051C020E030E048E452E4672D722D832D70
:10CA6000962D0F94CE4718160CF444C020E030E009
:10CA700048EC52E469857A858B859C850F94CE4776
:10CA80001816C4F120E030E04AE754E469857A855D
:10CA90008B859C850F942C450F949F4766507F4F44
:10CAA0008F4F9F4F24EFC22EDD24D394E12CF12C25
:10CAB000A70196010F94104629831A8220E030E0E6
:10CAC0004AE754E4672D722D832D962D0F942C4543
:10CAD0000F949F476E557D498F4F9F4FA701960139
:10CAE0000F9410462B831C82BE016F5F7F4F85E041
:10CAF0000E9454B888EE93E0A3CE8CEB9FE00F9495
:10CB0000EB140E947F29F6CF0F931F93CF93DF93EF
:10CB1000EC010E94503A64EF77E08CEB9FE00F94B9
:10CB2000EF148091680A9091690A892B19F586E1C2
:10CB300090E00F94983C8C012B853C854A85042E0F
:10CB4000000C550B688579850F9462181093690A5B
:10CB50000093680AF8018681978197FD08C061E01B
:10CB60000E94A7BD60E0F80186810E9479BD81E046
:10CB7000F8018183E881F9810484F585E02D62E084
:10CB8000CE01199581E090E0DF91CF911F910F9137
:10CB900008958FE090E090933F1180933E1188ECD0
:10CBA00090E00895FC018481958108956AE075E222
:10CBB000811102C06CE075E28BE09FE00D94571686
:10CBC00062EC70E28BE09FE00F945716F0E0E0E03B
:10CBD000199584EF91E008958091350B8823B1F089
:10CBE000E091360BF091370B309731F086819781C9
:10CBF0009093340B8093330B67E17EE18BE09FE0F1
:10CC00000F9457168BE09FE00D94EB14089560E0AD
:10CC10008DE00C9479BD61E08DE00C9479BD892B99
:10CC200071F0FB01828193810E94C8AF63EF74E2CF
:10CC30008BE09FE00F94571688EC90E0089590E009
:10CC400080E0F2CF0F931F93CF93DF93EB01029716
:10CC50000CF4A0C00A811B8160EF73E2C8010F943D
:10CC6000B33E892B61F40E942EB26F7E0E9488B27F
:10CC700088EC90E0DF91CF911F910F91089569EFBB
:10CC800073E2C8010F94B33E892B21F40E942EB2A7
:10CC90006061ECCF67EC73E28BE09FE00F94571676
:10CCA0000E942EB26295617081E0682770E04AE0D0
:10CCB00050E08BE09FE00F94F8158BE09FE00F941D
:10CCC000EB148091E70E9091E80E892B09F452C085
:10CCD0000A811B810E9449AF882309F44BC0F801E7
:10CCE00001900020E9F73197E01BF10BB09708F0B5
:10CCF00041C0A091E70EB091E80E52961C921E9290
:10CD0000519754961C921E92539784E890E01D967A
:10CD10009C938E931C971E961C921E9782E75596A5
:10CD20008C935597ED91FC9111970088F189E02D36
:10CD300060E270E0CD011995B8018091E70E909105
:10CD4000E80E0F9441168091E70E9091E80EDC01F9
:10CD5000ED91FC910190F081E02D60E019958091BA
:10CD6000E70E9091E80EDC01ED91FC910488F589C5
:10CD7000E02D19956A817B818BE09FE00F9441162D
:10CD800060EC73E28BE09FE00F9457168BE09FE01E
:10CD90000F94EB1480913E1190913F1102973CF05B
:10CDA00080EF9FEF90933F1180933E1161CF63EB33
:10CDB00073E285E19FE00F94571685E19FE00F94A1
:10CDC000EB1484EF91E056CFCF93DF93EB01029702
:10CDD000ACF160EF73E28A819B810F94B33E892BA3
:10CDE00029F40E942EB27E7F0E9488B269EF73E21E
:10CDF0008A819B810F94B33E892B29F40E942EB225
:10CE000071600E9488B26CE473E28BE09FE00F9443
:10CE100057160E942EB2672F609561704AE050E06D
:10CE200070E08BE09FE00F94F8158BE09FE00F948B
:10CE3000EB1488EC90E0DF91CF9108950E94353B90
:10CE4000F8CF892B71F0FB01828193810E9429B078
:10CE50006DE973E28BE09FE00F94571688EC90E049
:10CE6000089590E080E0F2CFEF92FF920F931F932E
:10CE7000CF93DF93CDB7DEB72C970FB6F894DEBF14
:10CE80000FBECDBF8C017B0183E695E09A83898339
:10CE90001B821C821D821E8298878F8319861A86A8
:10CEA0001B861C8605301105ECF0BE01695F7F4FC3
:10CEB000F701808591850E94D337892B99F0CE01A7
:10CEC00007960E94F3B0BE01695F7F4FF70186812C
:10CED00097810E94D337892B61F0CE0107960E947B
:10CEE000C5B10EC0CE0101960E94F3B00430110509
:10CEF00054F7CE0101960E94C5B103301105A4F18B
:10CF0000BE01695F7F4FF701848195810E94D3370D
:10CF1000892B51F1CE0107960E945CB1BE01695F79
:10CF20007F4FF701828193810E94D337892B19F1BA
:10CF3000CE0107960E948AB066E873E28BE09FE01C
:10CF40000F94571680E00E94ECB288EC90E02C968B
:10CF50000FB6F894DEBF0FBECDBFDF91CF911F910A
:10CF60000F91FF90EF900895CE0101960E945CB161
:10CF7000023011059CF6CE0101960E948AB0013064
:10CF80001105D1F6CE0101960E948AB06DE873E2D8
:10CF90008BE09FE00F945716CFCFCF93C1E068EEA0
:10CFA00073E080E090E00E94ECBF4AE050E06C2F1C
:10CFB0008BE09FE00F940E15CF5FC43181F784EFB3
:10CFC00091E0CF9108950F931F93CF93DF938C013E
:10CFD000EB010297C4F08A819B810F94653E809398
:10CFE000450299270E94F5B20230110549F08C8163
:10CFF0009D810F94653E8093440299270E94FFB261
:10D00000C8ECD0E002C0C0E9D1E062E773E28BE097
:10D010009FE00F9457164AE050E0609145028BE084
:10D020009FE00F940E156DE573E28BE09FE00F9487
:10D0300057164AE050E0609144028BE09FE00F9465
:10D040000E158BE09FE00F94EB14CE01DF91CF9192
:10D050001F910F910895009789F0FC0120852F7092
:10D06000253061F40E94A8AE009741F0FC012085B4
:10D070002F70243019F481859285089590E080E026
:10D0800008950F931F93CF93DF93CDB7DEB76997C2
:10D090000FB6F894DEBF0FBECDBFE0913511F09111
:10D0A0003611309709F460C080914211909143117C
:10D0B000892B09F459C08FEF838714861382148259
:10D0C00015821682178210861186128663EE70E230
:10D0D0008BE09FE00F9457168BE09FE00F94EB14CA
:10D0E000BE016E5E7F4F80913511909136110F9485
:10D0F0007A301816CCF5A895AE014F5F5F4F68E007
:10D10000CE0142960E945629198ABE016F5F7F4F59
:10D1100080914211909143110E94F6AD8C016EED09
:10D1200070E28BE09FE00F945716BE016F5F7F4F58
:10D130008BE09FE00F9441160115110591F0C80195
:10D140000E94303A8C01892B59F269ED70E28BE034
:10D150009FE00F945716B8018BE09FE00F944116A3
:10D16000BBCF64ED70E2B4CF88EC90E069960FB667
:10D17000F894DEBF0FBECDBFDF91CF911F910F910D
:10D180000895CF92DF92EF92FF920F931F93CF9368
:10D19000DF9300D000D0CDB7DEB78091590A81115E
:10D1A0009CC080913E1190913F1102970CF495C064
:10D1B0008091520A9091530A009709F48EC063E05F
:10D1C00078E00E94F6AD8C01009709F486C00E94B9
:10D1D00039AFE82EF12CE114F10409F47EC070E0BF
:10D1E00060E0C8010E942B686C01EA94EF2809F402
:10D1F00083C061E0C8010E94A8AEFC0101851285D0
:10D20000CE0101960E9419BBCE0101960E9437BB48
:10D2100066E979E18BE09FE00F945716B6018BE049
:10D220009FE00F94411664E377E08BE09FE00F945A
:10D2300041164AE050E0B8018BE09FE00F94F815EA
:10D2400064E377E08BE09FE00F94411669E57BE0B3
:10D250008BE09FE00F9441168BE09FE00F94EB145E
:10D2600062E072E08AED9FE00F94DB22D092D00F53
:10D27000C092CF0F1093D20F0093D10F89E59BE09E
:10D28000892BE9F581E098E09093D40F8093D30F38
:10D290008091330B9091340B009741F070E060E087
:10D2A0000E942B6890935B0A80935A0A80915A0AD5
:10D2B00090915B0A009731F19093D60F8093D50F30
:10D2C0001092D80F1092D70F81E08093590A6DE722
:10D2D00079E18BE09FE00F94571626960FB6F894ED
:10D2E000DEBF0FBECDBFDF91CF911F910F91FF9099
:10D2F000EF90DF90CF90089502E012E081CF89E5B2
:10D300009BE0C2CF80E594E0D7CFEF92FF920F93DE
:10D310001F93CF93DF9300D000D0CDB7DEB77C0151
:10D320008B0167EE75E18CEB9FE00F945716D701E8
:10D330001296ED91FC91608171818CEB9FE00F94CE
:10D3400041166EED75E18CEB9FE00F945716012EA0
:10D35000000C220B330B09831A832B833C8380E15F
:10D3600090E09E838D83BE016F5F7F4F8CEB9FE0CB
:10D370000E9450FE0F94EB1440E058E060E070E033
:10D38000C7010E943FE526960FB6F894DEBF0FBE98
:10D39000CDBFDF91CF911F910F91FF90EF90089536
:10D3A000CF92DF92EF92FF920F931F93CF93DF9371
:10D3B000CDB7DEB7C154D1090FB6F894DEBF0FBEAA
:10D3C000CDBF6C01AB0130E020E060E4CE010196FE
:10D3D0007C010E94E936F70101900020E9F73197BE
:10D3E0008F010E191F09A801B701C6010F94144B34
:10D3F000892B11F010E000E0C801CF5BDF4F0FB6C2
:10D40000F894DEBF0FBECDBFDF91CF911F910F917A
:10D41000FF90EF90DF90CF9008953F924F925F92F0
:10D420006F927F928F929F92AF92BF92CF92DF9234
:10D43000EF92FF920F931F93CF93DF93CDB7DEB799
:10D440002C970FB6F894DEBF0FBECDBF5C01362E11
:10D45000972E3A01690168E476E18CEB9FE00F9426
:10D4600057164AE050E0632D792D8CEB9FE00F9426
:10D47000F81560E476E18CEB9FE00F945716C3013A
:10D48000B0E0A0E08F839887A987BA8730E1432E68
:10D49000512C5C864B86BE01695F7F4F8CEB9FE011
:10D4A0000E9450FE4C016CE376E10F9457164AE05F
:10D4B00050E0B601C4010F94F81564E376E1C401AD
:10D4C0000F945716C701B0E0A0E089839A83AB831D
:10D4D000BC835E824D82BE016F5F7F4FC4010E949C
:10D4E00050FE0F94EB148091570A9091580A70E007
:10D4F00060E0892B09F047C081E090E09093580AE2
:10D500008093570A26E040E855E260E070E08DE540
:10D510009CE00F94A41730925D0D8DE59CE09093F4
:10D520005C0D80935B0D10926B0E10926D0E10923D
:10D530006C0E0130110509F44EC00CF041C0012BF6
:10D5400009F44EC0C114D10409F457C082E0C816D2
:10D55000D10409F062C07092E60D6092E50D109260
:10D56000E80D1092E70DF092EA0DE092E90D86E0E9
:10D570000E9404C31092580A1092570A882309F493
:10D5800056C0682F70E0C5010E94856990E080E078
:10D590002C960FB6F894DEBF0FBECDBFDF91CF91B2
:10D5A0001F910F91FF90EF90DF90CF90BF90AF90C1
:10D5B0009F908F907F906F905F904F903F900895D5
:10D5C0000330110581F00430110509F0BBCFFE24B2
:10D5D000EF24FE24B7CFFE2CEE24EE24EA94B2CF43
:10D5E000FF24FA94AFCFEF2821F492E0E92EF12C3A
:10D5F000EECFEE24E394F12CEACF7092E60D609228
:10D60000E50D90E080E0EE2011F080E09FEF909338
:10D61000E80D8093E70D85E0ABCF68E176E18CEB18
:10D620009FE00F9457161092580A1092570A81E003
:10D6300090E0AECF8F929F92AF92BF92CF92DF9247
:10D64000EF92FF920F931F93CF93DF93CDB7DEB787
:10D650002E970FB6F894DEBF0FBECDBF20913C11C0
:10D6600030913D11232B09F4BAC020913B112111B7
:10D67000B6C04C0180913B118F5F80933B1180912C
:10D680003A118F5F80933A110E94DEC19B01AC0179
:10D6900060913D0B70913E0B80913F0B9091400B40
:10D6A000A12CB12C65011BE0E12EF12C00E010E073
:10D6B0000E94F428882309F488C0F12C83E088169E
:10D6C0009104A1F00E94DEC19B01AC016091390B75
:10D6D00070913A0B80913B0B90913C0B14E6E12E3C
:10D6E000F12C00E010E00E94F428F82EE0913C11AB
:10D6F000F0913D11068117810115110509F447C00C
:10D70000F80180858F708630F1F51987088770E001
:10D7100060E0CE0108960F94CC09B401CE010896C2
:10D720000F943205FF2031F064E070E0CE010896DE
:10D730000F9432056AEA76E0C8010E94F6AD0097C0
:10D7400011F1FC0120852F702530E9F4C680D780C7
:10D75000C114D104C1F0DA82C982B801CE010196A8
:10D760000F94CC09B401CE0101960F943205FF202D
:10D7700031F064E070E0CE0101960F943205F601BD
:10D78000C280D380E5CFF80102811381B5CFF3E0E9
:10D790008F16910451F00E94DEC160933D0B70938F
:10D7A0003E0B80933F0B9093400BFF2051F00E9463
:10D7B000DEC16093390B70933A0B80933B0B9093CF
:10D7C0003C0B1092FB0F1092FC0F80913A1181508C
:10D7D00080933A1180913B11815080933B112E969A
:10D7E0000FB6F894DEBF0FBECDBFDF91CF911F9172
:10D7F0000F91FF90EF90DF90CF90BF90AF909F90F0
:10D800008F900895A89582E090E00C941A6B809117
:10D8100039118F5F80933911A89583E090E00E94C1
:10D820001A6B0F94A41A8091391181508093391189
:10D83000089565E278E28BE09FE00F94571662E16D
:10D8400078E28BE09FE00F94571664E078E28BE07B
:10D850009FE00F9457166CEF77E28BE09FE00F94F8
:10D8600057168BE09FE00F94EB146CEE77E28BE0A1
:10D870009FE00F94571660EE77E28BE09FE00F94E5
:10D88000571663ED77E28BE09FE00F9457166EEB2F
:10D8900077E28BE09FE00F9457166FEA77E28BE018
:10D8A0009FE00F94571667EA77E28BE09FE00F94B2
:10D8B000571666E977E28BE09FE00F94571660E712
:10D8C00077E28BE09FE00F94571663E677E28BE0F8
:10D8D0009FE00F94571669E577E28BE09FE00F9485
:10D8E00057166AE477E28BE09FE00F94571662E4E4
:10D8F00077E28BE09FE00F94571666E377E28BE0C8
:10D900009FE00F9457166CE177E28BE09FE00F9455
:10D9100057166DEF76E28BE09FE00F94571668EE96
:10D9200076E28BE09FE00F94571660ED76E28BE095
:10D930009FE00F94571662EC76E28BE09FE00F9425
:10D94000571666EB76E28BE09FE00F9457166EEA6F
:10D9500076E28BE09FE00F94571663EA76E28BE065
:10D960009FE00F94571666E976E28BE09FE00F94F4
:10D9700057166EE876E28BE09FE00F94571663E847
:10D9800076E28BE09FE00F94571664E776E28BE037
:10D990009FE00F9457166BE676E28BE09FE00F94C2
:10D9A00057166DE576E28BE09FE00F9457166FE413
:10D9B00076E28BE09FE00F94571663E476E28BE00B
:10D9C0009FE00F9457166BE376E28BE09FE00F9495
:10D9D00057168BE09FE00D94EB140F931F93CF939A
:10D9E000DF9300D000D0CDB7DEB70E94196C6EE295
:10D9F0007EE18BE09FE00F945716CE0101960E94C6
:10DA000019BBCE0101960E947D3703E615E01A830B
:10DA100009838091080D9091090DA0910A0DB09194
:10DA20000B0D8B839C83AD83BE83CE0101960E9438
:10DA30007D371A8309831B821C821D821E8280E52A
:10DA400090E00E9416BB44E050E0BE016D5F7F4F46
:10DA500081E090E00F94911D0F94881ECE010196F5
:10DA60000E947D371A8309831B821C821D821E82BD
:10DA700080E590E00E9416BB44E050E0BE016D5F7F
:10DA80007F4F85E090E00F94911D0F94881ECE018A
:10DA900001960E947D3764E57EE18BE09FE00F9464
:10DAA000571688EC90E026960FB6F894DEBF0FBEAE
:10DAB000CDBFDF91CF911F910F910895CF92DF924B
:10DAC000EF92FF921F93CF93DF9300D000D0CDB79A
:10DAD000DEB768E779E18BE09FE00F9457168FEE91
:10DAE000E82E8EE0F82E10E090E1C92ED12CF7013F
:10DAF00081917F01803130F46CE776E08BE09FE02C
:10DB00000F944116153041F1F7013197808190E073
:10DB1000B0E0A0E089839A83AB83BC83DE82CD82B0
:10DB2000BE016F5F7F4F8BE09FE00E9450FE66E773
:10DB300079E10F9457161F5F1630C9F626960FB677
:10DB4000F894DEBF0FBECDBFDF91CF911F91FF9044
:10DB5000EF90DF90CF9008958091F40E90E0B0E0C8
:10DB6000A0E089839A83AB83BC83DE82CD82BE0131
:10DB70006F5F7F4F8BE09FE00E9450FE0F94EB148D
:10DB8000DACFEF92FF920F931F93CF93DF9300D0E2
:10DB900000D01F92CDB7DEB77B01CE0107969F93D1
:10DBA0008F9301979F938F9301979F938F930197E3
:10DBB0009F938F9301979F938F9301979F938F9339
:10DBC0008E010F5F1F4F1F930F938AE098E09F9382
:10DBD0008F93DB0113968C9113978F9312968C91F0
:10DBE0008F930F94A94B0FB6F894DEBF0FBECDBF35
:10DBF0000697ECF468EC74E285E19FE00F94571609
:10DC0000D70112966D917C9185E19FE00F944116AA
:10DC100080E991E027960FB6F894DEBF0FBECDBF26
:10DC2000DF91CF911F910F91FF90EF900895809118
:10DC3000E70E9091E80E892B09F449C00E9449AF84
:10DC4000882309F444C0A091E70EB091E80E5296E3
:10DC50001C921E92519754961C921E92539784E8E0
:10DC600090E01D969C938E931C971E961C921E9777
:10DC700082E755968C935597ED91FC91119700880A
:10DC8000F189E02D64E070E0CD0119958091E70EF7
:10DC90009091E80EDC01ED91FC910280F381E02D82
:10DCA00046E050E0B801199586E0F801AFEEBEE01D
:10DCB00001900D928A95E1F78091E70E9091E80E20
:10DCC000DC01ED91FC910488F589E02D19950E9405
:10DCD0005E6D6AED74E28BE09FE00F94571688EC5E
:10DCE00090E098CFCF92DF92FF920F931F93CF9344
:10DCF000DF93F12C6115710509F492C06A01EB0103
:10DD00008C01CB010E94A7E3F82E882309F488C078
:10DD1000D2FE0AC0D8018C918B3009F44DC008F0B6
:10DD20003EC08A3009F44DC0D0FE09C0F8016081C0
:10DD300086EF860F843018F0CE010E94BEE6D1FE39
:10DD40006FC0D80114964D915D916D917C9117979C
:10DD500011968C918F70873038F0893008F440C06C
:10DD60008A50823008F465C0CE010E9464E4EE81DE
:10DD7000FF81309709F454C080858F709EEF980F13
:10DD8000923010F081114CC0D80111968C91982FCF
:10DD90009295907F80858F70892B808741C08C30D1
:10DDA000B9F040E050E062E070E08D3009F0BCCFA7
:10DDB000CE010E943FE5B8CF40E050E061E070E066
:10DDC000F7CF40E050E061E070E0CE010E9416E540
:10DDD00040E050E062E070E0CE010E9416E5A4CF82
:10DDE000EE81FF813097E1F080858F709EEF980F74
:10DDF000923010F0811114C0418752876387748775
:10DE0000EE81FF818085807F83608087EE81FF8146
:10DE10008085982F907F8F708067903609F4BDCFF2
:10DE20008F2DDF91CF911F910F91FF90DF90CF90B9
:10DE30000895CE010E9464E4F3CFCF93DF9300D026
:10DE400000D01F921F92CDB7DEB7FC01628398E02D
:10DE5000DE01119601900D929A95E1F729813A81A0
:10DE60004B815C816D817E818F81988528960FB66C
:10DE7000F894DEBF0FBECDBFDF91CF910895CF9351
:10DE8000DF9300D000D01F921F92CDB7DEB7FC0108
:10DE9000608398E0DE01119601900D929A95E1F76A
:10DEA00029813A814B815C816D817E818F8198854A
:10DEB00028960FB6F894DEBF0FBECDBFDF91CF918D
:10DEC0000895CF93DF9300D000D01F921F92CDB75B
:10DED000DEB7FC019181907F9B60918344835583E1
:10DEE0006683778388E0DE01119601900D928A9512
:10DEF000E1F729813A814B815C816D817E818F813F
:10DF0000988528960FB6F894DEBF0FBECDBFDF917F
:10DF1000CF910895CF93DF9300D000D01F921F922E
:10DF2000CDB7DEB7FC019181907F9A6091834483E5
:10DF300055836683778388E0DE01119601900D9208
:10DF40008A95E1F729813A814B815C816D817E81DF
:10DF50008F81988528960FB6F894DEBF0FBECDBF8F
:10DF6000DF91CF910895AF92BF92CF92DF92EF925F
:10DF7000FF920F931F93CF93DF9300D000D01F9297
:10DF80001F92CDB7DEB76115710509F45FC05A0164
:10DF90006B017C01CB010E94A7E3082F882369F164
:10DFA000D60116968D919C91009709F443C0FC010F
:10DFB0001085212F2F703EEF320F323010F02111DB
:10DFC0002EC012951F70B0FE59C0C6010E94DDE63A
:10DFD000F7018083112381F18181807F182B1183C8
:10DFE000D6011696ED91FC9181859285A385B48525
:10DFF000F70184839583A683B783802F28960FB675
:10E00000F894DEBF0FBECDBFDF91CF911F910F916E
:10E01000FF90EF90DF90CF90BF90AF9008952530A4
:10E0200049F460E00E94A8AE009721F0DC01189648
:10E030001C91C7CF10E0C7CFD6011696ED91FC9189
:10E0400080858F70823021F0833051F000E0D5CF91
:10E050004185528563857485C7010E948A6FCDCF43
:10E060004185528563857485F7018181807F876052
:10E0700081834483558366837783BFCF1123E1F285
:10E08000F701AACFCF93DF9300D000D01F921F9249
:10E09000CDB7DEB7FC016F3F710519F014F06FEFDB
:10E0A00070E077FD60E09181892F8F708150823020
:10E0B000C8F4648388E0DE01119601900D928A9580
:10E0C000E1F729813A814B815C816D817E818F816D
:10E0D000988528960FB6F894DEBF0FBECDBFDF91AE
:10E0E000CF910895907F91609183E3CFCF92DF929B
:10E0F000EF92FF92DC01362F1196EC911197EF70A1
:10E10000EC3008F0B6C0F0E08827E657FF488F4FA4
:10E110000D9487463C71C270C27039713971397182
:10E120000771C970397139719670967014968D9116
:10E130009D910D90BC91A02D662399F0B7FD9FC0D5
:10E140008F3F9105A105B10529F024F08FEF90E0F4
:10E15000A0E0B0E02FEF30E0A901481B590BCA0145
:10E160000CC0B7FD89C08F3F9105A105B10529F00D
:10E1700024F08FEF90E0A0E0B0E0FF90EF90DF9010
:10E18000CF90089514962C91822F90E06623A9F3E6
:10E19000E1CF1496CD90DD90ED90FC90179766231B
:10E1A00001F120E030E0A901C701B6010F94C64497
:10E1B00087FD65C020E030E04FE753E4C701B601BA
:10E1C0000F94CE4718160CF457C0A701960160E0D3
:10E1D00070E08FE793E40F94B9460F949847CB0112
:10E1E000CCCF20E030E0A901C701B6010F94C644AE
:10E1F00087FD42C020E030E04FE753E4C701B6019D
:10E200000F94CE471816DCF1C701B601E6CF14967D
:10E210006D917D918D919C9117973323B1F06D395C
:10E220005FEF75078507950754F1611524E67207BE
:10E23000810591050CF52CE93FEF4FEF5FEF0F944F
:10E240003246C90181509F4F98CF6D394FEF740707
:10E25000840794078CF0611554E6750781059105D4
:10E2600074F424E630E040E050E00F943246C901F7
:10E2700084CF8FEF9FEF81CF90E080E07ECF8FEF54
:10E2800090E07BCFCF93DF93EC01DB0189818F702E
:10E290008630E1F128F481508230C8F080E014C06B
:10E2A000873009F18A508230C8F72FEF30E00F94A1
:10E2B0009E4624E630E040E050E00F9432462C8346
:10E2C0003D834E835F8381E0DF91CF9108952FEFEF
:10E2D00030E00F949E4624E630E040E050E00F949A
:10E2E00032462C83F0CF2FEF30E00F949E4624E689
:10E2F00030E040E050E00F943246CA01B9010F947B
:10E30000CD446C837D838E839F83DDCF2CE933E600
:10E310000F949E4624E630E040E050E00F943246F1
:10E320002C833D834E835F83B9CFDC011196EC9142
:10E330001197EF70E150EB3008F039C0F0E088271A
:10E34000EB55FE488F4F0D948746C871C871D77141
:10E35000B071B071B971D071D071D071B071B0714C
:10E3600014966D917D918D919C9117970F94CD444A
:10E37000089514966D917D918D919C91179724E647
:10E3800030E040E050E00F943246CA01B901EECFD0
:10E3900014966C9170E090E080E00F94CB44089567
:10E3A00014966D917D918D919C911797089560E0E1
:10E3B00070E0CB010895DC011196EC911197EF709C
:10E3C000E150EB3008F037C0F0E08827E551FE4817
:10E3D0008F4F0D948746FD71FD711B72F671F671BA
:10E3E0000C72037203720372F671F67114966D91DA
:10E3F0007D918D919C911797089514966C9170E082
:10E4000090E080E0089514966D917D918D919C919E
:10E4100017970F949847089514966D917D918D915B
:10E420009C91179724E630E040E050E00F9432468C
:10E43000CA01B901089560E070E0CB010895DC01E4
:10E440001196EC911197EF70E150EB3008F03EC05F
:10E45000F0E08827E15DFD488F4F0D9487464572B7
:10E46000457266723A723A725F72507250725072AE
:10E470003A723A7214962D913D914D915C91179795
:10E48000A4E6B0E00F945146089514966C9184E68A
:10E49000689FB0011124072E000C880B990B08957A
:10E4A00020E030E048EC52E414966D917D918D911E
:10E4B0009C9117970F942C450F94984708951496A4
:10E4C0006D917D918D919C911797089560E070E01A
:10E4D000CB010895FC01A7812A2F2E7FC9F08181ED
:10E4E0008F7081508330A0F4A695A150BB0B2BE513
:10E4F00031E00F949E4624E630E040E050E00F9477
:10E500003246DA01C90187569F4FAF4FBF4F08957A
:10E510008FEF9FEF08952F923F924F925F926F92ED
:10E520007F928F929F92AF92BF92CF92DF92EF92A3
:10E53000FF920F93CF93DF9300D01F92CDB7DEB73A
:10E540007C017A8369835C834B83DB011C92FC0131
:10E550006081662309F44BC030FF49C0F9E06F9F2A
:10E56000B00111246854784ECD010F94083FD701B3
:10E5700011968C918F7041F04B815C8165E676E05D
:10E5800089819A810F94044BE981FA8101900020DE
:10E59000E9F7319729813A81E21BF30B19012E0E1D
:10E5A0003F1E4B815C814E1B5F0B415051095C83C8
:10E5B0004B83D7011196EC911197EF7009F4F5C0D8
:10E5C000E150EC3008F0F1C0F0E08827E551FD485B
:10E5D0008F4F0D948746FA729D730A746974847420
:10E5E00048731A741A741A7436731E73A0742980CF
:10E5F0003A80DFCFF7018481282F30E050E040E0FF
:10E60000002359F030E0A4E6B0E00F9464462FEF09
:10E6100030E040E050E00F9432465F934F933F93D9
:10E620002F938EE198E09F938F93FC81FF932B8132
:10E630002F933F922F920F943C4BB2C017968C9120
:10E6400017978F9316968C9116978F9315968C919A
:10E6500015978F9314968C918F9381E298E09F93F6
:10E660008F93BC81BF93EB81EF93E3CF17968C918F
:10E6700017978F9316968C9116978F9315968C916A
:10E6800015978F9314968C918F9385E298E0E7CF3E
:10E690001496CD90DD90ED90FC901797F7FE34C066
:10E6A00084E6882E912CA12CB12CC701B601A501BE
:10E6B00094010F9432469B01AC0188279927DC0115
:10E6C000821B930BA40BB50BBF93AF939F938F93B8
:10E6D00066277727CB016C197D098E099F09A50153
:10E6E00094010F9432465F934F933F932F9389E2A7
:10E6F00098E09F938F933C813F934B814F933F9240
:10E700002F920F943C4B4CC0C701B60124E630E079
:10E7100040E050E00F9432469F938F937F936F9326
:10E720005F934F933F932F938AE298E09F938F9349
:10E730009C819F93AB81AF93E2CFC7010E946A7225
:10E74000BC01D7011696CC9016971796DC901797B8
:10E75000D0FADD24D0F814969C9114971596FC906D
:10E76000EB80BC80292F30E050E040E077FD35C0E1
:10E77000011135C07F936F931F921F921F929F9339
:10E780001F92FF92DF92CF9283E398E09F938F9343
:10E79000FC81FF932B812F933F922F920F943C4B40
:10E7A0000FB6F894DEBF0FBECDBF89819A810F905E
:10E7B0000F900F900F90DF91CF910F91FF90EF90FE
:10E7C000DF90CF90BF90AF909F908F907F906F9091
:10E7D0005F904F903F902F900895002361F0292F74
:10E7E00030E0A4E6B0E00F9464462FEF30E040E064
:10E7F00050E00F9432465F934F933F932F931F92B5
:10E80000FF92DF92CF9286E398E09F938F93BF921F
:10E81000EF9275CF15968C9115971F928F93169640
:10E820009C91169717968C9181708F939F9389E393
:10E8300098E015CF14968D909D90AD90BC90179751
:10E8400020E030E0A901C501B4010F94C6442401C1
:10E85000350187FF04C077FA709477F87094C3018C
:10E86000B2010F9498476B01072E000C880B990B8F
:10E870000F94CD449B01AC01C301B2010F94B94682
:10E8800020E030E04AE754E40F942C450F942348ED
:10E890000F949847062F772E20E030E0A901C5019C
:10E8A000B4010F94C64487FF07C07F920F93DF9295
:10E8B000CF928FE398E0D3CE7F920F93DF92CF92E7
:10E8C00080E498E09F938F933C813F934B814F93DB
:10E8D000B0CE14968C9114971F928F9315968C91AD
:10E8E00015971F928F9316968C911F928F9386E3A4
:10E8F00098E09F938F93BC81BF93EB81EF933F92FE
:10E900002F920F943C4B4CCF17968C9117971F92D8
:10E910008F9314968C9114971F928F9315968C91C8
:10E9200015971F928F9316968C911F928F9383E366
:10E9300098E09F938F93BC81BF93EB81EF93DFCEE1
:10E9400014966D917C914B815C81C1010F94224B97
:10E950002CCFEF92FF920F93CF93DF93CDB7DEB71B
:10E96000A0970FB6F894DEBF0FBECDBF7C0100E0CC
:10E9700020E033E040E250E0BE016F5F7F4F0E9435
:10E980008B72BE016F5F7F4F8CEB9FE00F9441163F
:10E9900060EA78E18CEB9FE00F945716F7016181F4
:10E9A0006F704AE050E08CEB9FE00F940E1569E920
:10E9B00078E18CEB9FE00F9457164AE050E0F701A6
:10E9C00062818CEB9FE00F940E158CEB9FE00F940F
:10E9D000EB14A0960FB6F894DEBF0FBECDBFDF914B
:10E9E000CF910F91FF90EF900895CF93DF93EC01BB
:10E9F0006115710539F48F8181708F8381E0DF911A
:10EA0000CF9108958981982F9F7029F180E09430EB
:10EA1000B0F79B01770F440B550B29593109410978
:10EA20005109A4E6B0E00F9451462BE531E040E0F7
:10EA300050E00F94324637FF02C030E020E0253628
:10EA4000310514F024E630E02F5F220F8F818170B2
:10EA5000282B2F83D3CF807F82608983DACFFC017C
:10EA60009181892F8F7021F0823029F080E0089504
:10EA7000907F926091839B0177FF02C030E020E09D
:10EA80002E3681E0380714F02DE631E026838781A9
:10EA900030FB80F9878381E00895EF92FF920F9316
:10EAA0001F93CF93DF93FC01892B69F19081992308
:10EAB00051F19D3291F180ED890F8A3070F1C8E0FB
:10EAC000D0E0953211F1CEEFDFEF9B37F1F0C7E1E7
:10EAD000D0E09332D1F08F0181ECE82E87E1F82E5F
:10EAE000C1E0D0E0C7010F94E13EAC01B701C8011D
:10EAF0000F94FA3E892B49F0219689E0E80EF11C2B
:10EB0000C931D10579F7CFEFDFEFCE01DF91CF919A
:10EB10001F910F91FF90EF900895D0E0C0E0F5CFE6
:10EB2000EF92FF920F931F93CF93DF93EC01892B0A
:10EB300051F188858F70843009F5E984FA84C70122
:10EB40000E944D758C0118161906ECF4C7010F943C
:10EB5000F81AC801012E000CAA0BBB0B89879A87F3
:10EB6000AB87BC878885807F82608887C801DF91FA
:10EB7000CF911F910F91FF90EF900895823019F47B
:10EB800009851A85F3CF10E000E0F0CF2F923F9275
:10EB90004F925F926F927F928F929F92AF92BF92AD
:10EBA000CF92DF92EF92FF920F931F93CF93DF9359
:10EBB000CDB7DEB7A0970FB6F894DEBF0FBECDBFBE
:10EBC0006115710549F528E0FC01DE0111960190FF
:10EBD0000D922A95E1F729813A814B815C816D8103
:10EBE0007E818F819885A0960FB6F894DEBF0FBE08
:10EBF000CDBFDF91CF911F910F91FF90EF90DF90EC
:10EC0000CF90BF90AF909F908F907F906F905F90CC
:10EC10004F903F902F9008956B018C0164E876E04F
:10EC2000C6010E94F6ADFC01892B09F40EC1808556
:10EC30008F70843009F452C0853009F006C1E68037
:10EC4000F780E114F10409F400C1F70180858F70A9
:10EC5000823011F4E280F380E114F10409F4F5C08C
:10EC6000F70180858F70853011F0F701F3CFC70170
:10EC70000E9439AF8230C9F760E0C7010E94A8AE98
:10EC80005C010E94907561E0C7010E94A8AE4C0132
:10EC9000FC0180858F70823041F7C8010E94DB71D2
:10ECA000F401418452846384748464157505860577
:10ECB0009705D9F6A114B10409F4C7C019821A82C4
:10ECC0001B821C821D821E821F8218868A81807F81
:10ECD0008A83F5016185CE0101964EC069E876E030
:10ECE000818592850F94F44A892B09F0AEC0C80142
:10ECF0000E94DB71611571058105910509F48BC0D6
:10ED0000660F771F881F991F2FEF30E040E050E01B
:10ED10000F94324657FD15C023303105410551058A
:10ED20000CF05FC0DA01C9010196A11DB11D82304E
:10ED30009105A105B105D9F10397A105B10509F424
:10ED400050C019821A821B821C821D821E821F8261
:10ED500018868A81807F8A8367E0CE0101960E94AF
:10ED60001D6F29873A874B875C876D877E878F87E2
:10ED7000988B62E1CE0109960E943F6F298B3A8BF6
:10ED80004B8B5C8B6D8B7E8B8F8B988F49895A89CF
:10ED90006B897C898D899E89AF89B88D49835A8317
:10EDA0006B837C838D839E83AF83B88714CF198256
:10EDB0001A821B821C821D821E821F8218868A81F3
:10EDC000807F8A8367E0CE0101960E941D6F2987AC
:10EDD0003A874B875C876D877E878F87988B61E149
:10EDE000C9CF19821A821B821C821D821E821F8239
:10EDF00018868A81807F8A8367E0CE0101960E940F
:10EE00001D6F29873A874B875C876D877E878F8741
:10EE1000988B60E1AFCF19821A821B821C821D82FF
:10EE20001E821F8218868A81807F8A8367E0CE01D6
:10EE300001960E941D6F29873A874B875C876D87F3
:10EE40007E878F87988B62E095CF68E478E0C60173
:10EE50000E94F6AD7C01009709F4D1C0FC018085C9
:10EE60008F70853009F0BAC0C7010E9439AF843075
:10EE700009F0C5C060E0C7010E94A8AE5C0161E076
:10EE8000C7010E94A8AE6C0162E0C7010E94A8AE53
:10EE9000FC012185328543855485298F3A8F4B8F1C
:10EEA0005C8F63E0C7010E94A8AE7C01C8010E948C
:10EEB000DB71298D3A8D4B8D5C8D6217730784074A
:10EEC00095079CF419821A821B821C821D821E8265
:10EED0001F8218868A81807F8A8340E050E0BA01D1
:10EEE000CE0101960E94616F49CFF5010184F28540
:10EEF000E02DFE8FED8FF60121843284F70101842D
:10EF0000F285E02DF8A3EF8F19821A821B821C82F2
:10EF10001D821E821F8218868A81807F8A836101FA
:10EF2000032C000CEE08FF082D8D3E8D4901330F98
:10EF3000AA08BB08498D5A8D2A01550F6608770823
:10EF4000C8010E94DB719B01AC01241935094609F7
:10EF50005709C701B601681979098A099B090F94F5
:10EF60000046EF8DF8A19F01FF0F440B550B2419AC
:10EF70003509460957090F943246820E931EA41E86
:10EF8000B51EC1012D8D3E8D821B930B6F8D78A117
:10EF9000498D5A8D641B750B0F94734677FF02C021
:10EFA0006F5F7F4F75956795CB01770FAA0BBB0BF2
:10EFB000880E991EAA1EBB1EB7FC0BC0A601B70186
:10EFC000C814D904EA04FB040CF48ACFA401B501E7
:10EFD00087CF40E050E060E070E082CF81110FC049
:10EFE00019821A821B821C828A81807F8A834981CE
:10EFF0005A816B817C8180E090E0DC01CFCEF8010A
:10F00000408151816281738184819581A681B7811C
:10F01000C5CE4F925F926F927F928F929F92AF92E6
:10F02000BF92CF92DF92EF92FF920F931F93CF93F5
:10F03000DF93CDB7DEB760970FB6F894DEBF0FBE93
:10F04000CDBF6115710539F528E0FC01DE0111968F
:10F0500001900D922A95E1F729813A814B815C81DB
:10F060006D817E818F81988560960FB6F894DEBFA2
:10F070000FBECDBFDF91CF911F910F91FF90EF9009
:10F08000DF90CF90BF90AF909F908F907F906F90C8
:10F090005F904F9008956B018C0164E876E0C601A3
:10F0A0000E94F6AD5C01F801F080FF2009F456C023
:10F0B000009709F453C0FC0180858F70843009F4F7
:10F0C000C7C0853009F04AC080914502893020F4DC
:10F0D00080914402893050F06CE478E08CEB9FE042
:10F0E0000F9441168CEB9FE00F94EB14F501E68032
:10F0F000F780E114F10491F1F70180858F705701D9
:10F10000823061F0B12CA12CE114F10409F41DC18D
:10F11000F70180858F70853021F0F701E280F38060
:10F12000F3CFC7010E9439AF8230B9F760E0C70161
:10F130000E94A8AE0E9490754C0161E0C7010E9438
:10F14000A8AEF80120812815190439F7FC012085A3
:10F150002F70223011F7009709F001C168E478E0C0
:10F16000C6010E94F6AD7C01F80181818F7009F41F
:10F1700007C1E114F10409F47DC0F70180858F70A7
:10F18000853009F001C1C7010E9439AF843009F010
:10F19000FBC0C8010E94DB714B015C0160E0C7014C
:10F1A0000E94A8AEFC0181859285A385B485198251
:10F1B0001A821B821C821D821E821F82188688165C
:10F1C0009906AA06BB060CF499C08A81807F8A83BF
:10F1D00063E0C7010E94A8AE5C0162E0C7010E9423
:10F1E000A8AEFC01418452846384748461E0C70149
:10F1F0000E94A8AE4C0160E0C7010E94A8AEFC01CD
:10F20000C184D284E384F484C8010E94DB71F501D7
:10F2100021853285438554852419350946095709C6
:10F220006C197D098E099F090F940046F401218510
:10F230003285438554852C193D094E095F090F9489
:10F240003246BA01A901440D551D661D771D31C016
:10F2500069E876E0818592850F94F44A892B09F05C
:10F260007DCFF0E1FF1609F460C0FF1568F082E081
:10F27000F816E1F1F8014081518162817381848146
:10F280009581A681B78129C0E1E1FE16F1F1F2E195
:10F29000FF12F0CF19821A821B821C821D821E82ED
:10F2A0001F8218868A81807F8A8344E150E060E073
:10F2B00070E0CE0101960E94616F29873A874B87E3
:10F2C0005C876D877E878F87988B49855A856B858C
:10F2D0007C858D859E85AF85B88949835A836B83EC
:10F2E0007C838D839E83AF83B887B6CE19821A82C2
:10F2F0001B821C821D821E821F8218868A81807F4B
:10F300008A8340E050E0BA01D4CF19821A821B826E
:10F310001C821D821E821F8218868A81807F8A83BA
:10F3200040E850E060E070E0C4CF19821A821B828E
:10F330001C821D821E821F8218868A81807F8A839A
:10F340004FEF50E060E070E0B4CFA114B10409F4D5
:10F3500005CFF50180858F7009F400CFC5011982B2
:10F360001A821B821C821D821E821F8218862A819D
:10F37000207F2A83FC01418552856385748599CF5E
:10F38000E114F10409F476CFF70180858F7009F05C
:10F3900071CF19821A821B821C828A81807F8A83A4
:10F3A00049815A816B817C8180E090E0DC0195CFBE
:10F3B0008F929F92AF92BF92DF92EF92FF920F9344
:10F3C0001F93CF93DF93EC018A819B810E9439AF19
:10F3D000082F10E00430110554F40E94ECB3BC0176
:10F3E0008A819B810E94F9B30F5F1F4FF3CFEA819F
:10F3F000FB81068117810115110529F0F801828131
:10F4000093819D838C83EC81FD81309721F08281F3
:10F4100093819F838E83EE81FF81309749F0028034
:10F42000F381E02D309721F082819381998788873D
:10F430000115110549F0F80180858F70843009F4B9
:10F4400038C028F4823079F0DD24DA940DC085309C
:10F4500009F42CC08630C1F769EF75E0C8010E943D
:10F46000F6AD8C01E5CFD184DA86F4E1FD1508F420
:10F4700059C0ED2DF0E08827EF5BF5488F4F0D94D4
:10F4800087469E7A9E7A9E7A817A927A927A927A48
:10F49000927A927A927ABD7AAC7AEE7A117BFE7A7F
:10F4A000927A1C7B9E7A6B7B927A877B068117818E
:10F4B000BFCFA184B284A114B10409F4C5CFF50172
:10F4C0008081882309F4C0CF82E5882E86E1982EBA
:10F4D000F12CE12CDE2CC4010F94E13EAC01B4010F
:10F4E000C5010F94FA3E892B09F41FC1FFEFEF1AF3
:10F4F000FF0A89E0880E911CE7E1EE16F10451F74E
:10F50000A3CF8AE090E00F94983C8C01BE010E944A
:10F510002DFE88EA93E0F80191838083118610869E
:10F520001C870B87DF91CF911F910F91FF90EF9078
:10F53000DF90BF90AF909F908F90089588E090E00B
:10F540000F94983C8C01BE010E942DFE84E893E04C
:10F55000F80191838083E4CF8DE090E00F94983C94
:10F560008C01BE010E942DFE80E693E0F80191839C
:10F570008083C8010E94503AD3CF89E090E00F9475
:10F58000983C8C01FC01D383C2838EE393E091838A
:10F590008083CE010E94F7E3F8019583848380EC99
:10F5A0009BE090878783CE010E948EE4892B09F42B
:10F5B000B7CF70E060E0CE010E94EBE4F8018683F3
:10F5C000882331F0823009F0ABCF8DE59CE002C09A
:10F5D0008FE19FE0F80190878783A2CF8EE090E0D3
:10F5E0000F94983C8C01FC01D383C28382E394E0A6
:10F5F00091838083C8010E94843A92CF86E090E094
:10F600000F94983C8C01FC01D383C2838CE193E07E
:10F6100091838083CE010E94F7E3F8019583848370
:10F620007FCF86E090E00F94983C8C01FC01D3835F
:10F63000C2838AEF92E0ECCF8BE090E00F94983C8D
:10F640008C01FC01D383C28380E194E091838083A9
:10F65000168270E060E0CE010E94EBE497FD28C0C6
:10F66000F80195838483F80184819581009719F0CE
:10F67000863491052CF080E290E0F8019583848334
:10F6800061E070E0CE010E94A5E420E030E04AE7AE
:10F6900054E40F942C450F949F4761157105810523
:10F6A000910579F0F801678370878187928738CF59
:10F6B000919581959109F8019583848381E08683F2
:10F6C000D2CF88E893E1A0E0B0E0F801878390878B
:10F6D000A187B28725CF86E090E00F94983CFC018B
:10F6E000D383C2838EEE93E091838083158214824C
:10F6F000AC81BD81109741F018968C9118978F704E
:10F70000863011F4B583A483FC87EB870BCF84E0AC
:10F7100090E00F94983CFC01D383C2832CEC33E03F
:10F72000318320839C878B87FDCEC5010F94F81A07
:10F730008E2D90E0B0E0A0E0F80181879287A3874A
:10F74000B4878085807F826080878ECECF92DF9263
:10F75000EF92FF920F931F93CF93DF9300D000D0CF
:10F760001F921F92CDB7DEB77C0109831A832B83CA
:10F770003C834D835E836F837887CE0101960E9420
:10F78000B7AE8C018981882351F09B81923008F0BB
:10F79000BAC0823011F0853011F410E000E070E062
:10F7A00060E0C7010E94EBE4D82EC92E6BEF75E133
:10F7B0008CEB9FE00F9457164AE050E06D2D7C2DA6
:10F7C0008CEB9FE00F94F81569EF75E18CEB9FE0EF
:10F7D0000F9457164AE050E0B8018CEB9FE00F946D
:10F7E000F8158CEB9FE00F94EB148091570A9091E1
:10F7F000580A892BE9F040E053E0B701CE010196A9
:10F800000E94726E70E060E0C7010E94856990E01E
:10F8100080E028960FB6F894DEBF0FBECDBFDF9113
:10F82000CF911F910F91FF90EF90DF90CF900895AF
:10F8300081E090E09093580A8093570A26E040E8D0
:10F8400055E260E070E08DE59CE00F94A417D09243
:10F850005D0D8DE59CE090935C0D80935B0D1092A7
:10F860006B0E10926D0E10926C0E80ED97E09093DF
:10F87000E60D8093E50D1092E80D1092E70D01154D
:10F880001105E1F185E090E09093EA0D8093E90D98
:10F8900086E00E9404C3D82E64E670E080E090E029
:10F8A0000E94ECBFD1100AC062EF75E18CEB9FE0C3
:10F8B0000F9457168CEB9FE00F94EB1482ED97E0BA
:10F8C0009093E60D8093E50D1092E80D1092E70DF0
:10F8D00024E6209FC001219F900D11249093EA0DF2
:10F8E0008093E90D86E00E9404C31092580A10929A
:10F8F000570A882359F0682F70E086CF1092EA0DDE
:10F900001092E90DC5CF8FEF9FEF83CF81E090E09C
:10F9100080CF2F923F924F925F926F927F928F9201
:10F920009F92AF92BF92CF92DF92EF92FF920F938E
:10F930001F93CF93DF93CDB7DEB72C970FB6F89414
:10F94000DEBF0FBECDBF5C0109831A832B833C83CE
:10F950004D835E836F837887CE0101960E94B7AE98
:10F960001C01023011F0053011F4312C212CF5016D
:10F9700004811581F80180858F70853009F07FC082
:10F98000C8010E9439AFE82EF12CF2E0EF16F10425
:10F990000CF475C060E0C8010E94A8AEFC0181852E
:10F9A00092859C878B8761E0C8010E94A8AEFC010C
:10F9B000418452846384748488248A94982CF2E06D
:10F9C000EF16F10459F062E0C8010E94A8AEFC01F4
:10F9D00081849284F3E0EF16F104A1F48FE390E0C8
:10F9E0009A87898792E0C92ED12C29853A85D10141
:10F9F0000F94964624E630E040E050E00F94324603
:10FA000079011CC063E0C8010E94A8AEFC01818599
:10FA100092859A87898782E0C82ED12CF4E0EF1670
:10FA2000F10439F064E0C8010E94A8AEFC01C18471
:10FA3000D28489859A857101892BB9F68401960152
:10FA4000A2016B857C85C5010E940D6A2C960FB6BC
:10FA5000F894DEBF0FBECDBFDF91CF911F910F9104
:10FA6000FF90EF90DF90CF90BF90AF909F908F90DE
:10FA70007F906F905F904F903F902F90089590E00F
:10FA800080E0E4CFAF92BF92CF92DF92EF92FF92ED
:10FA90000F931F93CF93DF93CDB7DEB7CD56D10928
:10FAA0000FB6F894DEBF0FBECDBF5C01A7960FAFB7
:10FAB000A797A8961FAFA897A9962FAFA997AA9620
:10FAC0003FAFAA97AB964FAFAB97AC965FAFAC97F3
:10FAD000AD966FAFAD97AE967FAFAE9723961FAE44
:10FAE0001EAE2397FE01ED5BFF4F82E1DF011D9209
:10FAF0008A95E9F772961192119287E0DF011D92C3
:10FB00008A95E9F76AE578E08CEB9FE00F9441165F
:10FB1000B6018CEB9FE00F944116CE018A599F4F9E
:10FB20000E94A974F0FE2CC0A796EFADA797E8310C
:10FB300008F050C1F0E08827EF55F2488F4F0D9440
:10FB40008746F07EB97DE77EEA7EEA7EE77EB97D74
:10FB5000EA7EEA7EEA7EEA7EEA7EEA7EEA7EB97D97
:10FB6000B97DEA7EEA7EEA7EB97DB97DB97DEA7E1D
:10FB7000F07E66E075E1CE018B5A9F4F0F94DA3E1E
:10FB80000E9414AE882309F407C1809139118111B4
:10FB900003C1C114D10409F05EC030E020E043E0AD
:10FBA00050E060E4CE0101960E94E936D50112963C
:10FBB000ED91FC91608171814FE350E0CE0101969F
:10FBC0000F94044BF1FE0FC1A7968FADA79782301B
:10FBD00009F409C1853009F406C1A8968FADA8972C
:10FBE0008F709FE0980F9F70923018F0883009F066
:10FBF000FAC001E020E032E044E150E0BE016F5B7A
:10FC00007F4FCE018A599F4F0E948B72BE016F5B5E
:10FC10007F4FCE0101960E947BC26DED74E18CEBAB
:10FC20009FE00F945716BE016F5F7F4F8CEB9FE0F4
:10FC30000F9441166AED74E18CEB9FE00F94571618
:10FC4000BE016F5B7F4F8CEB9FE00F9441168CEBF6
:10FC50009FE00F94EB14A8968FADA8978F70870143
:10FC600000271072882311F0F1FC04C00115110562
:10FC700009F4F5C030E020E043E050E060E4CE015C
:10FC800001960E94E936D5011296ED91FC916081B2
:10FC900071814FE350E0CE0101960F94044BC114E3
:10FCA000D10469F067E279E0CE0101960F94DE4A53
:10FCB0004FE350E0B601CE0101960F94044B67E28A
:10FCC00079E0CE0101960F94DE4A4FE350E06FE9F0
:10FCD00074E10115110511F465E974E1CE01019695
:10FCE0000F94EA3EA8968FADA8978F70845082300B
:10FCF00008F09FC067E1CE018A599F4F0E943F6F75
:10FD00006F962FAF6F97A0963FAFA097A1964FAF7A
:10FD1000A197A2965FAFA297A3966FAFA397A49661
:10FD20007FAFA497A5968FAFA597A6969FAFA697EE
:10FD300000E020E033E044E150E0BE016F5B7F4F24
:10FD4000CE018A599F4F0E948B7265E874E18CEB5B
:10FD50009FE00F945716BE016F5F7F4F8CEB9FE0C3
:10FD60000F94411662E874E18CEB9FE00F945716F4
:10FD7000BE016F5B7F4F8CEB9FE00F9441168CEBC5
:10FD80009FE00F94EB140E9414AE882329F0809119
:10FD90003911882309F455C0A701FF0C660B770BB6
:10FDA000C5010E943FE590E080E0C359DF4F0FB6E8
:10FDB000F894DEBF0FBECDBFDF91CF911F910F91A1
:10FDC000FF90EF90DF90CF90BF90AF9008956FE0DD
:10FDD00075E1D1CE63EE74E18CEB9FE00F94571682
:10FDE000E894F0F8CDCEF0FE36CF66968FAD6697EC
:10FDF000882309F430CFBE016B5A7F4FCE010196A4
:10FE00000E947BC264ED74E18CEB9FE00F94571667
:10FE1000BE016F5F7F4F8CEB9FE00F94411661ED49
:10FE200074E18CEB9FE00F945716BE016B5A7F4F25
:10FE30000ACF20E032E0012B11F020E033E000E0B7
:10FE40007ACFBE016F5B7F4FCE0101960E947BC2CD
:10FE500040E052E060E070E0C5010E9416E5F0FE6F
:10FE600091C0A796EFADA797E150E53118F5F0E006
:10FE70008827E25CF0488F4F0D9487464B805A7F6D
:10FE80005A7F5A7F5A7F4B805A7F5A7F5A7F5A7FB8
:10FE90005A7F5A7F5A7F508048805A7F5A7F5A7FB4
:10FEA000537F4280458068EA75E1CE018B5A9F4FAF
:10FEB0000F94DA3E30E020E043E050E060E4CE0111
:10FEC00001960E94E936D5011296ED91FC91608170
:10FED00071814FE350E0CE0101960F94044BC114A1
:10FEE000D10469F067E279E0CE0101960F94DE4A11
:10FEF0004FE350E0B601CE0101960F94044B67E248
:10FF000079E0CE0101960F94DE4A4FE350E060E9BC
:10FF100074E1CE0101960F94EA3E6CE774E18CEB3C
:10FF20009FE00F945716BE016F5F7F4F8CEB9FE0F1
:10FF30000F94411669E774E18CEB9FE00F9457161C
:10FF4000BE016B5A7F4F8CEB9FE00F9441168CEBF8
:10FF50009FE00F94EB140E9414AE882309F41CCF89
:10FF600080913911811118CFBE016B5A7F4FCE019C
:10FF700001960E947BC240E051E060E070E0C50164
:10FF80000E9416E5F2FE7BC040E050E061E070E0C8
:10FF9000C5010E9468E5672B682B692B09F483C0B3
:10FFA00060E675E1CE018B5A9F4F0F94DA3E30E048
:10FFB00020E043E050E060E4CE0101960E94E93683
:10FFC000D5011296ED91FC91608171814FE350E073
:10FFD000CE0101960F94044BC114D10469F067E27D
:10FFE00079E0CE0101960F94DE4A4FE350E0B6016E
:10FFF000CE0101960F94044B67E279E0CE010196A1
:020000021000EC
:100000000F94DE4A4FE350E068EB74E1CE010196B5
:100010000F94EA3E63E774E18CEB9FE00F94571670
:10002000BE016F5F7F4F8CEB9FE00F94411660E73E
:1000300074E18CEB9FE00F945716BE016B5A7F4F13
:100040008CEB9FE00F9441168CEB9FE00F94EB1428
:100050000E9414AE882309F49FCE8091391181113A
:100060009BCEBE016B5A7F4FCE0101960E947BC290
:1000700040E054E060E070E0C5010E9416E581E0D8
:1000800090E093CE61EB75E110CF6AEB75E10DCF97
:1000900064E875E10ACFF5018285853009F00ACF61
:1000A0006BE775E102CF40E050E062E070E0C5012F
:1000B0000E9468E5672B682B692B19F062E775E1F0
:1000C00071CF67E575E16ECFAF92BF92CF92DF92AD
:1000D000EF92FF920F931F93CF93DF9300D000D046
:1000E0001F921F92CDB7DEB75C017B0160FF03C09A
:1000F000E894E0F8F4F8F4FC0DC00E946A38663920
:1001000071058105910530F080913E1190913F116C
:10011000059719F5A70144275770052E000C660BAB
:10012000770BC5010E943FE56FE574E18CEB9FE022
:100130000F9457168FEF9FEF28960FB6F894DEBFF7
:100140000FBECDBFDF91CF911F910F91FF90EF9028
:10015000DF90CF90BF90AF90089519821A821B82D2
:100160001C821D821E821F8218868A81807F8A835C
:1001700040E053E0B501CE0101960E94B36F40E02C
:1001800057E060E070E0C5010E9468E5E62AF72AC2
:10019000D12CC12C09811A812B813C814D815E813A
:1001A0006F817885C5010E94427DC6CF8F929F9254
:1001B000AF92BF92CF92DF92EF92FF920F931F9375
:1001C000CF93DF93CDB7DEB760970FB6F894DEBF5D
:1001D0000FBECDBF8C017B0140E058E060E070E0D5
:1001E0000E9468E5672B682B692B09F0A9C062E0C3
:1001F00070E0C8010E94EBE46C0119861A861B8628
:100200001C861D861E861F86188A8A85807F8A879F
:10021000D7FC96C040E052E0B801CE0109960E949A
:10022000B36F63E070E0C8010E94EBE4AC01181604
:10023000190614F04FE350E081E0C816D10429F408
:10024000EF2CFF0CFF08FF2404C082E0C816D10485
:10025000D4F32FEF30E0D7010F949E469A01550F4B
:10026000440B550B0F94324649016901C8010E94A5
:10027000DDE6E82EF12C60E0CE0109960E94767052
:1002800088169906F9F4CD2841F082E0E816F104C9
:1002900019F185E0E816F104F9F081E090E060964C
:1002A0000FB6F894DEBF0FBECDBFDF91CF911F9187
:1002B0000F91FF90EF90DF90CF90BF90AF909F9005
:1002C0008F900895CD2859F186E0E816F10441F0A9
:1002D00081E0E816F10421F061E0C8010E94BEE669
:1002E000B401CE0109960E94427040E052E0B8018C
:1002F000CE0109960E94726E82E0E816F10421F0A8
:1003000085E0E816F10429F460E071E0C8010E947C
:10031000648060E072E0C8010E946480BECF85E026
:10032000E816F10409F4B9CF82E0E816F10409F403
:10033000B4CF62E0C8010E94BEE660E071E0EBCF9E
:1003400090E080E0ACCFCF93DF93EC0140E053E04E
:1003500060E070E00E9468E5611571058105910516
:1003600099F020913E1130913F112630310561F412
:10037000CE010E94648040E053E060E070E0CE0176
:10038000DF91CF910C9416E5DF91CF910895FF9204
:100390000F931F93CF93DF9300D000D0CDB7DEB77C
:1003A0008C01BC01CE0101960F947812BE016F5FE3
:1003B0007F4F8CEB9FE00F9449168CEB9FE00F94DE
:1003C000EB14CE0101960F9470121A8219821C82CE
:1003D0001B821E821D826EE075E2CE0101960F9493
:1003E0001312F801248135818D819E81F12C28170B
:1003F000390738F0BE016F5F7F4FC8010E9479BC9A
:10040000F82ECE0101960F947012FF2069F0B8010A
:10041000CE0101960F947812CE0101960E941BCA5C
:10042000CE0101960F94701226960FB6F894DEBF97
:100430000FBECDBFDF91CF911F910F91FF90089517
:100440000F931F93CF93DF9300D000D0CDB7DEB7CB
:10045000A091E70EB091E80E109709F478C052967B
:100460001C921E92519754961C921E92539784E8A8
:1004700090E01D969C938E931C971E961C921E973F
:1004800087E755968C935597ED91FC9111970088CD
:10049000F189E02D70E060E0CD01199510E000E0F9
:1004A0008091E70E9091E80EDC01ED91FC9111979F
:1004B0001C962D913C910217130740F40190F08196
:1004C000E02D60E019950F5F1F4FEACF0088F1899A
:1004D000E02D70E060E0199502EB14E08091E70EEA
:1004E0009091E80EF80161918F01DC01ED91FC9192
:1004F0000190F081E02D1995B4E0063B1B0771F7E0
:100500008091E70E9091E80EDC01ED91FC9104885A
:10051000F589E02D199561E07AE0CE0101960F94FE
:100520008112CE0101960E941BCACE0101960F9442
:10053000701287E090E00E94F5B287E090E00E94A0
:10054000FFB263EE74E28BE09FE00F9457161092B7
:10055000070F1092060F80E090E19093020F8093B6
:10056000010F84E890E09093090F8093080F81E0D9
:100570008093030F82E780930A0F85EF9EE00E942D
:10058000E2D985EF9EE00E9448DA88EC90E026965A
:100590000FB6F894DEBF0FBECDBFDF91CF911F9194
:1005A0000F9108956F927F928F929F92AF92BF9218
:1005B000CF92DF92EF92FF920F931F93CF93DF932F
:1005C000CDB7DEB7AE970FB6F894DEBF0FBECDBF86
:1005D0008091520A9091530A892B09F460C6809148
:1005E0003A1181115CC680913A118F5F80933A1164
:1005F00066ED72E28BE09FE00F9457168BE09FE070
:100600000F94EB140091520A1091530A67E678E0B8
:10061000C8010E94F6AD90934111809340116DE6A0
:1006200078E0C8010E94F6AD90935D0A80935C0A61
:100630006CEF79E0C8010E94F6AD90933D11809374
:100640003C1164E778E0C8010E94F6AD9093370B47
:100650008093360B009749F1DC011696ED91FC91E1
:10066000309719F120852F702530F9F462EC72E291
:100670008BE09FE00F9457168091360B9091370BCB
:100680000E9439AF8093350B4AE050E0682F8BE031
:100690009FE00F940E158BE09FE00F94EB14E09118
:1006A000360BF091370B868197819093340B8093B2
:1006B000330B0E94C16869E778E08091520A9091FB
:1006C000530A0E94F6AD9093C10A8093C00A009726
:1006D00009F4B2C00E9439AF082F10E001151105CE
:1006E00009F4AAC0000F111F000F111F8091BE0A4C
:1006F0009091BF0A892B09F08EC07801013811054D
:100700001CF040E8E42EF12CC7010F94983C909324
:10071000BF0A8093BE0AE092BD0A10922E11109279
:100720002D111092320B1092310B10922C1110924D
:10073000301110922F11C70101960F94983C90939D
:1007400032118093311190932B1180932A118E0DC9
:100750009F1D90932511809324110E94DEC1609308
:10076000261170932711809328119093291190E0FE
:1007700080E0E0913111F0913211E80FF91F108201
:100780000196E816F906ACF782E090E090932E11FE
:1007900080932D118091310B9091320B009741F095
:1007A00061E00E94A7BD60E08091310B0E9479BD9D
:1007B00080E98093C9001092C8001092CD0083E0B8
:1007C0008093CC008EE08093CA00F0924302E092C6
:1007D0004202209131113091321180914202909168
:1007E0004302820F931F9093251180932411232B92
:1007F00009F45FC062E572E28CEB9FE00F9457163C
:10080000B7018CEB9FE00E940BB38BE992EE9093C3
:1008100023118093221168EA72E28BE09FE00F942B
:1008200057164AE050E0B8018BE09FE00F94F815AE
:100830008BE09FE00F94EB146FE778E08091520A11
:100840009091530A0E94F6AD8C01009709F471C093
:100850000E9439AF882309F46CC06FEF680FC8019C
:100860000E94A8AEFC01E184F284909120119923AA
:1008700059F0809170008E7F80937000109220114B
:1008800010923E0210923D0282E180933C0291114F
:100890000F94B72BC7010F94DF2B01E010E0E01697
:1008A000F10674F060E0C8010F94132C0F5F1F4F26
:1008B000F6CF6BE372E28CEB9FE00F947B16A5CF33
:1008C0006DE272E28CEB9FE00F9457160E946A383B
:1008D000AB01BC012AE030E08CEB9FE00F940615E1
:1008E0008CEB9FE00F94EB146CE872E28BE09FE0DE
:1008F0000F9457164AE050E0B7018BE09FE00F9449
:10090000F8158BE09FE00F94EB1466E872E28CEB35
:100910009FE00F9457160E946A38AB01BC012AE091
:1009200030E08CEB9FE00F9406158CEB9FE00F946A
:10093000EB140091520A1091530A63E878E0C80161
:100940000E94F6AD9093560A8093550A6AE878E0C3
:10095000C8010E94F6AD9093431180934211892BF8
:1009600009F448C080914411811144C0809135112F
:1009700090913611892B09F0DFC167E072E28CEBB0
:100980009FE00F9457168CEB9FE00F94EB148FE0D1
:1009900090E00F94983C8C0188E1D80111968C93DB
:1009A000119712961C9212971C921E961C921E92E0
:1009B0001D970E948EB81093361100933511012BAC
:1009C00009F08CC068EF71E285E19FE00F94571643
:1009D00085E19FE00F94EB1480E0817080934411D7
:1009E00080914411882331F066E772E28BE09FE04A
:1009F0000F9457161092381110923711E091401150
:100A0000F0914111309709F4CCC2C680D780009193
:100A10004011109141110115110509F4BBC2C11417
:100A2000D10409F4B7C2F60180858F70853099F73B
:100A3000C6010E9439AF823070F3A801B601CE0121
:100A400001960E94C4E7CE0101960E94A7E3882385
:100A5000E1F18C859D85009709F40DC2DC01ED91D3
:100A6000FC910284F385E02D1995892B49F08C8542
:100A70009D85DC01ED91FC910084F185E02D1995B7
:100A80008C859D85DC01ED91FC910680F781E02D40
:100A90001995892BD1F0CE0101960E94DDE68823BD
:100AA00041F040E051E060E070E0CE0101960E942C
:100AB0003FE58F819885892B41F040E052E060E06E
:100AC00070E0CE0101960E943FE5D6011296CD90CE
:100AD000DC90CE0101960E94B6E799CF0E948EB8B5
:100AE00080913511909136110F94412C8EE09DE04C
:100AF0000F94F32D811189C069ED71E28BE09FE0C5
:100B00000F947B1680913511909136110F94922F8E
:100B1000E0913511F091361181E08083809135119B
:100B2000909136110F94A02F65EC71E2811102C0F3
:100B300060EB71E28CEB9FE00F947B168091421189
:100B400090914311892B09F447CF809133119091F3
:100B50003411892B09F0E2C083E190E00F94983CB6
:100B60008C0180913511909136112BE033E0F80122
:100B7000328B218B968385831482108289E0818356
:100B800081E08283838310933411009333110E9498
:100B9000DEC16B017C01F0E1CF0EF7E2DF1EE11C4C
:100BA000F11CD8011596ED91FC9116978FEF838774
:100BB000148613821482158216821782108611867B
:100BC000128614961C92BB24B394BE01605E7F4FC4
:100BD000F801858196810F947A3018160CF099C02F
:100BE0000E94DEC16C157D058E059F0508F091C041
:100BF000DE01909698E080E0915039F1ED91E82780
:100C0000F0E0E65CF04D8491F7CF0E947F2980915F
:100C10003511909136110F94412C8EE09DE00F9488
:100C2000F32D81110BC063E971E28BE09FE00F941B
:100C300057168BE09FE00F94EB1480CF67E771E2CB
:100C400085E19FE00F947B16C7CE9FA19813BDCF7F
:100C5000D8018C91811138C015968D919C910F947B
:100C6000A02FBE01605E7F4FF801858196810F94B1
:100C7000732F40E064EBD80115968D919C910F94F1
:100C80004D2FF80185809680C4010F94D12EC401A8
:100C90000F94412C67E88EE09DE00F94051060E80A
:100CA0008EE09DE00F9405100E94FAB8C4010F94E5
:100CB000D12EA82ED80115968D919C910F94A02F1E
:100CC000A5FC02C0F801B082AE014F5F5F4FBE01CC
:100CD000605E7F4FC8010F94E12FD8011196AC9050
:100CE00088A1803109F4DDC2BE01605E7F4FC8017A
:100CF0000F9450308A1510F5F8018181D8011196B2
:100D00008C93119714968C9114978F5F14968C93F3
:100D10005CCFE0913311F09134111282E0914211D5
:100D2000F0914311E680F7803FE7D32E8091421186
:100D300090914311892B71F481E04FCE88A18031CD
:100D400011F48CE0DBCFBE01605E7F4FC8010F94D1
:100D50005030D4CFE114F10479F3BE01605E7F4FCF
:100D6000F701808191810E94F639882329F360E69A
:100D700071E28CEB9FE00F945716D7016D917C9137
:100D80008CEB9FE00F9441168CEB9FE00F94EB14DB
:100D90000091331110913411AE014F5F5F4FBE01CE
:100DA000605E7F4FC8010F943630882309F45EC01F
:100DB00088A1803109F45AC0DD82F80185819681CD
:100DC0000F94A02FBE01605E7F4FD80115968D91C4
:100DD0009C910F94732F40E06EE4F8018581968119
:100DE0000F944D2F40E06B81D80115968D919C9109
:100DF0000F944D2F40E06C81F801858196810F940E
:100E00004D2F88A1803141F040E06D81D8011596C9
:100E10008D919C910F944D2FF801858196810F94AF
:100E2000A02FBE01605E7F4FD80115968D919C91D9
:100E30000F94732FF801408168E4858196810F94A7
:100E40004D2F64E170E080E090E00E94ECBFD8019B
:100E50008C91882331F06AE070E080E090E00E949D
:100E6000ECBFF801858196810F94A02FD7011296CF
:100E7000ED90FC905BCF70E060E0CE0101960E94A7
:100E8000EBE48C01912C812C97FF06C01195019504
:100E9000110988248394912CCE0101960E94DDE6ED
:100EA000E82EF12C8B85853091F0863009F00DCE3F
:100EB000B02E61E0802F0E94A7BD61E0892809F46F
:100EC00043C0EA94EF2809F043C060E041C0EF2836
:100ED00029F462E0CE0101960E94BEE640E051E0B6
:100EE00060E070E0CE0101960E943FE58F81988519
:100EF000892B41F040E052E060E070E0CE010196C5
:100F00000E943FE561E0802F0E94A7BD60E0802F36
:100F10000E9479BD6EE672E28CEB9FE00F9457164B
:100F20004AE050E0B8018CEB9FE00F94F81569E6B9
:100F300072E28CEB9FE00F94571667E672E28CEB3F
:100F40009FE00F945716C1CDEA94EF2809F0BDCF6A
:100F5000E62EF12C8B2D0E9479BD62E672E28CEBBD
:100F60009FE00F9457164AE050E0B8018CEB9FE0E9
:100F70000F94F81560E672E28CEB9FE00F94571621
:100F80004AE050E0B7018CEB9FE00F94F8156EE556
:100F900072E2D5CFF80186819781909338118093C2
:100FA00037118CEB9FE00F94EB146CE471E28BE053
:100FB0009FE00F9457168BE09FE00F94EB14E091A5
:100FC0003C11F0913D11309709F4B0C080913A1175
:100FD0008F5F80933A11068117815E01F8E2AF0EB0
:100FE000B11C8DE5682E84E0782E95E7892E94E07B
:100FF000992E0115110509F494C0D80118968C9109
:101000008F70863009F06BC019A708A770E060E008
:10101000C5010F94CC098DA59EA5892B09F45FC04D
:101020008091520A9091530A892B09F458C0E8A480
:10103000F9A4E114F104C1F1F70180858F708630C5
:1010400099F5F9A2E8A270E060E0CE0180960F94D5
:10105000CC09EDA1FEA110821182128213826AEAEC
:1010600076E0C7010E94F6AD0097F1F0DC0118961A
:101070002C9118972F702530B9F41696CD90DC90EE
:10108000C114D10489F0DA82C982B701CE01019678
:101090000F94CC09EE81FF8110821182128213829B
:1010A000F601C280D380ECCFEDA5FEA5108211829F
:1010B000128213828AA5843068F462E0823008F0DC
:1010C00060E08BA50E94A7BDEDA5FEA58181807F74
:1010D000818305C08630E1F038F4853081F0D80195
:1010E00012960D911C9185CF803439F060E08234E6
:1010F000B1F78BA50E94A7BDF2CF62E0FACFBC8208
:10110000AB829A828982CE0101960E947027E7CF36
:10111000BC82AB827A826982CE0101960E94452808
:10112000DECF80913A11815080933A116FE371E2E2
:101130008BE09FE00F94571667E371E28BE09FE02E
:101140000F94571681E02091401130914111232BCB
:1011500009F480E00E94D6656EE271E28BE09FE0C8
:101160000F94571681E020913C1130913D11232BB3
:1011700009F480E00E94D6656FE171E28BE09FE0A8
:101180000F94571664E171E28BE09FE00F945716BD
:1011900081E02091550A3091560A232B09F480E012
:1011A0000E94D6656DE071E28BE09FE00F945716C8
:1011B00081E02091330B3091340B232B09F480E034
:1011C0000E94D66564E071E28BE09FE00F945716B1
:1011D00081E02091421130914311232B09F480E0EA
:1011E0000E94D6656BEF70E28BE09FE00F9457167C
:1011F0008091590A0E94D6658BE09FE00F94EB1412
:1012000066EF70E28BE09FE00F9457160E946A38F9
:10121000AB01BC012AE030E08BE09FE00F940615A3
:101220008BE09FE00F94EB1481E08093380B8AED04
:101230009EE00F941023882351F08AED9EE00F94D6
:10124000C82984E090E090933F1180933E118091F3
:101250003E1190913F11079731F484E090E0909314
:101260003F1180933E1180913A11815080933A1141
:101270008091380BAE960FB6F894DEBF0FBECDBF8F
:10128000DF91CF911F910F91FF90EF90DF90CF9062
:10129000BF90AF909F908F907F906F90089580E067
:1012A000E9CFBCE0BA1508F427CD4BCD8F929F92C1
:1012B000AF92BF92CF92DF92EF92FF920F931F9364
:1012C000CF93DF93CDB7DEB7CF55D1090FB6F894E2
:1012D000DEBF0FBECDBF8C016B016115710519F02A
:1012E0004115510579F564E779E18CEB9FE00F94A6
:1012F00057166BE679E18CEB9FE00F945716B80117
:101300008CEB9FE00F94411669E679E18CEB9FE04E
:101310000F9457168CEB9FE00F94EB14C15ADF4FDC
:101320000FB6F894DEBF0FBECDBFDF91CF911F91F6
:101330000F91FF90EF90DF90CF90BF90AF909F9074
:101340008F900895460F571FDA011C920E946A3849
:101350004B0163E679E18CEB9FE00F9457164AE06E
:1013600050E0B4018CEB9FE00F94F81560E679E152
:101370008CEB9FE00F945716B8018CEB9FE00F9415
:1013800041166DE579E18CEB9FE00F945716BAE3B7
:101390008B16B1E09B064CF460E579E185E19FE0B6
:1013A0000F94571685E19FE0B7CF6EE479E18CEB9F
:1013B0009FE00F945716B6018CEB9FE00F944116F7
:1013C0006CE479E18CEB9FE00F9457168CEB9FE077
:1013D0000F94EB141A821982FE0133968EE3DF011B
:1013E0001D928A95E9F780913E1190913F110597E2
:1013F00091F563E070E0C8010E94D0697C01892BFF
:10140000D1F5E091380DF091390D808180FF86CFC4
:1014100061E070E0C8010E94D069892B09F47ECF99
:1014200064E270E0C8010F94314B892B09F076CF4C
:101430006EE279E18CEB9FE00F945716B8018CEBCC
:101440009FE00F9441168CEB9FE00F94EB14C801C2
:101450000E94C9BC63CF61E070E0C8010E94D069FE
:101460007C01892B09F465C04FE350E0B801CE013F
:1014700001960F94224BA12CBB24B394E00EF11ED5
:1014800065E279E1C7010F94D13E892B09F45EC072
:1014900064E270E0C8010F94314B892B09F03ECF14
:1014A000B11003C0AA2009F439CF409140115091E6
:1014B0004111B701CE018F5B9F4F0E942CE7CE01F7
:1014C0008F5B9F4F0E94A7E3182F882359F0B60126
:1014D000CE018F5B9F4F0E94AAB411E01816190627
:1014E0000CF010E0CE018F5B9F4F0E94B6E71123F6
:1014F00009F414CF8981882309F410CF80913E111B
:1015000090913F11059709F409CF67E079E18CEBE1
:101510009FE00F945716BE016F5F7F4F8CEB9FE0EB
:101520000F9441168CEB9FE00F94EB14CE010196C3
:101530008FCF62E070E0C8010E94D0697C01892BE6
:1015400009F4ECCEAA24A394B12C98CFF601019013
:101550000020E9F73197EC19FD09329708F498CF8C
:10156000C8010E94C9BCB11003C0AA2009F4D6CE9C
:10157000F6018081882309F4D1CEC6010F94341A74
:10158000CDCE0F931F93CF93DF93CDB7DEB76F9779
:101590000FB6F894DEBF0FBECDBF2091520A309136
:1015A000530A232B09F4E6C020913A11022E000CB5
:1015B000330B82179307B4F460EF78E185E19FE085
:1015C0000F94571685E19FE00F94EB1480E06F961F
:1015D0000FB6F894DEBF0FBECDBFDF91CF911F9144
:1015E0000F9108956AED78E18CEB9FE00F94571608
:1015F0008CEB9FE00F94EB148091C20A8F5F809375
:10160000C20AE0914011F09141113097A1F1068199
:10161000178101151105C9F1D80118968C918F70A9
:10162000853029F5C8010E9439AF882301F1409126
:10163000401150914111F80160817181CE010196F4
:101640000E942CE7CE0101960E94A7E3882359F05F
:101650008C859D85009739F0DC01ED91FC9100842B
:10166000F185E02D1995CE0101960E94B6E7F801AB
:1016700002811381CECF6AEC78E18CEB9FE00F946E
:1016800057168CEB9FE00F94EB14109238111092C8
:10169000371162EC78E18CEB9FE00F9457168CEBDE
:1016A0009FE00F94EB1464E670E080E090E00E940D
:1016B000ECBF1092590A1092380B6AEA78E18CEB71
:1016C0009FE00F9457160E946A38AB01BC012AE0D4
:1016D00030E08CEB9FE00F9406158091520A9091B8
:1016E000530A009711F00E9453B91092530A1092B6
:1016F000520A10923D1110923C1110924111109219
:10170000401110925D0A10925C0A1092370B1092F1
:10171000360B1092340B1092330B10925B0A10921E
:101720005A0A1092350B1092C10A1092C00A1092F8
:101730004311109242111092560A1092550A65EA0E
:1017400078E18CEB9FE00F9457160E946A38AB014A
:10175000BC012AE030E08CEB9FE00F9406158CEB87
:101760009FE00F94EB1410922F0B8091C20A8150CE
:101770008093C20A81E02BCF4F925F926F927F924B
:101780008F929F92AF92BF92CF92DF92EF92FF9291
:101790000F931F93CF93DF93CDB7DEB7C659D1090F
:1017A0000FB6F894DEBF0FBECDBF8E010F5B1F4F8B
:1017B000D8011D921C92FE01ED5BFF4F8EE1DF010F
:1017C0001D928A95E9F78091E70E9091E80E892B9A
:1017D00009F4FEC10E9449AF882309F4F9C1A09120
:1017E000E70EB091E80E52961C921E9251975496B5
:1017F0001C921E92539784E890E01D969C938E93C2
:101800001C971E961C921E9782E755968C935597AF
:10181000ED91FC9111970088F189E02D60E270E074
:10182000CD0119954FE150E0B8018091E70E9091FC
:10183000E80E0E949EAF7C018091E70E9091E80E29
:10184000DC01ED91FC910488F589E02D1995E114F6
:10185000F10409F4BDC1F801EE0DFF1D1082809165
:10186000F40E1F928F938091F30E1F928F938091AD
:10187000F20E1F928F938091F10E1F928F938091A1
:10188000F00E1F928F938091EF0E1F928F938DE831
:1018900098E09F938F931F9280E48F93FE0131967F
:1018A0006F01FF93EF930F943C4B6DEF75E28BE06C
:1018B0009FE00F945716B8018BE09FE00F944116FC
:1018C000B6018BE09FE00F9441168BE09FE00F94F0
:1018D000EB147E01F1E6EF0EF11CD70113961C927A
:1018E0001E92129788EE93E0A0E0B0E0F7018483A7
:1018F0009583A683B78384E084878BEE94E09183FD
:10190000808316861586108B0787128A118A80E5D8
:1019100090E0948B838B178A65E175E28CEB9FE0F6
:101920000F94571669EE7EE0CE0187589F4F0F94B3
:101930007812BE0167587F4F8CEB9FE00F944916D9
:101940008CEB9FE00F94EB14CE0187589F4F0F94C0
:1019500070126CEB78E0CE0185579F4F0F94811287
:101960006CEB78E0CE0187589F4F0F948112BE0137
:1019700067587F4FCE018D579F4F0F94781240913B
:10198000ED0E5091EE0E6091E90E7091EA0ECE01CF
:101990008D579F4F0F949C110FB6F894DEBF0FBE6A
:1019A000CDBF811105C0CE018D579F4F0F940112FD
:1019B000C157DF4F48815981CF58D040C557DF4FBD
:1019C00068817981CB58D040CE018D579F4F0F94BD
:1019D0009C11811105C0CE018D579F4F0F940112AC
:1019E000BE016D577F4FCE018F569F4F0F947812D7
:1019F000CE018D579F4F0F947012CE0187589F4F85
:101A00000F947012CE0185579F4F0F9470128EEB7A
:101A100098E0CD57DF4F99838883C358D040C9578A
:101A2000DF4F19821882C758D040C757DF4F19823D
:101A30001882C958D040CF56DF4F88819981C1594B
:101A4000D040CB57DF4F99838883C558D04067EF8C
:101A500075E28CEB9FE00F9457160E946A38AB0139
:101A6000BC012AE030E08CEB9FE00F9406158CEB74
:101A70009FE00F94EB1464E670E080E090E00E9439
:101A8000ECBF87EC91E8D7011E969C938E931D972F
:101A900063E971E087EE93E00F94DB3F8C01892BC3
:101AA00009F4EEC083E090E00F94983CF80195872C
:101AB0008487DC011196FC92EE9212961C92C7016B
:101AC0000F941023882319F0C7010F94C829F70138
:101AD00061897289A388B4886115710509F48FC082
:101AE000CE0187589F4F0F949C16A501BE016758E1
:101AF0007F4FC7010F94782A181619060CF0BDC045
:101B0000D7011F96BC901F975096AC90DF92CF9252
:101B100080E795E29F938F931F930F930F946240FA
:101B2000DF92CF928BE695E29F938F931F930F9353
:101B30000F946240D8011C96ED91FC9181E0828364
:101B4000DF92CF9288E695E29F938F931F930F9336
:101B50000F946240D8011C96ED91FC911282AF92D5
:101B6000BF9282E395E29F938F931F930F930F94FD
:101B700062400FB6F894DEBF0FBECDBFB12C89E234
:101B8000C82E85E2D82EBB2D24E0B202F00111242C
:101B900083E890E08C0F9D1FE80FF91F80819181F1
:101BA0000097A1F12281338121153105C9F33F93BB
:101BB0002F939F938F93DF92CF921F930F930F9446
:101BC0006240B3940FB6F894DEBF0FBECDBFDBCF3B
:101BD00040E250E06FE276E2C8010F94083F61E115
:101BE00076E28BE09FE00F945716B8018BE09FE000
:101BF0000F9441168BE09FE00F94EB1430CE678575
:101C00007089A501C7010F94C32676CF8DE695E2B2
